:1000000000800020BD01000025CA0000DDC90000FD
:10001000DDC90000DDC90000DDC90000DDC9000048
:10002000DDC90000DDC90000DDC9000025CA0000EF
:1000300025CA0000DDC90000A5C00000A9C100005C
:1000400025CA000025CA000025CA000025CA0000F4
:1000500025CA000025CA000025CA000025CA0000E4
:1000600025CA000025CA000025CA000025CA0000D4
:1000700025CA000025CA000025CA000025CA0000C4
:1000800025CA000025CA000025CA000025CA0000B4
:1000900025CA000025CA000025CA000025CA0000A4
:1000A000E1A50000EDA5000025CA000025CA00005A
:1000B00025CA000025CA000025CA000025CA000084
:1000C00025CA000025CA000025CA000025CA000074
:1000D00025CA000025CA000025CA000025CA000064
:1000E00025CA000025CA000025CA000025CA000054
:1000F00025CA000091EA000025CA0000BDEB0000FF
:1001000025CA0000FDD3000025CA000025CA000052
:1001100025CA000025CA000025CA000025CA000023
:1001200025CA000025CA000025CA000025CA000013
:1001300025CA000025CA000025CA000025CA000003
:1001400025CA000025CA000025CA000025CA0000F3
:1001500095C20000A9C20000BDC20000D1C20000CB
:1001600025CA000019D7000025CA000025CA0000D2
:1001700025CA000025CA000025CA000025CA0000C3
:1001800025CA000025CA000025CA000025CA0000B3
:1001900025CA000025CA000025CA000025CA0000A3
:1001A00025CA000025CA000025CA000025CA000093
:1001B00025CA000025CA000025CA0000564B4CF293
:1001C000205210B51A804DF628121A8000BF00BFC9
:1001D0000CF02CFC514B4FF010621A60504A9A60A0
:1001E000504ADA60504A136813F4807304D14F49BF
:1001F0000B604FF4A85313604D4B1A78110703D5C9
:100200001A7842F008021A704A4B4B492A221A7097
:100210004A4A4B4B8B4204D252F8040F43F8040B6A
:10022000F8E7484B484900228B4202D243F8042B9E
:10023000FAE74649464A002352F8230041F82300D2
:1002400001336F2BF8D1434B434A802103F8011B44
:100250009342FBD1414B3D4A1A60414B8A221A70AE
:10026000A3F5805324225A70A0221A709A7992071B
:10027000FCD59A79D406FCD43A4A937903F00C035E
:10028000082B384BF9D103221A7140225A719A79FE
:100290009006FCD5334A9179324B4906FBD5324A58
:1002A000324911600221516020221A709A7902F0BD
:1002B0000C020C2AFAD12E4B2E4A1A602E4B2F4AD2
:1002C0001A6000225A60072243F8042C2C4AC3F813
:1002D0000C2D62B60CF05AFF144B1B68DA0705D5DB
:1002E00028480CF027FD284B284A1A60284B1B7819
:1002F0005B0609D5244C254B22689A4204D121483B
:100300000CF018FD002323600FF012FF0CF094FB9B
:100310000CF0C2FAFEE700BF0E200540308004401A
:10032000823F04000100002B10D0034014D0034092
:1003300002D0074000E00740949BFF1F3C390100BA
:100340004088FF1F949BFF1F98A3FF1F0082FF1F81
:100350000000000000E400E05FE400E008ED00E0E1
:100360000050064000400640448004400000030165
:1003700004800440C010050014E000E0FF76010096
:1003800000002020D049145F1CE00340A5C3945A0C
:1003900000F00740FFFFFFFFFFFFFFFFFFFFFFFF32
:1003A000FFFFFFFFFFFFFFFFFFFFFFFFFFFFFFFF5D
:1003B000FFFFFFFFFFFFFFFFFFFFFFFFFFFFFFFF4D
:1003C000FFFFFFFFFFFFFFFFFFFFFFFFFFFFFFFF3D
:1003D000FFFFFFFFFFFFFFFFFFFFFFFFFFFFFFFF2D
:1003E000FFFFFFFFFFFFFFFFFFFFFFFFFFFFFFFF1D
:1003F000FFFFFFFFFFFFFFFFFFFFFFFFFFFFFFFF0D
:10040000FFFFFFFFFFFFFFFFFFFFFFFFDEF9FFFF23
:1004100010B5054C237833B9044B13B10448AFF33E
:1004200000800123237010BD949BFF1F000000007B
:1004300040390100084B10B51BB108490848AFF31B
:1004400000800848036803B910BD074B002BFBD0A0
:10045000BDE81040184700BF00000000989BFF1F38
:1004600040390100949BFF1F0000000038B504468E
:10047000104621700A491D460FF03CFC01464FF022
:100480007E500FF0EBFC07490FF034FCE560606034
:10049000256165610CF00AFEE061204638BD00BFB1
:1004A000DB0FC9400024744938B50446104621705A
:1004B00009491D460FF01EFC01464FF07E500FF01B
:1004C000CDFC06490FF016FCE560606025616561B2
:1004D0000CF0ECFDE06138BDDB0FC940002474492D
:1004E00038B503780446032B20D8DFE803F01A1848
:1004F0001002C16840690FF0F3FA0D4905466068C3
:100500000FF0ACFC014628460FF0A8FC38BD0849A6
:1005100040680FF0A3FCE1680FF0ECFB38BDC06849
:1005200038BDC16840690FF0DBFA38BD002038BD26
:100530000024744970B504460E460CF0B7FD05461C
:10054000E069281A0FF082FBE3682361E5616661C8
:10055000A061014660680FF081FC0146A060104870
:100560000FF07CFC0EF052FF0EF0F2FB0FF064FA7D
:10057000054601464FF07E500FF0B2FA61690FF068
:10058000B9FB2169064628460FF0B4FB0146304608
:100590000FF0A8FAE0602046BDE87040FFF7A0BF6A
:1005A000000080BF38B50E201C4C0CF04FF821889D
:1005B0001B4B884205461A881DDA0023511AB1F5F3
:1005C000805FAABF1B03C3EB03330131142093FBED
:1005D000F1F10CF0C1FB134B1988F1B923889D424E
:1005E00010DAC3F57F630F33282091FBF3F1BDE8E8
:1005F00038400CF0B1BB9042D4BFC1EB0003C1EB5B
:100600000203DBE740F6FF718D42D4BFC3EB050167
:10061000C3EB0101C1EB0131E3E738BD7E9CFF1F55
:10062000329EFF1FE89DFF1F10B504460BF010FE21
:10063000204610BD70B44C88A04220D9012301335C
:10064000DBB21CB2660031F8144084421D46F6D37A
:10065000A04211D005F10045013D965B31F815101F
:1006600032F81530401AF21A00FB02F0641A90FBBF
:10067000F4F4E01870BC7047905B70BC70470226C1
:100680000125E5E700280CDA064A434282FB0320F5
:10069000DA17C2EB600000EB4000A3EB8000C0F172
:1006A0000C007047ABAAAA2A2DE9F0470C200BF0EA
:1006B00099FF0C200CF04EFCBB4914200CF05AFCA6
:1006C000BA49BB4809F092FC022103200CF0E8FC77
:1006D000022104200CF0E4FC022105200CF0E0FCD7
:1006E000022106200CF0DCFC01210A200CF0D8FCD1
:1006F000012109200CF0D4FC01210D200CF0D0FCCC
:10070000012128200CF0CCFC012114200CF0C8FCA5
:10071000012116200CF0C4FC172001210CF0C0FCB4
:1007200004200CF0AFFC00283BD005200CF0AAFC04
:10073000054600283CD0002528469E4C207006F037
:10074000CDFE24784CBB284608F0DEFA9A4B9B4934
:100750001B889B4D098829709A4A9B4EA3F5AF715F
:1007600040F23A7303FB01F382FB0312DB17A3EBA6
:100770006213323301210D2033600CF07DFC6420C4
:100780000CF0B6FC4FF416710A200CF0E5FA5D216E
:100790008E4809F0D5FF90B9FEE7BDE8F04709F0B3
:1007A00035BB06200CF06EFC0028BED10125C4E745
:1007B00003200CF067FCB0FA80F04009BDE764202C
:1007C0000CF096FC21460A200CF0C6FA4FF4967104
:1007D00009200CF0C1FA5C217D4809F0B1FF00B995
:1007E000FEE764200CF084FC214609200CF0B4FAEA
:1007F0004FF4967116200CF0AFFA5B21754809F0A2
:100800009FFF00B9FEE764200CF072FC2146162021
:100810000CF0A2FA4FF4967117200CF09DFA6420A8
:100820000CF066FC214617200CF096FA64200CF0C0
:100830005FFC21460D200CF01FFC674A67481268D8
:10084000DFF8E8A1DFF8A091654EDFF8E481654F9D
:1008500000230121FFF728FE0123C9F8004034607E
:10086000C8F800408AF8003004240F200CF032FE53
:10087000D8F8003003440E20C8F800300BF0E6FE34
:10088000D9F800309AF800200344C9F80030152048
:10089000002A78D00BF0DAFE33681844306004F098
:1008A000010080F0010005F06BFB3B88002B14BFBA
:1008B0004B20DC200CF01CFC013CD6D1D8F80030D9
:1008C000D9F80020484930683C88DFF868E1474F94
:1008D000002BB8BF0333002AB8BF033292100A605E
:1008E0004349444A098812880028B8BF03309B1046
:1008F000801030605E1A19443E60CEF800103E4F02
:100900003E4E3F49C8F80030C2EB000E0244C7F823
:1009100000E032600B605CB94FF4FA7005F040FB08
:1009200005F02AFB07F0CEF84FF4AF600CF0E0FBC7
:10093000344B012404201C600CF0A4FB10B9324B92
:1009400028701C70314B1B881C2B23D0304C04F1B9
:10095000C80523200BF07AFE44F8040F01200CF0A8
:10096000C7FBA542F5D12B4A2B4B1078187008F025
:10097000D5F805F0FDFA45F6BF5228492848BDE8EC
:10098000F0470BF01BBC11200CF0A4FD3368184499
:10099000306084E7234B18880028D7D0224BC0B2A0
:1009A000197808F003F8D1E7001B3746801A0600D3
:1009B000A090FF1FF09BFF1F2C9EFF1F429EFF1F5A
:1009C0004C9CFF1FB5814E1B008AFF1FEC9BFF1F35
:1009D0007C9CFF1F209CFF1F2489FF1FAC9DFF1FD5
:1009E000B09BFF1FDA9DFF1FCC9BFF1F049EFF1FC4
:1009F000128AFF1F5C89FF1F149CFF1F509CFF1F62
:100A0000449EFF1F0C9EFF1FDB9BFF1F129EFF1FBC
:100A1000889CFF1F9C9DFF1F779DFF1FA505000061
:100A2000249EFF1F549CFF1F0E9CFF1FA09DFF1FB5
:100A3000009EFF1F7C9DFF1FF0B40E8886420DD2E2
:100A400003F10043013B31F81350854202D9F0BC59
:100A5000FFF7F0BD32F81300F0BC70471088F0BC0F
:100A6000704700BF094B1B880C2B09D8084A80B27D
:100A700052F8232028B143F6FE73984203D9108C14
:100A80007047108870470349FFF7D4BDE89BFF1FEC
:100A900060140100FC150100374A38491088384AB3
:100AA000F8B5384B12881B68834248DB9342A8BFD5
:100AB000134698420B60C8BF002342DD101AB0F500
:100AC000804FAABF9B03C3EB8333013093FBF0F04D
:100AD000FFF7C8FF2C4B2D4F1C883B68C0F3C61591
:100AE00005FB04F47F2CA8BF7F249D42064608D056
:100AF000274B1B88002B38D1264B1B88002B30D16D
:100B00003D60254D2B689E4205D0214B1B885A1F06
:100B1000032A1DD92E60214D2B689C420ED0204BFC
:100B2000188848B11A4B1F4A1B88D35C834203D0F4
:100B3000C0B2E1B207F03AFF2C60F8BDF8BD034641
:100B400008609A42D4BFC0EB0203C0EB0303B5E7D1
:100B5000144AD05C2030C0B206F07F0107F026FFB7
:100B6000D8E7284607F096FFCAE70E4A2946D05C28
:100B700007F01CFFC0E700BF7E9CFF1FB89BFF1F54
:100B8000329EFF1FE49DFF1FD09BFF1F2C9CFF1F69
:100B9000D09DFF1F769CFF1F3C9EFF1F789CFF1F70
:100BA000DE9DFF1F048AFF1F2DE9F04F012089B051
:100BB0000CF090FCAF4B186000200CF08BFCAE4B9F
:100BC000AE4A1B8810600C2B00F03B81AC4BAD4A49
:100BD00019880093AC4B52F8214000221A70AB4B9D
:100BE000AB4D1B88AB4A2E88013B32F91370002EA7
:100BF0005CD0A94BA94A1B88A9491278013B31F95D
:100C00001380002A40F0DF8011200CF063FCA54B1C
:100C10000193D3F800A00646B24540F3DF80A24B13
:100C2000DFF8A4921B88A14A012BD9F80030B2F852
:100C300000B09F4A02922046C8EB030800F09A8257
:100C40000FF004F8029A52F82B100FF053F80146F7
:100C500000200EF045FF0FF013FACAEB0802B04572
:100C6000B8BFB0469042CAEB080880F2968200FBFB
:100C70000888013298FBF2F08E4BDFF85082029325
:100C8000D8F80030034403EBD3735B10C8F800308E
:100C90002B88012B12D1884BDFF834B20393874B9A
:100CA000DBF8005004934FF0000A47E07D4B0193BE
:100CB000DFF814927F4BDFF8148202937E4B03938C
:100CC0001D460F200CF006FC2B689842824641DA44
:100CD000754A1288012A00F01D82744A0593128811
:100CE000734D049220460EF0B1FF049ADFF8E0B194
:100CF00055F82210DBF800500EF0FCFF01460020F2
:100D00000EF0EEFE0FF0BCF9EF1B059B5745A7EB6D
:100D10000302B8BF5746FF1A9042BABF013200FB28
:100D20000777474397FBF2F7D8F80020634B04930B
:100D3000BB1803EBD3735B10C8F80030604B1B8803
:100D4000013B032B00F2B082DFE813F06301A9013D
:100D5000C4008601594B04931B68984240F3C2813A
:100D6000514A1288012A00F0A682504A079311883E
:100D70004F4A0691204605920EF068FF059A0699A3
:100D8000DFF84CB152F82110DBF800500EF0B2FF42
:100D90000FF076F9079B2F445745A7EB0302A8BF36
:100DA0005746FF1AD8F800309042BABF00FB0777C9
:100DB0000132474397FBF2F73B4403EBD3735B10DD
:100DC000C8F80030BAE715200BF040FC354B019312
:100DD000D3F800A00646B2453FF721AF354B02934A
:100DE000D3F800A0B24580F289812F4BDFF8D8906C
:100DF0001B882E4A012BD9F80030B2F800B02C4ADB
:100E000003922046984400F070820EF01FFF039A70
:100E100052F82B100EF06EFF0FF032F9B045CAEB0E
:100E20000802A8BFB046CAEB08089042B6BF00FB54
:100E3000088800FB08F8013298FBF2F0DFF88C809C
:100E40001EE7204B1B78002B3FF4C0AE0C4B0D4A25
:100E5000198800930C4B52F8210001221A700EF0F1
:100E6000F5FE4FF07C510EF045FF0FF009F90446F6
:100E7000B5E600BF1C9CFF1F129EFF1F509EFF1F68
:100E8000229CFF1F8889FF1FC29BFF1F108AFF1F24
:100E9000889DFF1F44190100608AFF1FA09DFF1F4E
:100EA000B4150100149CFF1F629CFF1FE49BFF1FF1
:100EB0005C190100509CFF1F049EFF1F7C9DFF1FBB
:100EC0005E89FF1FDA9BFF1FB09BFF1F189EFF1F4D
:100ED000009EFF1F28460EF0B9FEB2490EF00AFF31
:100EE000054650460EF0B2FEAF490EF003FF014634
:100EF00028460EF0F7FD0FF0C3F80546CBF800507A
:100F0000D9F800000EF0A2FEA6490EF0F3FE074647
:100F100030460EF09BFEA4490EF0ECFE014638462A
:100F20000EF0E0FD0FF0ACF8C9F800009F4AA04BAE
:100F3000168819889F4AA04B12681B889F4FC6EBE2
:100F4000050E3544039EC6F800E0461A084404998D
:100F50000D6001990E6002993E8808609A4280F205
:100F600089810025C3EB060E954974450F6880F210
:100F70007681611C9F4205FB01F50EF1010E95FB88
:100F8000FEF5C0F2BE81BE42A8BF3E46F61A01FB86
:100F900006F494FBFEF49A4200F33681BB42C0F2A1
:100FA0003381884C20680EF051FE87490EF0A2FE76
:100FB00086490EF097FD0FF063F8A0F5FF531C3B38
:100FC000082B98BF4FF40050D8F800301844002880
:100FD0002060C0F24281B0F5804F80F252817C4B9C
:100FE0001B781BB1B0F5005F40F05381794D2B7831
:100FF000002B40F05481784D20682B68714C98424A
:1010000004D080B207F0B0FD23682B6009B0BDE8C2
:10101000F08F28460EF01AFE70490EF06BFE054662
:1010200050460EF013FE6E490EF064FE014628464F
:101030000EF058FD0FF024F80546CBF80050D9F813
:1010400000000EF003FE65490EF054FE07463046E0
:101050000EF0FCFD62495FE728460EF0F7FD5A49A5
:101060000EF048FE054650460EF0F0FD5D490EF0CC
:1010700041FE014628460EF035FD0FF001F8054609
:10108000CBF80050D9F800000EF0E0FD4E490EF00C
:1010900031FE074630460EF0D9FD52493CE728465E
:1010A0000EF0D4FD50490EF025FE054650460EF0D8
:1010B000CDFD4E490EF01EFE014628460EF012FDF3
:1010C0000EF0DEFF0546CBF80050D9F800000EF018
:1010D000BDFD45490EF00EFE074630460EF0B6FD4A
:1010E000424919E7D8F80030DFF810B103EBD373A9
:1010F0005B10DBF80050C8F800301FE6DFF8008115
:10110000DFF80091D8F8003003EBD3735B10C8F818
:101110000030BDE5364A06931188364A05912046CF
:101120000492DFF8D8B00EF091FD049A0599DBF82F
:10113000005052F821100EF0DDFD0EF0A1FFEF1B64
:10114000069B5745A7EB0302B8BF5746FF1AD8F8CE
:1011500000309042BABF013200FB0777474397FB4C
:10116000F2F73B4403EBD373234A04925B10C8F8B5
:101170000030E3E50EF06AFD029A52F82B100EF0F3
:10118000B9FD0EF07DFFCAEB0802B045B8BFB0460E
:101190008242CAEB08083FF76AAD00FB08F898FBEB
:1011A000F2F069E5CDCC4C3FCDCC4C3E128AFF1F0E
:1011B0005C89FF1F1C9CFF1FE09DFF1F009CFF1F01
:1011C000509EFF1FBC89FF1F9A99193FCDCC4C45FB
:1011D000069FFF1F749CFF1F2089FF1F3333733F3F
:1011E000CDCC4C3DCDCCCC3E6666663FCDCCCC3D27
:1011F000E49BFF1F5C1901007C9DFF1F009EFF1FE9
:10120000189EFF1FB09BFF1F009B1B88002B3FF405
:10121000C8AE2B1B002BB8BF5B42092B47DD05F581
:1012200000500130001B0EF011FD3B493B4C0EF00D
:1012300061FD054620680EF009FD39490EF05AFDA2
:10124000014628460EF04EFC0EF01AFFD8F800308A
:10125000184400282060BFF6BEAE002213E09F4273
:1012600005FB04F5B8BF002195FBFEF54BDA91FBB9
:10127000FEF490E6B242D4BFC3EB0205C3EB060511
:1012800070E643F6FF72274B22601B78002B3FF479
:10129000ADAE04F071FE244B01221A70ABE604F0EF
:1012A00067FE00232B70A6E6D9F800003EE64FF457
:1012B00000501A4C88E61D491D4A069320460D88A9
:1012C00005920EF0C3FC059ADFF868B052F82510BD
:1012D000DBF800500EF00EFD014600200EF000FC81
:1012E0000EF0CEFE2F44069B56E50EF0AFFC039A9F
:1012F00052F82B100EF0FEFC014600200EF0F0FB21
:101300008AE51E4642E6B742D4BFC3EB0701C3EBF2
:10131000060104FB01F1AAE7CDCCCC3EBC89FF1F3E
:101320009A99193F069FFF1F749CFF1FE49BFF1FA4
:101330005C190100009EFF1F08B5244B1B88FBB100
:10134000234B1B78FBB1234B1B78E3B1224B1B785B
:10135000CBB1224B1B78B3B1214B22481A78C2B9CA
:10136000214A22490088128809680244B1EB620FC1
:1013700009DD01221A706420BDE8084004F010BEA7
:10138000174A117801B908BD1370BDE8084007F08D
:10139000B5BB154A16490088128809680244B1EBAA
:1013A000620FF0DD00221A7007F0A8FB642004F041
:1013B000F7FD642004F0F4FD642004F0F1FD4FF427
:1013C0001670BDE808400BF093BE00BF8A9DFF1F5A
:1013D0002E9EFF1F2F9EFF1F309EFF1F319EFF1F5F
:1013E000E69BFF1F009CFF1FE09DFF1F1C9CFF1F33
:1013F000509EFF1F38B5114C232025780BF026F99D
:101400000F4A42F82500131F02F1C400002253F8CE
:10141000041F83420A44FAD123780A4907480A4C38
:101420000133DBB2322B81FB025108BF0023D217FC
:10143000C2EB21120370226038BD00BFD29BFF1F98
:101440008C9CFF1F1F85EB51FC9DFF1F2DE9F04F6A
:10145000B84CB94D2068B94F83B00EF0F7FBB849CE
:101460000EF048FC064610200CF034F80EF0EEFBAF
:10147000B4490EF03FFC31460EF034FB0EF000FE96
:101480002988206088423B8843DA9E465B1A7F2B7E
:101490004FF0000247DDD2015E1C92FBF6F2AA4E2D
:1014A000DFF8C882B6F800C0C8F80020BCF1190FF8
:1014B00000F0DF80BCF11A0F00F01781BCF11E0FA5
:1014C00000F020810126B146A04A1288002A00F0CF
:1014D0009D808842C0F207817045D4BFC1EB0000F7
:1014E000C1EB0E009A42BABF02FB00000133504329
:1014F00090FBF3F3964A1360964B1888C0B9964A4E
:101500001288AAB9954B197801B11A7003B0BDE8D9
:10151000F08F9842D4BFC1EB0002C1EB03029E469C
:101520005B1A7F2BB7DCC2EBC21292FBF3F2B6E779
:101530002988D4F800E0DFF80082DFF8F8A17145CF
:101540006CDCDFF818C29CF80020002A2ED14FF086
:10155000010B04288CF800B028D1002E40F09481B3
:101560007D4B18880028D1D0B9F1000FCED0236868
:101570002C883A88A34280F265810023141B7E2CBC
:10158000774DD5BFC3EB8313C3EBC3135B000134AB
:1015900093FBF4F42B680134A34203D0C0B2E1B250
:1015A00007F004FA2C6003B0BDE8F08F012800F0CA
:1015B000F680022800F0EB800328D1D1694B1B880C
:1015C000092BCDD0002ECBD023682E883A88B34289
:1015D00080F27B810023961B7E2EDFF88CA1D5BF85
:1015E000C3EB8313C3EBC3135B00013693FBF6F627
:1015F000DAF800300136B34203D0F1B24A2007F0E6
:10160000D5F9CAF80060ABE716469146BCF11E0F4B
:101610007FF472AF0022DFF858817EE04F4B1A78DA
:10162000002A3FF473AF002401281C7000F0A4804E
:10163000022840F00E81002E00F0A3804A4D2B6856
:10164000002B00F09E800420214607F0AFF9424BAA
:101650002C60188800283FF459AFB9F1000F3FF40F
:1016600055AFC0B2002107F0A1F93D4B00221A602E
:101670004CE7DFF8FC8098F80020C2B1DFF8D89082
:10168000B9F800A0BAF1000F11D0DFF8E89099F88E
:1016900000B0934578D05FFA8AF07F2107F086F991
:1016A00098F80030B6F800C089F8003010E0DFF894
:1016B000C49099F800A0924566D0274B0021187875
:1016C00007F074F998F80030B6F800C089F80030D7
:1016D0001E4B1A88002A97D0BCF11E0F40F00681DD
:1016E0000026B14619E00020FCE6DFF8848098F877
:1016F0000020002A0BBF012600264FF000094FF002
:101700000109E1E6DFF86880104B98F800601A885C
:10171000B6FA86F676094FF0000998F80030002BEB
:101720003FF4E8AE2988B7F800E02068C1EB0E036B
:10173000CFE600BF109CFF1F969DFF1F8C9DFF1FD3
:101740009A99193FCDCCCC3E129EFF1F389EFF1FA9
:10175000849CFF1F1A9CFF1F1E9EFF1F179EFF1FCA
:10176000F49BFF1FD09DFF1F889CFF1FF89DFF1F4C
:10177000DA9BFF1FD69BFF1F1EB1614D2B68002B0C
:101780007BD1604B188865E70026B1469CE6002EA9
:101790003FF4E6AEDFF868A1DAF800202EE0002E74
:1017A0003FF4DEAEB7F80080F045D4BFC1EB0802CD
:1017B000C1EB0E02C1EB0808B8F17E0FDFF840A1C3
:1017C000D5BFC2EB8212C2EBC212520008F101086F
:1017D00092FBF8F8DAF8002008F10108424506D03B
:1017E0005FFA88F10120009307F0E0F8009B188869
:1017F000CAF8008002287FF4DFAE42462168B5F8BF
:1018000000803888414559DA0021C8EB0008B8F15A
:101810007E0FD3BFC1EB8111C1EBC11108F10108EB
:10182000490091FBF8F808F10108904506D05FFAED
:1018300088F10420009307F0B9F8009B1888CAF8D3
:101840000080B9E69342D4BFC4EB0303C4EB0203A8
:1018500094E6032827D12C4B1B88092B91D0002E0E
:101860008FD0274D2B68002B8BD04A20214607F0C4
:101870009DF8244B2C601888ECE6214607F096F87A
:10188000204B2C601888E5E640207F218DE80C0075
:1018900007F08CF8019B009A188858451CD0022844
:1018A0007FF48AAE76E704287FF46BAF002E3FF416
:1018B00068AF2146402007F079F862E78142D4BF43
:1018C000C8EB0101C8EB00019FE79342D4BFC6EB10
:1018D0000303C6EB02037EE6B8F80010DAF800E076
:1018E000B7F800808E45FFF665AF5DE72988B7F849
:1018F00000E020680026C1EB0E03B146E9E500BF19
:10190000889CFF1F1E9EFF1FD09DFF1F08B50F4B19
:101910001B88022B0FD0032B12D0042B03D00C4BAF
:1019200001221A7008BD7F21092007F03FF8084BFB
:1019300001221A7008BD7F21412007F037F8EEE739
:101940004021092007F032F8E9E700BF829CFF1F21
:101950003E9CFF1F38B51C4B1B881D2B26D01B4BF4
:101960001B88012B25D01A4A1A4B14881B681A4A67
:10197000A342128818DB9342D4BFC4EB0303C4EB29
:101980000203141B7F2CC6BFDB010134C3EBC3135E
:1019900093FBF4F4114D2B689C4203D0E1B2052077
:1019A00007F004F82C6038BD0023EAE70C4B1C88D4
:1019B000F0E70C4B0C4A0D491B6812680C689B1A27
:1019C0001C1B84F30704E5E7129EFF1F889DFF1F81
:1019D0003A9CFF1FC89BFF1F109EFF1FBC9BFF1F51
:1019E0000E9CFF1F449EFF1F2889FF1F989DFF1F0D
:1019F00010B50F4C23685BB90E4B1B88022B11D01E
:101A0000033B012B09D90C4A00231370236010BD3E
:101A10000021052006F0CAFFEEE70021092006F0AC
:101A2000C5FFF0E70021412006F0C0FFEBE700BF53
:101A3000BC9BFF1F829CFF1F3E9CFF1F08B5274BCE
:101A40001B78ABB115200AF001FE254A254B128800
:101A500018601D2A15D0244A1288EAB1012A25D01F
:101A6000224B1B78002B34D0BDE80840FFF7C0BFE5
:101A700011200BF02FFD1A4A1A4B128818601D2AEC
:101A8000E9D11B4B1B78002BEAD0184B1B780BB30A
:101A9000BDE80840FFF75EBF164A1288002ADFD073
:101AA000154A1B6812889A42DADCEEE70F200BF029
:101AB00011FD104B114A1B88106033B1104B114AB5
:101AC0001B6812689B1A9842DFDD084B1B78002BBD
:101AD000CAD108BDFFF71AFFDAE700BFA09DFF1FBC
:101AE000129EFF1FC89BFF1F889DFF1F3E9CFF1F6C
:101AF000DA9BFF1F829CFF1F3A9CFF1F989DFF1FD0
:101B0000449EFF1F2889FF1F2DE9F04FA64C227825
:101B1000012A95B000F02582C0F0ED81022A00F084
:101B2000C980A248DFF81CE390F80080A048A14DCE
:101B3000A14FA24EA24BA3490390A3480290A348F1
:101B40009EF800B000902D78A1483F7896F800E00C
:101B50001B780978DFF8F4C2DFF8F492DFF8F4A21A
:101B60000190012A94BF013200222270994A9A48BA
:101B700013709A4A80F800B015709948994A077016
:101B800082F800809848994A03701170BEF1000FE6
:101B900040F0FF80964A10880D2800F09D81954CFA
:101BA00000202070024604462DB19148008800288C
:101BB00040F09E810546904806882544002E40F05E
:101BC0004B818E488E4C009E007836782478013008
:101BD000A0EB4600002C40F02C82019C94F800E021
:101BE000CEEB0004BEF1000F40F04F820026DFF87C
:101BF00050E202989EF800E00078A41BA4EB4E048B
:101C00003C44CBEB040410B1B7FA87F040099CF8D0
:101C100000602718BC1B1EB11EF1000618BF01266C
:101C200099F800009AF80090039FC6EB040EC0EBF1
:101C30000E00A0EB4900804497F800C0714FC3EB41
:101C40000803A3EB41010C2313FB0C1139606E4B0D
:101C50006E4C6F4E1B886F482488376800886E4E24
:101C6000033B03EB4303C4EBC40401EB83033C4499
:101C700003440C3B56F824001D4405440AB1674B4D
:101C80001960674B1A68954200F02281654A6648E0
:101C90001168079107990160126808926348089AD1
:101CA00000881D60521A824284BF614A156015B0D7
:101CB000BDE8F08F5F4F08AE0025E9B25E4808F03E
:101CC00003FD57F8043B0135C01A0C2D46F8040BF0
:101CD000F3D15A4B3D4D00953D4DB3F800C00195F1
:101CE000109D09980F99464EDFF8D0A0DFF8C490F8
:101CF000DFF8CC80654511AA8CCAAE46ACBF4FF068
:101D0000000E4FF0010E8445D4BF0020012030703A
:101D10008C452E480B9D254E8AF800E0D4BF00214B
:101D20000121017094452A4921480390D4BF002223
:101D300001220A709C45424A23480290D4BF0023E6
:101D40000123BC45AB46D4BF002701271370AC4527
:101D5000194B0C9D1F70D4BF4FF0000B4FF0010BBF
:101D6000384B227883F800B0AC45DFF858C098F8BB
:101D700000309CF8001096F80080DFF8D0C0DFF843
:101D8000D4A0D4BF0025012589F80050DFF8C09009
:101D9000E7E62D4A174814880122182C027040F2F9
:101DA0005081002400E700BF769DFF1FCC9DFF1FE0
:101DB000819DFF1F569EFF1F3C9CFF1F5B9EFF1FC8
:101DC000CD9DFF1FCE9DFF1F649CFF1F219EFF1F07
:101DD000229EFF1F559EFF1F949DFF1F579EFF1FB2
:101DE000589EFF1F599EFF1F5A9EFF1F169EFF1FE2
:101DF0005C9EFF1FDA9BFF1FC09BFF1F148AFF1F03
:101E0000489EFF1FD49DFF1FEC9DFF1F089EFF1FD4
:101E1000849CFF1FD49BFF1F74170100089CFF1FA9
:101E2000349CFF1F449FFF1F249CFF1F1C9EFF1F0D
:101E30004C9EFF1F2C89FF1F7C9CFF1F2C9EFF1FA9
:101E4000239EFF1F3D9CFF1F129EFF1F549EFF1FDE
:101E5000149EFF1F159EFF1F012E00F07F81022E92
:101E600000F0DE81032EA14B00F014811E78009B50
:101E70009CF800E01878029B99F800C093F8008065
:101E8000019B9AF800401F78A6EB4E03A4EB840454
:101E9000CCEB030CC0EB80760CEB0403C0EB8600AC
:101EA000034403EB480303EB810327B1904909780E
:101EB000002940F05D82012603998E480978C1F11E
:101EC000060101EB4101334403EB81010160BEE6F1
:101ED00089498A4A0968DFE6002D3FF460AE884AE6
:101EE000884E14880122182C327040F2AA80744661
:101EF000A0F10D055FE6844F08AE0025E9B28348E6
:101F000008F0E2FB57F8043B0135C01A062D46F8ED
:101F1000040BF3D17E4A7F4B039216461B880D9A21
:101F200000219A423170C0F299800C997A4A8B4212
:101F3000CCBF01210021117040F3E1817749784A3B
:101F400091F80080774B11780398774A0292052226
:101F50001B78DFF8FCC1DFF8FC91DFF8FCA1027010
:101F600057E0724F08AE0025E9B2714808F0ACFBAB
:101F700057F8043B0135C01A0C2D46F8040BF3D179
:101F8000644B0C9D1F88684B02930B9B0A98099A1F
:101F9000089EDFF8C4A1DFF8BC910F99DFF8B0C14B
:101FA000BB42ACBF4FF0000E4FF0010EAF42D4BFAA
:101FB000002501258742109B8CF80050D4BF0020DB
:101FC00001209742D4BF00220122B742D4BF4FF074
:101FD00000084FF001088AF800209F42514A89F812
:101FE0000000D4BF002301234C481370129A80F8DC
:101FF00000808F424C4E4A4886F800E0D4BF002152
:102000000121974201703ADC00224A48404D039575
:1020100002704948494A4A4E4A4D07784A4800905A
:102020004A4892F800E096F800B02D7822780190A6
:1020300097E5019C46B12678002E40F05D81441E54
:10204000D5E50C3C0122AFE594F800E00138CEEB79
:102050000004BEF1000F7FF4CAADC7E52F49304A36
:10206000304B91F8008011782F4A35701B7802921E
:10207000DFF8DCC0DFF8DC90DFF8DCA0C9E7119AFC
:102080009742D4BF00220122BFE7002E3FF4AEAD3D
:102090000126ACE51C780298009B9CF800601B7838
:1020A00090F800C099F8007001989AF8008090F8B4
:1020B00000E0A4EB4604E71BA8EB8800C3EB8374A5
:1020C0003844C3EB8403034403EB4C0303EB810369
:1020D000BEF1000F40F051810126039905480978AF
:1020E00033440C2414FB01310160B0E5148AFF1F56
:1020F000239EFF1FD49DFF1F249CFF1F449FFF1F93
:10210000129EFF1FDA9BFF1F488AFF1FEC9BFF1FD9
:10211000819DFF1F2C9EFF1F319EFF1FCC9DFF1F27
:10212000CE9DFF1FCD9DFF1F649CFF1F188AFF1FC0
:10213000209CFF1F069CFF1F3C9CFF1F5B9EFF1FF8
:102140003D9CFF1F569EFF1F219EFF1F229EFF1FCB
:10215000549EFF1F149EFF1F159EFF1FA74CDFF804
:10216000A8E2207805909EF8004000980494059C11
:10217000007800900134A4EB40040498002840F05B
:10218000AC80019890F800E00498261ACEEB060087
:102190000490BEF1000F40F09B8074460298984E68
:1021A00000780190049836780296041BA4EB46044C
:1021B00001983C44CBEB0404002800F08480B7FA7B
:1021C00087F040099CF800602044871B1EB10298EC
:1021D000061C18BF012699F800009AF80040BE1BA3
:1021E000301AA0EB440080440098C3EB0803A3EB33
:1021F0004103002864D1BEF1000F40F0C880734451
:10220000002C77D100290CBF00206FF00900039942
:102210007C4C097803440C2010FB0131216016E549
:10222000009C019E24780094774C367801969AF8A9
:10223000006094F800A0724C744899F800E094F89B
:1022400000909DF80440847080F806E080F80390C8
:102250009CF800C09DF80040DFF8D091DDF800E068
:1022600080F808800470077180F805C0C67141725B
:1022700080F801A04FF0000801200021634C0E46B9
:102280005FFA88FA4F46F44607E0022809D00A2987
:102290000BD014F801CF17F8010F844501F10101AB
:1022A000F3D101360A29F6B2F3D1092E00F28F805C
:1022B00008F10108B8F1100F45D019F80A0FDCE752
:1022C0004FF0000E9BE701987CE7CEEB04000490F2
:1022D0000098041C18BF012460E7009800285ED015
:1022E000019890F800E0BEF1000FEED1601E04905E
:1022F000744653E700208AE7841B012677E40B9994
:10230000434A8B42CCBF0121002111704CDC0A9959
:10231000404A8B42CCBF01210021117040F38E80D6
:102320003D493E4A91F800803D4B117803983D4A63
:10233000029203221B78DFF8F8C0DFF8F890DFF88C
:10234000F8A0027065E62D4837490478C86B0299F9
:10235000013409782044CBEB000008440021039BA2
:102360001C78284B401A0C2111FB040119606EE403
:102370001BF1000618BF01269EE5214909780029B6
:102380003FF4AAAE1BF1000618BF0126A5E602988D
:1023900000280CBF4FF0000E4FF0090E2FE70198F8
:1023A00090F800E03046F0E61B491C4A91F80080A6
:1023B0001B4B117803981B4A029204221B78DFF80A
:1023C00070C0DFF87090DFF870A0027021E60B4853
:1023D0001549047851F828000299013409782044FD
:1023E000CBEB00000844002BB8D0BAF1000FB5D1F8
:1023F000BBF1000FB2D00121B1E700BF148AFF1F6B
:10240000239EFF1FD49DFF1F489EFF1F589CFF1F48
:10241000309EFF1F2F9EFF1FCC9DFF1FCE9DFF1FD5
:10242000CD9DFF1F649CFF1FC089FF1F2016010068
:10243000549EFF1F149EFF1F159EFF1F0999184AE7
:102440008B42CCBF01210021117012DD1549164AC3
:1024500091F80080154B11780398154A02920222D8
:102460001B78DFF850C0DFF85090DFF850A0027002
:10247000CFE5089A0B49DFF83CC091F80080DFF8FF
:102480003890DFF838A09342074A084B1178084A81
:102490001B7802927FF7BDAD039801220270B8E568
:1024A0002E9EFF1FCC9DFF1FCE9DFF1FCD9DFF1FAA
:1024B000649CFF1F549EFF1F149EFF1F159EFF1F4D
:1024C0002DE9F04F3B4B1B788BB0002B6DD10E20CC
:1024D0000AF0BCF80DF0BAFB01463748374E384DCC
:1024E000FEF728F83448FDF7FBFF0DF0C9FD80F337
:1024F0000C003060FFF708FB2C68012C7CD0022C0C
:1025000000F09E82032C00F0AD832E4E33682E4ADD
:102510002E4E0993099B177830682D4C0721012214
:10252000181A11FB07229042236000F28482294E80
:1025300032689A1A0D2A00F27782274E32689A1A68
:10254000132A00F26C82254E32689A1A252A1AD96B
:10255000234B1B88002B40F05E81224B1B78002B05
:1025600040F05981FEF746FF1F4B1B881B3B9BB277
:10257000022B04D81D4B1B78002B40F04F8103F039
:1025800021FD236833601A4D2A689B1A502B00F2F4
:102590000582184B1B88012B00F01D8206F09AFA69
:1025A00006F0C8F80BB0BDE8F08F07F0B7FA0BB033
:1025B000BDE8F08FF09BFF1FAC9DFF1FE49DFF1F48
:1025C0000C9EFF1F449FFF1F789DFF1F909DFF1FC4
:1025D000A89DFF1F6C9CFF1F449CFF1F489CFF1F72
:1025E0008A9DFF1FE69BFF1F129EFF1FDA9BFF1FA6
:1025F000849DFF1FE89DFF1FDFF810939E4AB9F8E6
:1026000000001378834204D0C3B21846137006F05A
:102610009DF9DFF8F482994AB8F8003011789942B0
:1026200004D0974F3978002940F0C586954A336821
:102630001288954E9A42C0F2F680944A1278002A87
:1026400040F0F180DFF8C8A2BAF8003023B9904B0F
:102650001B88002B00F0F8848E4A8F4B11881B8852
:102660008E4A0B4412685B1093428D4A126880F2C6
:102670006E8400219342B4BF01230B460491009362
:10268000ACBF4FF0010B8B4605910E2009F0DEFF29
:10269000844B854A1B68176803930133A7F25232B3
:1026A000002B8446029240F39786802BA8BF80239C
:1026B0007E4A7F4912780191002A00F0BE80097895
:1026C000914200F0BA80B8F80010DFF83CE299427D
:1026D00001F06A806A49AEF80030764B4FF0010E87
:1026E00081F800E01978DFF82CE2019B8EF80010E9
:1026F0001A70009B002B00F00F81BAF80030002BFD
:1027000000F00A816C4B1B685A1C002A40F3688653
:10271000802A00F36486694C69496A4824880988DC
:1027200000682144B0EB610FC1F2AB82A3F1480213
:102730000F2A02D8473BA9F800300E2009F086FF87
:102740006FF454731F44874202DC5F4B00221A70FF
:102750005E4B1B88002B00F0F2835D4B5D4A1B78BB
:102760001178994240D0002B3ED05B490C78002C68
:1027700000F0E886594991F800C0BCF1000F40F024
:10278000DF86574F0097574F57480297544F0078AE
:1027900087F800C0534F4FF0010E87F800C081F852
:1027A00000E0002841F0768050490978002900F0C7
:1027B000A4874F4903910C460978002940F09A8775
:1027C0004C48484F0078397001210297217058B168
:1027D000434842490090002008700099029F087009
:1027E000039901243C7008701370434B1B88A3F1BC
:1027F0001B02012A40F2BA851D2B7FF487AE3D4FA4
:102800003B78002B41F00D803C4C2378002B40F0AE
:102810004B8423707AE6FEF78FFDA3E62B68012B2D
:102820007FF4ADAEADE63168354A0691069835497C
:10283000106002220B602A6004E71E49DFF8D4E032
:10284000097800293FF451AF9EF8000081423FF41F
:102850004CAF03984B2840F36E871833802BB8F8A1
:102860000000A8BF802398423FF43FAF2648038072
:1028700003480123037038E7779DFF1F4C9CFF1F1F
:10288000DB9BFF1F7E9CFF1F449FFF1FE69BFF1FDC
:10289000729CFF1F009CFF1FE09DFF1F1C9CFF1FE1
:1028A000509EFF1F089CFF1FCC9BFF1F409EFF1FD9
:1028B000309CFF1F419EFF1FD49DFF1F969DFF1F51
:1028C0008C9DFF1F109CFF1F809DFF1F9E9DFF1F63
:1028D000069CFF1FB49BFF1F589EFF1FDC9DFF1F20
:1028E000209EFF1F809CFF1F599EFF1F559EFF1FAC
:1028F000B59BFF1FDA9BFF1F129EFF1FD69BFF1F7A
:10290000409CFF1FA49DFF1F429EFF1F9C9DFF1F19
:10291000389CFF1F319CFF1F029B9C45BFF60DAFEB
:10292000AC4B1B88002B3FF408AFBBF1000F7FF4CA
:10293000E9AEA94B1B881BB1059B002B7FF4E2AECF
:10294000049B002B3FF4F9AEA44B1A78002A7FF4C5
:10295000F4AEDFF8049399F8004001221A70002CBD
:1029600040F03F839E4B1B78002B01F0F4879D4B7A
:102970001B78002B02F0D2829B4B1B78002B7FF43C
:10298000DCAE9A4B1B78002B3FF4D7AEB8F8003082
:1029900097490A3BA8F800300A70CEE604F0E6FD3D
:1029A000944B1B7873B9944B1B785BB9934B1B7892
:1029B00043B9934B1B782BB9924B1B7813B903F097
:1029C000D7FA01E003F0E0FA23682B608E4B1B88F6
:1029D000012B7FF4E3AD8D4A8D4B11688D481A7839
:1029E000A1F118032A2101FB03F10160002A00F084
:1029F0009082894A1368994200F32A8380F23483D3
:102A000086480068D0F17F0048BF03308010013055
:102A10001B1A994200F32883136019467BE2FFF7E3
:102A20000DF8236833608EE5FEF7BEF8FEF70EFD65
:102A30002368336081E5FEF72FF82368336076E57D
:102A4000774A34681288A24204DB6E4B1B78002B55
:102A500000F02583734E744833680793734B0799CE
:102A600000681B88091A994263D8002B61D0704B0B
:102A7000198800293FF44AAD6E4B6F481B680088E7
:102A8000A342B8BF23469A4241F3F1806B4B1A60D0
:102A9000DFF8C88188F800105C4FFDF7FDFF38684B
:102AA0007F2840F34985664B7F3883FB0032C3178C
:102AB000C3EB620303EB4303A0EB83007330614B72
:102AC00001931B883860002B40F05C864B4B0093D1
:102AD0001B78002B00F097835B4C2378002B00F0D1
:102AE0009283DFF87C91DFF858A14FF0000B0CE0E7
:102AF00003F17300C0B298F8001005F07FFF23784F
:102B00000BF1010B5B4540F37E833B6859F8040FE2
:102B10001844A0F17F038AFB0321DA17C2EB61029C
:102B200002EB42027F28A3EB8203E1DCFDF7AAFD62
:102B3000E0E7404B40491B6808883D49A342B8BFC5
:102B400023469A4200F392823C4C09888342A8BFF4
:102B50000346236000299BD19A42C8BF0B4640F32D
:102B60008C82801AB0F5804FAABF9B03C3EB8333DE
:102B7000013093FBF0F0FDF775FFC0F3C6100DF0C8
:102B800065F8324B044618880DF060F83049074666
:102B900020460DF0AFF8014638460DF0ABF821465F
:102BA0000CF0A0FF4FF07E5104460DF041FA0028D2
:102BB00041F05280274920460DF058FA002840F095
:102BC000638620460DF082FAC0B2DFF8908088F864
:102BD000000061E7729CFF1FA29DFF1F809DFF1FE9
:102BE000559EFF1F949DFF1F579EFF1F589EFF1F5E
:102BF000DB9BFF1F809CFF1FDC9DFF1F209EFF1F94
:102C0000B59BFF1FE69BFF1FE89DFF1F4C9EFF1F0C
:102C10003E9CFF1F349EFF1FE09BFF1FBC9BFF1FBE
:102C20007E9CFF1F449FFF1F409CFF1F709CFF1F47
:102C3000D89BFF1FA49DFF1F329EFF1FB89BFF1F45
:102C4000ABAAAA2A189CFF1F8489FF1FC49BFF1FE1
:102C5000CDCCCC3D0000FE42819DFF1F659CFF1F37
:102C60005C89FF1FC04B34681988A14253DDBF4BFC
:102C70001B78002B4FD1DFF8409399F800007F2894
:102C800040F3CB85A3F155337F3803F1004383FB39
:102C90000032C317C3EB620303EB4303A0EB8300D3
:102CA0007330B34B01931B88C0B289F80000002B2E
:102CB00040F0BD87AF4B00931B78002B00F06F8472
:102CC000AD4C2378002B00F06A84AC4FDFF8B4825F
:102CD0004FF0000A0AE003F17300C0B205F0B6FE3F
:102CE00023780AF1010A534540F3598457F8043F09
:102CF00099F800001844A0F17F0388FB0321DA173C
:102D0000C2EB610202EB42027F28A3EB8203E2DC0A
:102D1000FDF7B8FCE1E79A4F38687F2840F3B481AB
:102D2000984B7F3883FB0032C317C3EB620303EB7E
:102D30004303A0EB83007330DFF87C9299F800A086
:102D4000824500F00782904B1B88002B43D18F4AAD
:102D50008F4812680088914205DC8242D4BFC1EBE3
:102D60000203C1EB0003411AB1F5804FA6BF9B03DC
:102D70000131C3EB833393FBF1F0FDF773FEC0F336
:102D8000C6100CF063FF834B044618880CF05EFFFE
:102D90008149804620460CF0ADFF014640460CF0CC
:102DA000A9FF21460CF09EFE4FF07E5104460DF027
:102DB0003FF9002840F0AB86784920460DF056F9DF
:102DC000002840F05E8520460DF080F9C0B2DFF8A3
:102DD000EC8188F80000BAF17F0F40F3A9836948BD
:102DE000AAF17F0A80FB0A304FEAEA73C3EB600066
:102DF00000EB4000AAEB800073305E4B00931B7821
:102E0000C0B289F80000002B40F00983644B0393A3
:102E10001B78002B40F0F584624B02931B78002B4B
:102E200040F01D87524B0193029B1B78FBB15E4B18
:102E30001B88012B00F0E985022B00F03F87032B54
:102E400001F0D080042B01F0F282052B01F06E839B
:102E5000062B01F04085072B01F05786082B02F066
:102E60000B80092B02F0D6800A2B02F01083009B06
:102E70001B78002B00F05184019B3D4C19880029E0
:102E800000F0A78438687F2840F3C6823D4B7F3826
:102E900083FB0032C317C3EB620303EB4303A0EBD6
:102EA000830073303860002940F05684009B1B7803
:102EB000002B00F05A81304C2378002B00F0558114
:102EC000DFF8B8A0DFF8F4804FF0000B0CE003F15E
:102ED0007300C0B298F8001005F090FD23780BF154
:102EE000010B5B4540F341813B685AF8040F254ACA
:102EF0001844A0F17F0382FB0321DA17C2EB6102C1
:102F000002EB42027F28A3EB8203E0DCFDF7BAFB71
:102F1000DFE7264B1960264B1B68A92202FB03F34F
:102F2000002BBCBF03F57F533F339B13543B194425
:102F300081F30C01282009F00FFFFFF72FBB194C7C
:102F40001C480C49164A237003700B704CE49342E2
:102F50004FF0000B80F29B800123CDF800B0CDF83C
:102F600014B00493FFF791BB7E9CFF1FE69BFF1FED
:102F7000189CFF1F209EFF1F8489FF1F5C89FF1F75
:102F80004C9EFF1FABAAAA2AD89BFF1FB89BFF1F0E
:102F9000329EFF1FC49BFF1FCDCCCC3D0000FE42E4
:102FA000B59BFF1F809CFF1F9E9DFF1FE09BFF1F87
:102FB000BC89FF1FDC9DFF1FD29DFF1F659CFF1F6B
:102FC000A94B1B78002B7FF4B8AB039BA74A243B8B
:102FD00083F34703D9B25B20136005F0E7FC99F84F
:102FE0000040032C30D1DFF8D88298F80030002B55
:102FF00042F08E819E4F3B78002B42F07C819A4CB0
:103000002378002B42F06A819A4B1B78002B42F008
:103010003D81994A1380994B1B78002B42F08481A3
:10302000974B7F221A8098F800306BB93B785BB9D8
:1030300023784BB9934A7F210720138005F0B6FC13
:103040007F210B2005F0B2FC8F4B1F68FFF775BB8B
:103050008E480068D0F17F0048BF033003EBA00327
:1030600001339942BFF6D8AC116054E7884B098808
:103070001A6000297FF40CAD13469842D4BFC2EB0E
:103080000003C2EB03036CE5FDF7FCFA54E60123F1
:10309000CDF810B0CDF800B00593FFF7F6BA0123D4
:1030A0002B607C4EFFF732BA7B4B6A20198805F003
:1030B00001FE3B782370FFF729BA029B1B78FBB116
:1030C000764B1B88012B00F01984022B00F07486CC
:1030D000032B00F0FD87042B01F08581052B01F007
:1030E0009B82062B01F00C84072B01F0B985082B7D
:1030F00001F07686092B01F0AE870A2B02F08C8155
:10310000019B1B88002B00F03083009B1B783BB990
:10311000039B1B7823B9029B1B78002B00F052877E
:103120005F4B1B78002B00F044815E490B78082B25
:1031300000F23F815C483A6800685C4C0133DBB2C6
:103140005F1E101A44F827000B70594B3468198819
:1031500089F800208C424F4E7FF7D8A93268554B32
:103160000892089A1A60FFF7D1B9039B1B78002BCD
:10317000A3D03B68A3F10C007F2840F331834E4875
:103180008B3B80FB0320DA17C2EB600000EB4000B2
:10319000A3EB800303F17300DFF82881C0B298F835
:1031A000001005F02BFC009B1B78002B85D03D4CBC
:1031B0002378002B81D0DFF810A14FF0000B0CE03A
:1031C00003F17300C0B298F8001005F017FC2378E3
:1031D0000BF1010B5B457FF770AF3B685AF8040FAA
:1031E000354A1844A0F18B0382FB0321DA17C2EBA6
:1031F00061020C3802EB42027F28A3EB8203DFDC82
:10320000FDF740FADEE7264B1B78002B40F0C18229
:103210003B682A4A1278002A7AD0A3F10C007F2852
:1032200040F3F882244A8B3B82FB0321DA17C2EB7E
:10323000610202EB4202A3EB820303F17300C0B20E
:1032400098F8001005F0DAFB009B1B78002B5ED08D
:10325000144C2378002B5AD0DFF86C90DFF858A07C
:103260004FF0000B3EE000BF589EFF1FFC9BFF1F6E
:10327000579EFF1F949DFF1F769CFF1F599EFF1FA7
:10328000D89BFF1FD09DFF1FCC9BFF1FBC9BFF1F28
:10329000B89BFF1F449FFF1F0E9CFF1F9E9DFF1F9B
:1032A000DC9DFF1F8489FF1FDC9BFF1F6089FF1FC0
:1032B0007E9CFF1FEC9EFF1FABAAAA2AB59BFF1F97
:1032C000559EFF1F659CFF1F5C89FF1F03F1730064
:1032D000C0B298F8001005F091FB23780BF1010BB8
:1032E0005B4514DD3B6859F8040F1844A0F18B03CB
:1032F0008AFB0321DA17C2EB61020C3802EB4202AF
:103300007F28A3EB8203E1DCFDF7BCF9E0E73B6833
:10331000B74A1278FAB1B74A1288012A00F0FA8344
:10332000022A00F0CA85032A00F05287042A01F01D
:10333000A380052A01F0DD81062A01F0FC82072A1C
:1033400001F03E83082A01F01B86092A01F0BA86A3
:103350000A2A02F02A80019A1288002A00F00B82C1
:10336000A54903220B702A60FFF7D0B8A34F3B7822
:10337000002B3FF449AAA24C207802F08DFEA14B0D
:103380001B78002B00F0658223887E2B00F261827F
:103390009D4A0133108899B22180002800F069828B
:1033A000C9B2C0B2994C05F001FB3B782370FFF71E
:1033B000ADB83A68C9E6DBB21846137005F0D4FA26
:1033C000934B94491A46944B184600230B703B705C
:1033D00013700370FFF72AB90123FFF769B980243E
:1033E0008E498F4B8F4A09881B8812680B44B2EBB9
:1033F000630FBFF6A2A9814B1B78002B40F0DA8146
:10340000B8F80030884AA3423FF497A9874B14804C
:1034100001221A70FFF791B9FDF734F942E5844BA8
:1034200001931B88002B42F0E2807B4B0393704B8F
:103430000293804C23786BB3DFF80882DFF8F8A1A1
:103440004FF0000B09E003F17300C0B205F0FEFA83
:1034500023780BF1010B5B451CDD58F8043F99F80C
:1034600000001844A0F17F038AFB0321DA17C2EBA6
:10347000610202EB42027F28A3EB8203E3DCFDF74B
:1034800001F9E2E75A4B029305F0E0FA009B1B7842
:10349000002BCED1039B1B78002B3FF4C5AC99F8D1
:1034A0000030A3F10C007F2840F3A88162488B3BD9
:1034B00080FB0320DA17C2EB600000EB4000A3EBB7
:1034C000800303F17300C0B205F0C0FA009B1B78C3
:1034D000002B00F08881574C2378002B01F01882D4
:1034E000DFF86081DFF850A14FF0000B0AE003F134
:1034F0007300C0B205F0AAFA23780BF1010B5B450B
:103500007FF792AC58F8043F99F800001844A0F1F6
:103510008B038AFB0321DA17C2EB61020C3802EB42
:1035200042027F28A3EB8203E1DCFDF7ABF8E0E782
:103530005046FDF7A7F860E4FDF7A4F8FFF7BFBA1F
:10354000002008703D49087840B131490091097860
:10355000002900F09C81009F0021397038490978CA
:1035600000297FF426A9002C40F0C780002840F0F5
:10357000C480224C264F94F800E0274C03941C4C46
:103580000294254C23492070194C0097087038701C
:103590002070BEF1000F7FF41EA9FFF725B91E4B66
:1035A0001B78002B70D099F80030A3F10C007F2815
:1035B00040F36A83204A8B3B82FB0321DA17C2EB7C
:1035C000610202EB4202A3EB820303F17300C0B27B
:1035D00005F03CFA009B1B78002B55D0154C237846
:1035E000002B51D0174FDFF850804FF0000A35E024
:1035F000809CFF1F9E9DFF1FD29DFF1FDA9BFF1F18
:103600000E9CFF1F5A9EFF1F549CFF1FD69BFF1F3F
:10361000209EFF1FDC9DFF1FB59BFF1F8C9DFF1F82
:10362000969DFF1F109CFF1F429EFF1FDB9BFF1FED
:10363000189CFF1F8489FF1FABAAAA2A599EFF1F4F
:10364000559EFF1F5C89FF1F03F17300C0B205F098
:10365000FDF923780AF1010A534515DD57F8043FB7
:1036600099F800001844A0F18B0388FB0321DA17B6
:10367000C2EB61020C3802EB42027F28A3EB82030B
:10368000E2DCFCF7FFFFE1E7894B1B78FBB1894BDC
:103690001B88012B00F02086022B00F01A87032BD9
:1036A00001F09480042B01F04D81052B01F07D8306
:1036B000062B01F01584072B01F04E85082B01F035
:1036C0004386092B01F03C870A2B01F01987019BE7
:1036D0001B88002B00F0A682774B1B78002B40F054
:1036E0009C82764B764A198834680020012310604A
:1036F0002B602FE503980021017072490978002999
:103700003FF472A86A4902910978002900F00787FE
:10371000029800210170FFF767B8039B1B78002B0C
:103720007FF4AAAB029B1B78002B7FF4A5AB019B17
:103730001988FFF7A7BB243B002BB8F8000040F323
:103740003B8498423EF4D1AF9BB25F48A8F800306A
:1037500001230370FEF7C9BFDFF87081C0B298F88B
:10376000001005F04BF9FFF7A1BB584B38781978DA
:1037700005F044F9C9E4D8B298F8001005F03EF914
:103780003B68EDE5C0B298F8001005F037F9FFF797
:103790009DB97F21402005F009F94D494D4A3B680C
:1037A0000B600021117034E54B4BDFF84CE11978C8
:1037B000FEF79BBF4B2C40F33E821834802CB8F8A8
:1037C0000030464AA8BF8024A3427FF41FAEFEF714
:1037D000B4BF99F8000005F039F92188FFF752BB12
:1037E000FCF750FFD8E4029B1B78002B7FF41FAB43
:1037F000039B1B78002B7FF43FAB98E7FCF742FF5D
:1038000061E6374B01931B88002B7FF43BAE284BBE
:10381000029344E6FCF736FF11E5FCF733FFFFF7B0
:1038200040BA304C207802F037FC2F4B1B781BB18C
:1038300023887E2B41F230802C4B1B7823B12388C8
:10384000284A002B41F05080294C3B782370FEF72A
:103850005DBE264B1B78002BF6D02388214A002B17
:10386000F2D02449013B088899B2118000287FF4E6
:1038700097ADC8B21E4C05F00DF93B782370FEF7EA
:1038800045BE7F20FFF7A3BA7F20FFF79EB9084F00
:10389000094902974FF0000C81F800C0009F02997F
:1038A0004FF0010E87F800E081F800C056E600BF37
:1038B000809CFF1F9E9DFF1FDC9DFF1F7E9CFF1FA6
:1038C000B89BFF1FDA9BFF1FDB9BFF1F659CFF1F41
:1038D000DC9BFF1F8489FF1F419EFF1F429EFF1F2D
:1038E000189CFF1F0E9CFF1F5A9EFF1F599EFF1F13
:1038F000D69BFF1F549CFF1F319CFF1FDFF8B0A316
:103900003868BAF80030E54AE54CC31A82FB031E5A
:10391000D917C1EB6E0101EB4101A3EB810303EB6E
:10392000430354F8233018447F2840F34A847F38F7
:1039300082FB0032C317C3EB620303EB4303A0EB2C
:1039400083007330DFF86C83DFF86CB398F80010F5
:10395000C0B205F053F8BBF80030022B7FF6D0ABB5
:103960003968BAF80030CD4ACB1A82FB030ED8175B
:10397000C0EB6E0000EB4000A3EB800303EB4303BE
:1039800004EB8303586808447F2840F3AA867F38F5
:1039900082FB0032C317C3EB620202EB4202A0EBD0
:1039A00082007330C0B298F8001005F027F8BBF819
:1039B0000030032B7FF6A4AB3968BAF80030B74A61
:1039C000CB1A82FB030ED817C0EB6E0000EB400051
:1039D000A3EB800303EB430304EB8304A0680844D8
:1039E0007F2840F357817F3882FB0032C317C3EB37
:1039F000620202EB4202A0EB8200733098F80010E2
:103A0000C0B204F0FBFFFFF77BBBDFF8A4A299F87C
:103A10000000BAF80030A14AA14CC31A82FB031E71
:103A2000D917C1EB6E0101EB4101A3EB810303EB5D
:103A3000430354F8233018447F2840F3C6837F386B
:103A400082FB0032C317C3EB620303EB4303A0EB1B
:103A500083007330DFF860B2C0B204F0F7FFBBF848
:103A60000030022B7FF603AA99F80010BAF8003054
:103A70008A4ACB1A82FB030ED817C0EB6E0000EB0C
:103A80004000A3EB800303EB430304EB830358687C
:103A900008447F2840F329867F3882FB0032C31711
:103AA000C3EB620202EB4202A0EB82007330C0B2B1
:103AB00004F0CCFFBBF80030032B7FF6D8A999F8AF
:103AC0000010BAF80030754ACB1A82FB030ED817E3
:103AD000C0EB6E0000EB4000A3EB800303EB43035D
:103AE00004EB8304A06808447F2840F3C7807F3834
:103AF00082FB0032C317C3EB620202EB4202A0EB6F
:103B000082007330C0B204F0A1FFFFF7B0B901200A
:103B1000FFF75DB9DFF898A16049BAF80020604C62
:103B20009A1A81FB020ED017C0EB6E0000EB40002A
:103B3000A2EB800202EB420254F8220018447F28D4
:103B400040F3BD83A0F17F0381FB0321DA17C2EBB1
:103B5000610000EB4000A3EB80007330DFF858B148
:103B600098F80010C0B204F049FFBBF80030022BF7
:103B700050D93968BAF80030484ACB1A82FB030E94
:103B8000D817C0EB6E0000EB4000A3EB800303EB03
:103B9000430304EB8303586808447F2840F31286EC
:103BA0007F3882FB0032C317C3EB620202EB420292
:103BB000A0EB82007330C0B298F8001004F01EFF32
:103BC000BBF80030032B25D93868BAF80030334AE7
:103BD000C31A82FB031ED917C1EB6E0101EB410131
:103BE000A3EB810303EB430304EB8304A3681844B2
:103BF0007F284CDD7F3882FB0032C317C3EB6202A3
:103C000002EB4202A0EB82007330C0B298F80010C1
:103C100004F0F4FE3B68FFF79EBB0021402004F057
:103C2000C5FE5EE599F8000004F010FF54E504F0CD
:103C30000DFFFFF73FB8243C002CB8F8003040F3EC
:103C4000BB85A3423EF479ADA4B2164BA8F8004060
:103C500001221A70FEF771BD0120FEF7B6BF124BAC
:103C600001931B88002B7FF40FACFFF7DDB80F4AE0
:103C70008342A8BF03461360FEF70ABFFCF702FDAC
:103C800040E71446FFF7B7BBFCF7FCFC9FE4FCF7EA
:103C9000F9FCBAE7FCF7F6FCB0E600BFABAAAA2A2B
:103CA00024150100DB9BFF1F189CFF1FB89BFF1F03
:103CB000D89DFF1F659CFF1FEE9BFF1FDFF818A319
:103CC00099F80000BAF80030C14AC24CC31A82FB0E
:103CD000031ED917C1EB6E0101EB4101A3EB810378
:103CE00003EB430354F8233018447F2840F3E88360
:103CF0007F3882FB0032C317C3EB620303EB43033D
:103D0000A0EB83007330DFF8D4B2C0B204F09EFEA3
:103D1000BBF80030022B7FF6AAA899F80010BAF879
:103D20000030AB4ACB1A82FB030ED817C0EB6E00F3
:103D300000EB4000A3EB800303EB430304EB83039E
:103D4000586808447F2840F3F2857F3882FB0032B0
:103D5000C317C3EB620303EB4303A0EB8300733091
:103D6000C0B204F073FEBBF80030032B7FF67FA8CF
:103D700099F80010BAF80030954ACB1A82FB030E6E
:103D8000D817C0EB6E0000EB4000A3EB800303EB01
:103D9000430304EB8304A06808447F287FF76EAFD9
:103DA0007F3882FB0032C317C3EB620303EB43038C
:103DB000A0EB83007330A5E6DFF81CA23868BAF8E0
:103DC0000030834A834CC31A82FB031ED917C1EB10
:103DD0006E0101EB4101A3EB810303EB430354F8B4
:103DE000233018447F2840F36E837F3882FB0032F3
:103DF000C317C3EB620303EB4303A0EB83007330F1
:103E0000DFF8DC81DFF8D4B198F80010C0B204F01C
:103E1000F5FDBBF80030022B7FF672A93968BAF8BD
:103E200000306B4ACB1A82FB030ED817C0EB6E0032
:103E300000EB4000A3EB800303EB430304EB83039D
:103E4000586808447F2840F36A857F3882FB003237
:103E5000C317C3EB620303EB4303A0EB8300733090
:103E6000C0B298F8001004F0C9FDBBF80030032B75
:103E70007FF646A93868BAF80030554AC31A82FB63
:103E8000031ED917C1EB6E0101EB4101A3EB8103C6
:103E900003EB430304EB8304A36818447F287FF7F4
:103EA000F9AE7F3882FB0032C317C3EB620303EB2A
:103EB0004303A0EB83007330A0E5DFF81CA1444965
:103EC000BAF80020434C9A1A81FB020ED017C0EBBF
:103ED0006E0000EB4000A2EB800202EB420254F8BD
:103EE000220018447F2840F3F182A0F17F0381FB78
:103EF0000321DA17C2EB610000EB4000A3EB800066
:103F00007330DFF8D8B098F80010C0B204F076FD36
:103F1000BBF80030022B7FF67DAE3968BAF800306E
:103F20002B4ACB1A82FB030ED817C0EB6E0000EBB6
:103F30004000A3EB800303EB430304EB83035868C7
:103F400008447F2840F3EF847F3882FB0032C31798
:103F5000C3EB620303EB4303A0EB83007330C0B2F7
:103F600098F8001004F04AFDBBF80030032B7FF6F0
:103F700051AE3868BAF80030154AC31A82FB031EE6
:103F8000D917C1EB6E0101EB4101A3EB810303EBF8
:103F9000430304EB8304A36818447F287FF777AEBC
:103FA0007F3882FB0032C317C3EB620303EB43038A
:103FB000A0EB8300733028E601283EF496AB012382
:103FC000FFF7C3BB99F8000004F040FDFFF7A8B865
:103FD000ABAAAA2A00180100D89DFF1FEE9BFF1F65
:103FE000659CFF1FDFF8E4A299F80000BAF80030E2
:103FF000B44AB54CC31A82FB031ED917C1EB6E013C
:1040000001EB4101A3EB810303EB430354F823309D
:1040100018447F2840F3DB817F3882FB0032C317CE
:10402000C3EB620202EB4202A0EB82007330DFF8C6
:10403000A0B2C0B204F00AFDBBF80030022B7EF63D
:1040400016AF99F80000BAF800309E4AC31A82FBF6
:104050000321DA17C2EB610202EB4202A3EB8203F7
:1040600003EB430304EB83035B6818447F2840F3AE
:1040700028847F380C2290FBF2F302FB130073308C
:10408000C0B204F0E3FCBBF80030032B7EF6EFAEC9
:1040900099F80000BAF800308A4AC31A82FB03215B
:1040A000DA17C2EB610202EB4202A3EB820303EBDD
:1040B000430304EB8304A36818447F287FF7DEAD35
:1040C0007F380C2290FBF2F302FB1300733019E5EA
:1040D000DFF8F8A13868BAF800307A4A7A4CC31A87
:1040E00082FB031ED917C1EB6E0101EB4101A3EB6B
:1040F000810303EB430354F8233018447F2840F333
:1041000063817F3882FB0032C317C3EB620202EB8C
:104110004202A0EB82007330DFF8B881DFF8B0B163
:1041200098F80010C0B204F069FCBBF80030022B14
:104130007EF6E6AF3868BAF80030624AC31A82FBEE
:104140000321DA17C2EB610202EB4202A3EB820306
:1041500003EB430304EB83035B6818447F2840F3BD
:10416000A7837F380C2290FBF2F302FB130073301D
:10417000C0B298F8001004F041FCBBF80030032BEB
:104180007EF6BEAF3868BAF800304E4AC31A82FBDA
:104190000321DA17C2EB610202EB4202A3EB8203B6
:1041A00003EB430304EB8304A36818447F287FF7E1
:1041B00071AD7F380C2290FBF2F302FB13007330D9
:1041C0001CE4FCF75FFAFFF7BDBBFCF75BFA41E4C8
:1041D000DFF8F8A03B49BAF800203B4C9A1A81FB63
:1041E000020ED017C0EB6E0000EB4000A2EB800285
:1041F00002EB420254F8220018447F2840F3EA8080
:10420000A0F17F0381FB0321DA17C2EB610101EB0F
:104210004101A3EB81007330DFF8B4B098F80010CF
:10422000C0B204F0EBFBBBF80030022B7FF6F2AC1F
:104230003868BAF80030234AC31A82FB0321DA1720
:10424000C2EB610202EB4202A3EB820303EB4303E6
:1042500004EB83035B6818447F2840F336837F3880
:104260000C2290FBF2F302FB13007330C0B298F8FB
:10427000001004F0C3FBBBF80030032B7FF6CAAC80
:104280003868BAF800300F4AC31A82FB0321DA17E4
:10429000C2EB610202EB4202A3EB820303EB430396
:1042A00004EB8304A36818447F287FF7F0AC7F38C1
:1042B0000C2290FBF2F302FB13007330A5E4FCF731
:1042C000E1F94BE4ABAAAA2A90180100D89DFF1F80
:1042D000EE9BFF1F659CFF1FDFF834A399F80000D9
:1042E000BAF80030C24AC34CC31A82FB0317D9176D
:1042F000C1EB670101EB4101A3EB810303EB430336
:1043000054F8233018447F286ADD7F3882FB00325E
:10431000C317C3EB620202EB4202A0EB82007330D0
:10432000DFF8F0B2C0B204F091FBBBF80030022B12
:104330007FF6CDA999F80000BAF80030AC4AC31A4C
:1043400082FB0321DA17C2EB610202EB4202A3EB0C
:10435000820303EB430304EB83035B6818447F2869
:1043600040F3B6827F380C2290FBF2F302FB13007D
:104370007330C0B204F06AFBBBF80030032B7FF649
:10438000A6A999F80000BAF80030994AC31A82FB2E
:104390000321DA17C2EB610202EB4202A3EB8203B4
:1043A00003EB430304EB8304A36818447F2814DD64
:1043B0007F380C2290FBF2F302FB13007330C0B283
:1043C00004F044FBFFF783B9FCF75CF9A4E6FCF7C3
:1043D00059F92CE6FCF756F91EE7FCF753F9EEE71E
:1043E000FCF750F99CE7DFF828A23868BAF80030EB
:1043F0007F4A814CC31A82FB031ED917C1EB6E01A1
:1044000001EB4101A3EB810303EB430354F8233099
:1044100018447F28D8DD7F3882FB0032C317C3EBF6
:10442000620303EB4303A0EB8300733074E6DFF811
:10443000E0A199F80000BAF800306D4A6E4CC31A3A
:1044400082FB031ED917C1EB6E0101EB4101A3EB07
:10445000810303EB430354F8233018447F28B6DD6F
:104460007F3882FB0032C317C3EB620303EB4303C5
:10447000A0EB83007330DAE5DFF894A15C49BAF869
:1044800000205D4C9A1A81FB020ED017C0EB6E0023
:1044900000EB4000A2EB800202EB420254F8220043
:1044A00018447F2896DDA0F17F0381FB0321DA17F2
:1044B000C2EB610000EB4000A3EB80007330ABE681
:1044C000FCF7E0F81FE4FCF7DDF899E4FCF7DAF814
:1044D00017E5DFF83CA199F80000BAF80030444A2B
:1044E000464CC31A82FB0317D917C1EB670101EBD6
:1044F0004101A3EB810303EB430354F82330184439
:104500007F287FF76DAF7F3882FB0032C317C3EB84
:10451000620303EB4303A0EB8300733000E73848EA
:104520000090384838490390FEF755B9DFF8E0A00D
:1045300099F80000BAF800302D4A344CC31A82FBB7
:104540000321DA17C2EB610202EB4202A3EB820302
:1045500003EB430354F8233018447F2840F3AE8123
:104560007F380C2290FBF2F302FB13007330DFF86C
:10457000A4B0C0B204F06AFABBF80030022B19D91B
:1045800099F80000BAF800300C22C11A91FBF2F33E
:1045900002FB131302FB03435B6818447F2840F3BC
:1045A00067847F3890FBF2F302FB13007330C0B2D4
:1045B00004F04CFABBF80030032B7EF658ACBAF886
:1045C000003099F800000C22C11A91FBF2F302FBB3
:1045D000131302FB0344A36818447F287FF74EABF4
:1045E0007F3890FBF2F302FB13007330FFF78ABAB7
:1045F000ABAAAA2A24150100141A01000018010010
:10460000209EFF1FB59BFF1FDC9DFF1FC0160100F2
:10461000D89DFF1FEE9BFF1FDFF898A33868BAF8FC
:104620000030DA4ADA4CC31A82FB0321DA17C2EBF4
:10463000610202EB4202A3EB820303EB430354F853
:10464000233018447F2840F336817F380C2290FBBA
:10465000F2F302FB13007330DFF85C83DFF85CB326
:1046600098F80010C0B204F0C9F9BBF80030022B72
:104670001AD93868BAF800300C22C11A91FBF2F34B
:1046800002FB131302FB03435B6818447F2840F3CB
:10469000EC837F3890FBF2F302FB13007330C0B25F
:1046A00098F8001004F0AAF9BBF80030032B7EF64E
:1046B00027ADBAF8003038680C22C11A91FBF2F32A
:1046C00002FB131302FB0344A36818447F287FF7FF
:1046D000E1AA7F3890FBF2F302FB13007330FFF77F
:1046E0008DB9FBF7CFFFFFF75DB9FBF7CBFFFFF706
:1046F000DEB9DFF8C0A2A549BAF80020A44C9A1A86
:1047000081FB0210D117C1EB600101EB4101A2EB6B
:10471000810202EB420254F8220018447F2840F341
:10472000B880A0F17F030C2093FBF0F200FB123065
:104730007330DFF888B298F80010C0B204F05EF968
:10474000BBF80030022B1AD93868BAF800300C22B6
:10475000C11A91FBF2F302FB131302FB03435B68E4
:1047600018447F2840F3B9837F3890FBF2F302FBB3
:1047700013007330C0B298F8001004F03FF9BBF892
:104780000030032B7FF646AABAF8003038680C22B6
:10479000C11A91FBF2F302FB131302FB0344A3685B
:1047A00018447F287FF773AA7F3890FBF2F302FB4F
:1047B00013007330FFF729BA012B3DF4BEAF01247B
:1047C000FFF743BAFBF75EFFFFF7F5B9DFF8E4A1A7
:1047D00099F80000BAF800306C4A6E4CC31A82FB9C
:1047E0000321DA17C2EB610202EB4202A3EB820360
:1047F00003EB430354F8233018447F2846DD7F3809
:104800000C2290FBF2F302FB13007330DFF8ACB123
:10481000C0B204F01BF9BBF80030022B19D999F88B
:104820000000BAF800300C22C11A91FBF2F302FB2F
:10483000131302FB03435B6818447F2840F3A380F3
:104840007F3890FBF2F302FB13007330C0B204F028
:10485000FDF8BBF80030032B7EF639AFBAF8003014
:1048600099F800000C22C11A91FBF2F302FB13131A
:1048700002FB0344A36818447F287FF7AEAD7F385E
:1048800090FBF2F302FB1300733098E5FBF7FAFE9E
:10489000BCE7FBF7F7FE4CE701339BB22380D9B2AC
:1048A00005203D4C04F082F83B782370FDF72EBEC6
:1048B000FBF7E8FE5CE4FBF7E5FECDE6FBF7E2FE86
:1048C00055E6FBF7DFFEFFF7DBBBFBF7DBFECDE4D6
:1048D000FBF7D8FE4DE5DFF8DCA099F80000BAF848
:1048E00000302A4A2D4C29E6013B9BB2D9B2052063
:1048F000294C138004F05AF83B782370FDF706BE6C
:10490000DFF8B0A03868BAF80030204A234C8AE6B5
:10491000029B1B78002B7EF48AAAFEF7ADBAFBF748
:10492000B1FEFFF79DBAFBF7ADFEFFF718BBFBF733
:10493000A9FEFFF715BADFF87CA01449BAF80020E9
:10494000164CDCE6DFF86CA099F80000BAF80030ED
:104950000E4A134C42E7134B1B78002B00F0CB821E
:10496000114B1B78002B7DF4E8AE104B1B78002B0D
:104970003DF4E3AEB8F800300D490A33A8F8003032
:104980000A70FDF7DABEFBF77DFE5FE7ABAAAA2A45
:10499000C016010090180100D69BFF1F841901006A
:1049A000141A0100949DFF1F579EFF1F589EFF1F62
:1049B000DB9BFF1FD89DFF1F659CFF1FEE9BFF1F0A
:1049C000A14C2288002A00F02283A049DFF88CB293
:1049D0000988BBF800000331884227DD9C489D49C7
:1049E0000088B1F800E0DFF870C2181A0C2190FBC3
:1049F000F1F901FB19004FF0900909FB0EFE01FBD4
:104A000000E06FF00B0E5CF8000003440EFB023078
:104A10007F2840F338857F3890FBF1F301FB1300CA
:104A20007330C0B298F8001003F0E8FFBBF8002024
:104A300023881344022B23DD854B864A38681B8864
:104A4000B2F800C0DFF810E2C31A0C2193FBF1F2B8
:104A500001FB1232902303FB0CF301FB023373447E
:104A60005B6818447F2840F3A2857F3890FBF1F300
:104A700001FB13007330C0B298F8001003F0BEFFC2
:104A8000BBF8002023881344032B23DD704B714AAD
:104A900038681B88B2F800C0DFF8BCE1C31A0C21EB
:104AA00093FBF1F201FB1232902303FB0CF301FBA9
:104AB000023373449B6818447F2840F37C857F3819
:104AC00090FBF1F301FB13007330C0B298F80010B3
:104AD00003F094FFBBF8002023881344042B7FF7D6
:104AE00099A85A4B1B88012B7FF494A83A68A2F12D
:104AF0000C007F287FF7CBA88B3A0C2092FBF0F3B9
:104B000000FB13207330FFF780B84F4C2388002B35
:104B100040F01783DFF844B14D494E4A098899F8AF
:104B20000000B2F800E0DFF83081C1EB000C0C228D
:104B30009CFBF2F102FB11C14FF0900C0CFB0EFE3E
:104B400002FB01E16FF00B0E58F8011008440EFB58
:104B500003007F2840F3F583A0F17F0393FBF2F07D
:104B600002FB10307330C0B203F070FFBBF80020BE
:104B700023881344022B22DD354A364B118899F8DD
:104B80000000B3F800C0DFF8D0E0411A0C2291FB1E
:104B9000F2F302FB1311902303FB0CF302FB01332E
:104BA00073445B6818447F2840F392847F3890FBFD
:104BB000F2F302FB13007330C0B203F047FFBBF8FF
:104BC000002023881344032B22DD214A214B118826
:104BD00099F80000B3F800C0DFF87CE0411A0C221D
:104BE00091FBF2F302FB1311902303FB0CF302FB86
:104BF000013373449B6818447F2840F3C1847F3895
:104C000090FBF2F302FB13007330C0B203F01EFFFF
:104C1000BBF8002023881344042B7EF728A90B4BF4
:104C20001B88012B7EF423A999F80020A2F10C0027
:104C30007F287FF723A88B3A0C2092FBF0F300FB30
:104C400013207330FEF75EBF689CFF1F0C9CFF1F94
:104C5000D89DFF1F829DFF1F20120100EE9BFF1FAA
:104C6000B84C2388002B40F06182DFF810B3B649BE
:104C7000B64A0988D7F80080B2F800E0B448C1EB22
:104C8000080C0C229CFBF2F102FB11C14FF0900CBE
:104C90000CFB0EFE02FB01E16FF00B0E405880444E
:104CA0000EFB03807F2840F3B483A0F17F0393FBC6
:104CB000F2F002FB10307330A64BC0B2197803F04B
:104CC0009DFEBBF8002023881344022B23DD9E4A5F
:104CD0009E4B11883868B3F800C0DFF874E2411ABF
:104CE0000C2291FBF2F302FB1311902303FB0CF354
:104CF00002FB013373445B6818447F2840F3FA8356
:104D00007F3890FBF2F302FB13007330914BC0B27B
:104D1000197803F073FEBBF8002023881344032B9B
:104D200023DD894A894B11883868B3F800C0DFF861
:104D300020E2411A0C2291FBF2F302FB13119023A3
:104D400003FB0CF302FB013373449B6818447F2878
:104D500040F320847F3890FBF2F302FB13007330A2
:104D60007C4BC0B2197803F049FEBBF800202388C1
:104D70001344042B7EF7C4A9774B1B88012B7EF4C8
:104D8000BFA93A68A2F10C007F2840F3B1808B3AAA
:104D90000C2092FBF0F300FB132073306D4BC0B27C
:104DA000197803F02BFEFEF7ABB9DFF89CA199F858
:104DB0000000BAF80030694CC11A0C2291FBF2F3E2
:104DC00002FB131302FB03F3E35818447F287FF719
:104DD0005DAD7F3890FBF2F302FB1300733015E5F5
:104DE0005F4B1A88182A13D03B681344A3F11800AC
:104DF0007F2840F3C9830C20973B93FBF0F200FB24
:104E0000123303F17300534BC0B2197803F0F6FD6F
:104E1000544B55491A78022A94BF013200221A7065
:104E20001A7831F81200182810D10424022A02F14D
:104E30000100C2B288BF002231F81200182804D144
:104E4000013CF3D11A70FEF75BB91A703B6803445A
:104E5000A3F118007F284BDD0C20973B93FBF0F269
:104E600000FB123303F1730098E7FBF70BFC16E429
:104E7000FBF708FCFFF79BBB394B1B88182B12D0A4
:104E800099F800201344A3F118007F2840F33583DC
:104E90000C20973B93FBF0F200FB123303F17300FD
:104EA000C0B203F0D3FD2F4A2F4B127833F81230E3
:104EB000182B3DF4DCAF99F800201344A3F118003F
:104EC0007F287EF7DBAE0C20973B93FBF0F200FBD4
:104ED000123303F17300FEF715BEFBF7D3FB49E471
:104EE000DFF864A099F80000BAF800301F4C63E7BF
:104EF000FBF7C8FB52E71E4B1B78002B7EF460A823
:104F00001C4B1B78002B3DF418ACB8F800301A4944
:104F10000133A8F800300A70FDF70FBC144B1B7862
:104F2000002B7DF40AAC134B1B78002B3DF405AC31
:104F3000B8F800301049013BA8F800300A70FDF7BE
:104F4000FCBB00BF689CFF1FD89DFF1F829DFF1FF9
:104F500020120100659CFF1F0C9CFF1FC016010062
:104F6000FA9BFF1F669CFF1FF09DFF1F8419010025
:104F7000579EFF1F589EFF1FDB9BFF1FEE9BFF1FCF
:104F8000C94A1288182A12D01344A3F118007F28A6
:104F900040F30A830C20973B93FBF0F200FB1233A3
:104FA00003F17300C0B298F8001003F027FDBF4B67
:104FB000BF491A78022A94BF013200221A701A7867
:104FC00031F81200182811D10424022A02F101003C
:104FD000C2B288BF002231F81200182805D1013C66
:104FE000F3D11A703B68FEF7B6B91A703B680344F8
:104FF000A3F118007F287EF74AAE0C20973B93FB65
:10500000F0F200FB123303F17300FEF7FEBDDFF890
:10501000C8B2E3E4A74B1B88182B12D099F80020E4
:105020001344A3F118007F2840F3B8820C20973B6B
:1050300093FBF0F200FB123303F17300C0B203F0F4
:1050400005FD9A4A9C4B127833F81230182B7FF4E6
:1050500032AFFDF70CBF974B1A88182A13D03B6864
:105060001344A3F118007F2840F39B820C20973B48
:1050700093FBF0F200FB123303F173008F4BC0B2CD
:10508000197803F0BBFC894B8B491A78022A94BF2C
:10509000013200221A701A7831F8120018287FF4B1
:1050A000D5AE0424022A02F1010294BFD2B200223A
:1050B00031F8120018287FF4C8AE013CF2D11A7002
:1050C000FEF71EB87B4A1288182A12D01344A3F1A7
:1050D00018007F2840F30B820C20973B93FBF0F2E3
:1050E00000FB123303F17300C0B298F8001003F014
:1050F00085FC6E4B70491A78022A94BF0132002257
:105100001A701A7831F8120018287FF46FAF04244F
:10511000022A02F1010294BFD2B2002231F8120039
:1051200018287FF462AF013CF2D15AE7644ADFF8F5
:10513000A8B11288BBF80010033291427FF7C1ADCD
:1051400095E55F4ADFF890B11288BBF80010033292
:1051500091427FF70BADDFE45A4C2388002B40F0DF
:10516000BB81DFF874B1584999F80000574A0988A3
:105170001788DFF85CE1411A0C2291FBF2FC02FB7C
:105180001C114FF0900C0CFB07F702FB01716FF044
:105190000B075EF80110014407FB03107F2840F362
:1051A000F6817F3890FBF2F302FB13007330C0B23C
:1051B00003F04CFCBBF8002023881344022B21DDB4
:1051C000414B424A99F800001B88B2F800E0404F7A
:1051D000C31A0C2193FBF1F201FB1232902303FB63
:1051E0000EF301FB02333B445B6818447F2840F315
:1051F000E9817F3890FBF1F301FB13007330C0B2FB
:1052000003F024FCBBF8002023881344032B21DD8A
:105210002D4B2E4A99F800001B88B2F800E02C4F65
:10522000C31A0C2193FBF1F201FB1232902303FB12
:105230000EF301FB02333B449B6818447F2840F384
:10524000D0817F3890FBF1F301FB13007330C0B2C3
:1052500003F0FCFBBBF8002023881344042B7EF7EB
:1052600036AA174B1B88012B7EF431AA99F800202F
:10527000A2F10C007F287FF7B0A88B3A0C2092FB9C
:10528000F0F300FB13207330FFF799B8114B0122A4
:105290007F2107201A8003F089FB7F210B2003F078
:1052A00085FBFDF7B8BE00BFFA9BFF1F669CFF1F82
:1052B000F09DFF1F029CFF1F649DFF1F659CFF1F49
:1052C0000C9CFF1F689CFF1FD89DFF1F829DFF1F26
:1052D00020120100769CFF1FEE9BFF1FC74B04228C
:1052E0007F2107201A8003F061FB00210B2003F0CF
:1052F0005DFBFDF789BEC14B02227F2107201A808A
:1053000003F054FB7F210B2003F050FBFDF777BE29
:10531000BA4B002107201C8003F048FB7F210B20A3
:1053200003F044FBFDF766BEB54B00227F2107204A
:105330001A8003F03BFB7F210B2003F037FBFDF7C6
:1053400072BEFBF79FF90EE4AE4B1B88182B12D0F0
:1053500099F800201344A3F118007F2840F34481FA
:105360000C20973B93FBF0F200FB123303F1730028
:10537000C0B203F06BFBA44AA44B127833F812308E
:10538000182B3EF4A4A999F800201344A3F11800A7
:105390007F287FF722A80C20973B93FBF0F200FBBD
:1053A000123303F17300FFF70AB8994A1288182ADA
:1053B00012D01344A3F118007F2840F300810C2081
:1053C000973B93FBF0F200FB123303F17300C0B282
:1053D00098F8001003F012FB8B4B8E491A78022AC2
:1053E00094BF013200221A701A7831F8120018287E
:1053F0007FF4FCAD0424022A02F1010294BFD2B270
:10540000002231F8120018287FF4EFAD013CF2D1F0
:10541000E7E5FBF737F94FE47D4B1A88182A13D0DC
:105420003B681344A3F118007F2840F3D4800C207C
:10543000973B93FBF0F200FB123303F17300764BC2
:10544000C0B2197803F0DAFA6F4B72491A78022A5F
:1054500094BF013200221A701A7831F8120018280D
:105460007FF4F4AC0424022A02F1010294BFD2B208
:10547000002231F8120018287FF4E7AC013CF2D189
:105480001A70FDF73DBEFBF7FDF8FFF7CABA604B97
:105490001B88182B12D099F800201344A3F1180090
:1054A0007F2840F39B800C20973B93FBF0F200FB9E
:1054B000123303F17300C0B203F0C8FA524A554BDD
:1054C000127833F81230182B7FF4F5ACFDF7CFBC0F
:1054D000FBF7D8F8FFF770BB504ADFF854B11288D9
:1054E000BBF80010033291427FF764AE3BE6FBF756
:1054F000C9F8F9E5FBF7C6F808E4FBF7C3F8CFE411
:10550000434B1B88182B11D099F800201344A3F1AA
:1055100018007F2859DD0C20973B93FBF0F200FB2D
:10552000123303F17300C0B203F090FA364A394BDC
:10553000127833F81230182B7FF425AFFEF7C7B876
:10554000374B1B88182B11D099F800201344A3F176
:1055500018007F283CDD0C20973B93FBF0F200FB0A
:10556000123303F17300C0B203F070FA264A2D4BD8
:10557000127833F81230182B7FF405AFFEF7A7B876
:10558000FBF780F8FFF741BBFBF77CF83BE4FBF748
:1055900079F80CE6FBF776F8FFF7E2BBFBF772F859
:1055A0004CE5FBF76FF869E5FBF76CF8FAE4FBF7FD
:1055B00069F8FFF760BAFBF765F8FFF786BAFBF703
:1055C00061F804E7FBF75EF819E6FBF75BF8AAE77A
:1055D000FBF758F8C7E7FBF755F830E7FBF752F849
:1055E00069E7FBF74FF832E6FBF74CF8C0E60E4BE5
:1055F00003930E4B0293FDF747BF00BFD09DFF1FE3
:10560000D89BFF1FFA9BFF1F669CFF1FF09DFF1F8B
:10561000049CFF1F6C9DFF1F659CFF1F0C9CFF1FC0
:10562000029CFF1F649DFF1FB59BFF1F809CFF1FF7
:10563000EE9BFF1F38B507F0A5F80E4804F0DCFF1D
:105640000D4804F0D9FF0D4804F0D6FF00234FF0B9
:105650007E5201210A48FAF709FF0A4B0A4A0B4910
:10566000802400251C7118461D60BDE838400AF0F2
:105670004DBD00BFEC9BFF1F209CFF1F7C9CFF1FAC
:10568000AC9DFF1F249EFF1F1C89FF1F29060000E1
:1056900043682A20198803F00DBB00BF10B50446EB
:1056A00022206368198803F005FBE3682420198829
:1056B000BDE8104003F0FEBA10B504460A20636846
:1056C000198803F0F7FAE3680C201988BDE8104048
:1056D00003F0F0BA10B5044606206368198803F099
:1056E000E9FAE36808201988BDE8104003F0E2BA3F
:1056F00010B5044602206368198803F0DBFAE368FA
:1057000004201988BDE8104003F0D4BA70B50E4CDF
:1057100084B01225042201230646039002932046FA
:105720008DE824001423102106F06AF906220923CB
:10573000029303960195204600921423102106F04F
:105740005FF904B070BD00BF889EFF1F2DE9F041D6
:10575000224D82B0012602B284B200922846019600
:105760007823192106F092F804F10C0212B28DE8A8
:1057700044002846A7197823192104F1020806F0ED
:1057800085F83FB20FFA88F819233A462846194699
:105790000196CDF8008006F079F878233A4628463D
:1057A0001946CDF80080019604F10A070B3406F083
:1057B0006DF83FB224B278233A46284619468DE860
:1057C000500006F063F8192300943A4601962846E3
:1057D000194606F05BF802B0BDE8F081889EFF1F15
:1057E0002DE9F0411E4682B01446002A6AD0099B7A
:1057F0004D4A00EBC305012C6F8929896868A7EB26
:10580000010382FB03E21A444FEAE373C3EBA213E2
:1058100002887BD0042C38D112FA83F3994203DC3E
:105820009F423946A8BF1946089A0180B6F9003050
:10583000BDF920803D48971D4FF0000E3FB219463C
:1058400042460097CDF804E006F020F829896A89DD
:105850006B68521A1B885C2AA3EB010359DD03EB2A
:1058600043030132C3EB431393FBF2F303F11B0237
:1058700013B20120328019464246019000972B480E
:1058800006F004F82A4B00221A702A4B022CB3F9B6
:10589000001045D0082C31D100221A8091422DD021
:1058A000089AB6F9003021480632012412B200925B
:1058B00019460194BDF9202005F0E8FF204602B00A
:1058C000BDE8F0811C4D1D4A2B681268CB1A93422B
:1058D0000F4617D9164A338811781448012918BF82
:1058E00001241470089A06321BB212B28DE814001B
:1058F0001946BDF9202005F0C9FF2F60012002B034
:10590000BDE8F081204602B0BDE8F0819BB2D31A19
:1059100084E75C2101FB03F393FBF2F21B32A7E760
:105920004A1C12B21A80B9E7C94216B2889EFF1FFC
:10593000059FFF1F689EFF1FEC9EFF1FEC290100C3
:1059400030B583B000230C4605B2009326225B23BA
:105950001C210C4805F0EAFC2946012326220948AF
:1059600004F0F4FF002C24B205DB2146012326229B
:10597000044804F0EBFF044A044B15801C8003B07C
:1059800030BD00BF889EFF1F628AFF1F648AFF1F11
:10599000F0B59B4C237883B01BB19A4B4FF6FF7246
:1059A0001A80994BB3F90030C3B9984A954B1068E7
:1059B000B3F9002080F30C005B2303FB00F000131D
:1059C0001C3082425ED04FF0FF31FFF7B9FF9048A4
:1059D00005F010FD0023237003B0F0BD012B36D07D
:1059E000022B6ED0032B53D0042BF3D1252200259C
:1059F0008DE8240076231C218548864E864F05F0CD
:105A000045FF17E0B0F5AF7FA8BF4FF4AF70323855
:105A100003FB00F387FB0321DB17C3EB61111C3190
:105A200009B201231D442522794804F08FFF0C2D73
:105A300000F08480E9B2794804F046FE56F8042B61
:105A4000801A31284FF05B03DCDC1C21E9E7744B42
:105A50001A68B2F52F7F32DB41F25C239342A8BF74
:105A60001346A3F52F735B226E4802FB03F380FB02
:105A70000320DB17C3EBA0201C30624BB3F90030CE
:105A80008342A0D1684BB3F9003001339BD1A1E729
:105A9000664B1B68B3F5FA7F11DBB3F57A6FA8BFCD
:105AA0004FF47A63A3F5FA7261485B2303FB02F3B8
:105AB00080FB0320DB17C3EB20201C30DDE71C201C
:105AC000DBE75C4B1B68B3F5FA7F33DBB3F57A6F2A
:105AD000A8BF4FF47A63A3F5FA7255485B2303FB22
:105AE00002F380FB0320DB17C3EB20201C30524B5A
:105AF0001B68B3F5FA7F1FDBB3F57A6FA8BF4FF4CD
:105B00007A63A3F5FA724A495B2303FB02F381FB34
:105B10000321DB17C3EB21211C313A4BB3F90030D1
:105B200083427FF452AF404BB3F900308B427FF495
:105B30004CAF4FE71C20DAE71C21EEE726220025B8
:105B40008DE8240076231C2131483C4E324F05F06D
:105B50009DFE16E0B0F5AF7FA8BF4FF4AF703238AE
:105B600003FB00F387FB0321DB17C3EB61111C313F
:105B700009B201231D442622254804F0E7FE0C2D1E
:105B80000CD0E9B22E4804F09FFD56F8042B801A81
:105B900031284FF05B03DDDC1C21EAE727220025DA
:105BA0008DE8240076231C211948264E1A4F05F053
:105BB0006DFE17E0B0F5AF7FA8BF4FF4AF7032387D
:105BC00003FB00F387FB0321DB17C3EB61111C31DF
:105BD00009B201231D4427220D4804F0B7FE062D0B
:105BE0003FF4F5AEE9B2184804F06EFD56F8042B08
:105BF000801A31284FF05B03DCDC1C21E9E700BF91
:105C00005E9EFF1F628AFF1F649EFF1FE49DFF1FB1
:105C1000889EFF1F188AFF1F4B48371B209CFF1FC1
:105C2000C89BFF1FD3058541648AFF1F109CFF1F7F
:105C3000011FB8121C9CFF1F509EFF1F2C89FF1FC5
:105C40007C9CFF1F488AFF1FEC9BFF1F2DE9F04F34
:105C5000DFF8EC82B74CB8F900604D7854F8264074
:105C600087B08246039305B10D78DFF8FCB2002AB5
:105C700034D19BF800308BBBAF4EB6F90000002842
:105C800000F0CE80012800F02481012032232A4632
:105C9000019000935146A94B2046FFF7A1FD002536
:105CA0000746B6F90030022B40F3F480002333801E
:105CB000B8F90030A24A002BC0F2F880042BC4BF10
:105CC00000231380039B002B40F0F680002D0CBFB7
:105CD00038464FF0FF3007B0BDE8F08F964EE368CE
:105CE0002268984804930027059237808BF800704B
:105CF00005F074FA1120FFF729FD4FF0010919236F
:105D00002821CDF804900091242219468D4805F0F1
:105D1000BDFD782328212422CDF8049000918948E4
:105D2000194605F0B3FD4946864806F045F90222BA
:105D30001921844806F03CF9DDF8149048460AF031
:105D4000BFFF494602467F4806F0CCFA7D4806F080
:105D5000DFFA394614227B4806F02AF903227A49F1
:105D6000784806F0BFFA774806F0D2FA394623227F
:105D7000744806F01DF903227449724806F0B2FA1D
:105D8000704806F0C5FA049B002B72D10123704ABB
:105D900018461370FFF7BAFC208963896768191ADF
:105DA0005C293A885BDC131A5C2202FB03F292FB4B
:105DB000F1F31B33674A6348138001271BB21A2291
:105DC00019468DE88400142205F060FD049BDBB1C8
:105DD000218A638AE768581A5C283A886FDD521A6C
:105DE00002EB4202C2EB4212431C92FBF3F31B3361
:105DF000524A54481380012738221BB28DE8840090
:105E00001946322205F042FD534A544BB6F90000C0
:105E1000012111704FF6FF721A8000287FF432AF13
:105E2000DFF848914E4AD9F800301268C3EB0A03F4
:105E300093424CD9464B1A78012A18BF012018709A
:105E40000127FFF763FCC9F800A0012D4ED0042DF7
:105E500059D0022D60D0082D64D0002521E7121AF8
:105E600002EB4202C2EB42124B1C92FBF3F31B33D8
:105E7000A0E72F20FFF76AFC39463222314806F0AE
:105E800097F8032237492F4806F02CFA2D4806F0E0
:105E90003FFA7BE77FF40CAFE368002B3FF406AFDB
:105EA000B8F90030264A002BBFF608AF0423138050
:105EB000039B002B3FF40AAFFFF76AFD06E7511A78
:105EC0005C2202FB01F292FBF0F31B3390E70746E2
:105ED000BBE7002714238DE888002A4651461D4B56
:105EE0002046FFF77DFC3D460746DAE6B8F800306D
:105EF0008BF800500133A8F80030636983B10025A6
:105F000020469847CDE6B8F800300122013BA8F8BA
:105F100000308BF80020F0E7012333800025C7E62E
:105F20001D46BEE66369002232804FF0FF35002B2C
:105F3000E6D1BDE6688AFF1F689EFF1F629EFF1FB5
:105F4000649EFF1F889EFF1F641B0100681B0100E9
:105F5000059FFF1F609EFF1F5E9EFF1F628AFF1F3F
:105F6000EC2901006C1B0100669EFF1FEC9EFF1FC9
:105F700001210D2007F080B800210D2007F07CB82A
:105F800001460D2007F078B808B50D2007F07AF823
:105F9000B0FA80F149090D20BDE8084007F06CB85F
:105FA00010B5002144080D2007F066F8204607F0E0
:105FB0009FF80D20012107F05FF82046BDE8104052
:105FC00007F096B82D4A2E4B10881B68984210B5E2
:105FD00049DA2C4A1288141A9A42A8BF1A46B4F514
:105FE000157F36DA121A40F2532303FB02F393FBB8
:105FF000F4F105310A2006F0AFFE234B1978C9B33E
:10600000224B23491B6840F2271283F3070302FB4C
:1060100003F381FB03211944DB17C3EBA111053105
:10602000092006F099FE1B4B1968F1B181F30701B5
:1060300040F22712164802FB01F380FB03211944AA
:10604000DB17C3EBA11105311620BDE8104006F0A7
:1060500083BE131A4FF41572611C02FB03F393FB0A
:10606000F1F10531C6E70021C4E71620BDE8104074
:1060700006F072BE092006F06FFED4E77E9CFF1F7B
:10608000B89BFF1F329EFF1F3E9CFF1FBC9BFF1F44
:1060900009040281F89DFF1F7F2838B5A8BF7F2023
:1060A0000F4C4FF4167202FB00F284FB02311144D4
:1060B000D2170546C2EBA1110A2006F04DFE7F3D26
:1060C0004FF4967303FB05F384FB03211944DB179C
:1060D000A3EBA1110920BDE8384006F03DBE00BF8A
:1060E00009040281C368B3F9003030B583EAE37470
:1060F000A4EBE374002BA0B218DB012300E01346ED
:1061000003EB830252009442F9DA0A4D90FBF3F25A
:1061100085FB03E403FB1200DB173032D3EBA4034F
:1061200080B201F8012BF1D10B7030BD2D230B7023
:106130000131E2E76766666638B5094D822420467C
:1061400002F0D2FD35F8021B00B28842204601D091
:1061500002F0B0FD0234A4B28A2CF0D138BD00BFE9
:106160006C9DFF1F024B8020198802F0A3BD00BF69
:10617000049CFF1F38B5094D7824204602F0B4FD79
:1061800035F8021B00B28842204601D002F092FD91
:106190000234A4B2802CF0D138BD00BF649DFF1F33
:1061A000024B7620198802F085BD00BF029CFF1FBC
:1061B00038B5094D4624204602F096FD35F8021BFD
:1061C00000B28842204601D002F074FD0234A4B22D
:1061D0004E2CF0D138BD00BFF09DFF1F024B442074
:1061E000198802F067BD00BFFA9BFF1F024B4E20CB
:1061F000198802F05FBD00BF189CFF1F024B9A2058
:10620000198802F057BD00BF689CFF1F024B982001
:10621000198802F04FBD00BF0C9CFF1F024B8C2061
:10622000198802F047BD00BF829DFF1F024B9C20D2
:10623000198802F03FBD00BFEE9BFF1F024B962066
:10624000198802F037BD00BFD89DFF1F024B8A207E
:10625000198802F02FBD00BF9E9DFF1F024B10202A
:10626000198802F027BD00BF9C9DFF1F024B2C2008
:10627000198802F01FBD00BFE89BFF1F024B1E20C4
:10628000198802F017BD00BFE49BFF1FC3680E20F2
:10629000198802F00FBD00BF024B2820198802F0B8
:1062A00009BD00BFEC9DFF1F024B6420198802F05E
:1062B00001BD00BFE89DFF1F024B5A20198802F064
:1062C000F9BC00BFD09BFF1F024B1620198802F0BB
:1062D000F1BC00BFD89BFF1F024B2E20198802F093
:1062E000E9BC00BF709CFF1F024B3020198802F0F0
:1062F000E1BC00BFC49BFF1F024B1820198802F0AD
:10630000D9BC00BF829CFF1F024B1A20198802F0E3
:10631000D1BC00BF229CFF1F024B1C20198802F039
:10632000C9BC00BF1A9CFF1F024B6620198802F0EF
:10633000C1BC00BF1E9EFF1F024B7220198802F0D5
:10634000B9BC00BF389EFF1F024B2020198802F005
:10635000B1BC00BF1C9EFF1F024B3220198802F007
:10636000A9BC00BF129EFF1F024B6820198802F0D3
:10637000A1BC00BF549CFF1F024B6C20198802F087
:1063800099BC00BFC09BFF1F024B6E20198802F012
:1063900091BC00BF5C9EFF1F024B5220198802F087
:1063A00089BC00BF5E89FF1F024B5020198802F094
:1063B00081BC00BF108AFF1F024B5420198802F0D5
:1063C00079BC00BF128AFF1F024B5C20198802F0C3
:1063D00071BC00BF608AFF1F024B5E20198802F06B
:1063E00069BC00BF5C89FF1F024B6020198802F066
:1063F00061BC00BF889DFF1F024B5620198802F028
:1064000059BC00BF629CFF1F244B1B880B2B43D839
:10641000DFE803F00B10151A1F24292E33383D0630
:10642000084604221E490AF009BD084604221D49F7
:106430000AF004BD084604221B490AF0FFBC0846C6
:1064400004221A490AF0FABC0846042218490AF044
:10645000F5BC0846042217490AF0F0BC084604229D
:1064600015490AF0EBBC0846042214490AF0E6BCC0
:106470000846042212490AF0E1BC084604221149E8
:106480000AF0DCBC084604220F490AF0D7BC0846D3
:1064900004220E490AF0D2BC704700BFD89DFF1FEE
:1064A000D8260100C42401007823010060240100E3
:1064B0007C230100D02701008023010084230100F8
:1064C000FC25010088230100E42601008C23010043
:1064D000064B074A10B41C88064B0846002C14BF14
:1064E00011461946042210BC0AF0A8BC389CFF1FB4
:1064F0009023010094230100064B074A10B41C8826
:10650000064B0846002C14BF11461946042210BC45
:106510000AF094BC729CFF1F902301009423010099
:10652000064B074A10B41C88064B0846002C14BFC3
:1065300011461946042210BC0AF080BC8A9DFF1F38
:106540009023010094230100064B074A10B41C88D5
:10655000064B0846002C14BF11461946042210BCF5
:106560000AF06CBCDA9DFF1F902301009423010008
:10657000064B074A10B41C88064B0846002C14BF73
:1065800011461946042210BC0AF058BC769CFF1F25
:1065900090230100942301001B4B1B880A2B0AD86F
:1065A000DFE803F00A0E12161A1E22262A2E060013
:1065B000164B186808607047154B186808607047DC
:1065C000144B186808607047134B186808607047D0
:1065D000124B186808607047114B186808607047C4
:1065E000104B1868086070470F4B186808607047B8
:1065F0000E4B1868086070470D4B186808607047AC
:106600000C4B1868086070479E9DFF1FBC2301005B
:1066100094230100982301009C230100A023010082
:10662000A4230100A8230100AC230100B023010032
:10663000B4230100B8230100F0B52B4E2B4FDFF837
:10664000C4E005460FCE87B06C460FC496E8030041
:106650003B68274A274F44F8040B40F6CC3083426E
:10666000C8BF3A46BEF800602180012E118892789A
:10667000ADF80D108DF80F202AD032D340F6CA02A3
:10668000022E18BF00229A4226DCA3F698031A496C
:106690001A4AC3EB031381FB03011944DB17C3EB55
:1066A0006123243382FB0321DA17C2EBA10202EB40
:1066B0008201A3EB4103303330328DF813308DF873
:1066C00011206946284616220AF0B8FB07B0F0BD33
:1066D00040F698029A42D8DD094B1868CDF81100AF
:1066E000EFE740F6FC02CEE7D0230100FC9DFF1F40
:1066F000C4230100C02301003B773B9867666666B0
:10670000C8230100749DFF1FF8B5174C174E22785F
:10671000174D33782F888E46003218BF012201466C
:106720007046FFF793FA002398423370237015DB0D
:1067300014BF012000202B889F420ED040F23A72F5
:10674000A3F5AF730B490C4C02FB03F381FB03125F
:10675000DB17A3EB621332332360F8BD0749012234
:1067600018460A702270E6E70C8BFF1F799EFF1F08
:106770002C9EFF1FB5814E1B008AFF1F049FFF1F29
:10678000014B187802F02EBAE89EFF1F014B1878D3
:1067900002F042BA8490FF1F134BB3F9003030B5BA
:1067A00083EAE374A4EBE374002BA0B218DB0123AB
:1067B00000E0134603EB830252009442F9DA0B4DDA
:1067C00090FBF3F285FB03E403FB1200DB1730328E
:1067D000D3EBA40380B201F8012BF1D10B7030BDD3
:1067E0002D230B700131E2E78490FF1F6766666618
:1067F000144BB3F9003070B583EAE375A5EBE3758C
:10680000002BACB21ADB012300E0034603EB83004C
:1068100040008542F9DA0C4E94FBF3F086FB03E569
:1068200003FB1044DB173030D3EBA503A4B201F80F
:10683000010BF1D105480B70106070BD2D230B705A
:106840000131E0E7D09BFF1F67666666E823010021
:10685000134BB3F9003030B583EAE374A4EBE3746F
:10686000002BA0B218DB012300E0134603EB8302E8
:1068700052009442F9DA0B4D90FBF3F285FB03E4EE
:1068800003FB1200DB173032D3EBA40380B201F814
:10689000012BF1D10B7030BD2D230B700131E2E7DC
:1068A0005E89FF1F67666666134BB3F9003030B52B
:1068B00083EAE374A4EBE374002BA0B218DB01239A
:1068C00000E0134603EB830252009442F9DA0B4DC9
:1068D00090FBF3F285FB03E403FB1200DB1730327D
:1068E000D3EBA40380B201F8012BF1D10B7030BDC2
:1068F0002D230B700131E2E7108AFF1F6766666681
:10690000134BB3F9003030B583EAE374A4EBE374BE
:10691000002BA0B218DB012300E0134603EB830237
:1069200052009442F9DA0B4D90FBF3F285FB03E43D
:1069300003FB1200DB173032D3EBA40380B201F863
:10694000012BF1D10B7030BD2D230B700131E2E72B
:10695000128AFF1F67666666134BB3F9003030B5C5
:1069600083EAE374A4EBE374002BA0B218DB0123E9
:1069700000E0134603EB830252009442F9DA0B4D18
:1069800090FBF3F285FB03E403FB1200DB173032CC
:10699000D3EBA40380B201F8012BF1D10B7030BD11
:1069A0002D230B700131E2E7608AFF1F6766666680
:1069B000134BB3F9003030B583EAE374A4EBE3740E
:1069C000002BA0B218DB012300E0134603EB830287
:1069D00052009442F9DA0B4D90FBF3F285FB03E48D
:1069E00003FB1200DB173032D3EBA40380B201F8B3
:1069F000012BF1D10B7030BD2D230B700131E2E77B
:106A00005C89FF1F6766666608B5702002F06CF946
:106A1000044B1988884204D07020BDE8084002F079
:106A200049B908BD749DFF1F08B5742002F05CF9D8
:106A3000044B1988884204D07420BDE8084002F055
:106A400039B908BD089EFF1F054B1B880846042264
:106A500013B904490AF0F2B903490AF0EFB900BFCB
:106A6000189CFF1FF0230100EC2301000E4B1B8834
:106A7000032B17D8DFE803F0110C070208460422A5
:106A80000A490AF0DBB90846042209490AF0D6B9D6
:106A90000846042207490AF0D1B9084604220649EB
:106AA0000AF0CCB9704700BF829DFF1F002401008F
:106AB000FC230100F8230100F423010010B40A4B69
:106AC0000A4C0A4693E8030083B0238802AC04E929
:106AD000030004EB8303104653F8081C052203B09F
:106AE00010BC0AF0ABB900BFF41B0100E89DFF1F0A
:106AF00030B40A4B0A4D0C4693E8070084B02B884B
:106B000004AD05E9070005EB8303204653F80C1C90
:106B1000042204B030BC0AF091B900BFFC1B010094
:106B2000749DFF1FF0B40C4D0C4F0E460FCD8CB072
:106B300001AC0FC40FCD0FC495E807003B8884E873
:106B400007000CAA02EB8303304653F82C1C0422E6
:106B50000CB0F0BC0AF072B9081C0100D09DFF1FF8
:106B6000F0B40A4D0A4F0E460FCD86B001AC0FC4EB
:106B70002A683B88226006AA02EB8303304653F85A
:106B8000141C042206B0F0BC0AF058B9341C0100F1
:106B9000829CFF1FF0B40A4D0A4F0E460FCD86B0FF
:106BA00001AC0FC42A683B88226006AA02EB83036B
:106BB000304653F8141C0C2206B0F0BC0AF03EB963
:106BC000481C01001A9CFF1FF0B40A4D0A4F0E46E4
:106BD0000FCD86B001AC0FC42A683B88226006AA9C
:106BE00002EB8303304653F8141C042206B0F0BCB9
:106BF0000AF024B95C1C0100089EFF1F164B1B887D
:106C00000BB31BB283EAE370A0EBE370002B30B54B
:106C100084B21DDB012300E0134603EB8302520024
:106C20009042F9DA0D4894FBF3F280FB03E503FB95
:106C30001244DB173032D3EBA503A4B201F8012BC9
:106C4000F1D10B7030BD0846042205490AF0F6B8B0
:106C50002D230B700131DDE7549CFF1F67666666CC
:106C600004240100F0B40A4D0A4F0E460FCD86B041
:106C700001AC0FC42A683B88226006AA02EB83039A
:106C8000304653F8141C042206B0F0BC0AF0D6B803
:106C9000701C0100C09BFF1F054B1B881BB9054BD7
:106CA0001868086070470846042203490AF0C6B80D
:106CB000689CFF1F9423010090230100164B1B8842
:106CC0000BB31BB230B583EAE374A4EBE374002B7F
:106CD000A0B21CDB012300E0134603EB8302520049
:106CE0009442F9DA0D4D90FBF3F285FB03E403FBCC
:106CF0001200DB173032D3EBA40380B201F8012B72
:106D0000F1D10B7030BD064B1868086070472D2319
:106D10000B700131DEE700BFE49BFF1F676666660C
:106D200094230100164B1B880BB31BB230B583EACA
:106D3000E374A4EBE374002BA0B21CDB012300E09E
:106D4000134603EB830252009442F9DA0D4D90FB97
:106D5000F3F285FB03E403FB1200DB173032D3EBC5
:106D6000A40380B201F8012BF1D10B7030BD064BAA
:106D70001868086070472D230B700131DEE700BFF3
:106D8000DE9DFF1F6766666694230100164B1B8815
:106D90000BB31BB230B583EAE374A4EBE374002BAE
:106DA000A0B21CDB012300E0134603EB8302520078
:106DB0009442F9DA0D4D90FBF3F285FB03E403FBFB
:106DC0001200DB173032D3EBA40380B201F8012BA1
:106DD000F1D10B7030BD064B1868086070472D2349
:106DE0000B700131DEE700BFD89BFF1F6766666648
:106DF00008240100174B1B881BB31BB270B583EA34
:106E0000E375A5EBE375002BACB21EDB012300E0BC
:106E1000034603EB830040008542F9DA0E4E94FBF3
:106E2000F3F086FB03E503FB1044DB173030D3EBB4
:106E3000A503A4B201F8010BF1D108480B70106052
:106E400070BD074B1868086070472D230B70013127
:106E5000DCE700BF709CFF1F67666666CC230100FD
:106E600094230100164B1B880BB31BB230B583EA89
:106E7000E374A4EBE374002BA0B21CDB012300E05D
:106E8000134603EB830252009442F9DA0D4D90FB56
:106E9000F3F285FB03E403FB1200DB173032D3EB84
:106EA000A40380B201F8012BF1D10B7030BD064B69
:106EB0001868086070472D230B700131DEE700BFB2
:106EC000C49BFF1F6766666694230100164B1B88F0
:106ED0000BB31BB230B583EAE374A4EBE374002B6D
:106EE000A0B21CDB012300E0134603EB8302520037
:106EF0009442F9DA0D4D90FBF3F285FB03E403FBBA
:106F00001200DB173032D3EBA40380B201F8012B5F
:106F1000F1D10B7030BD064B1868086070472D2307
:106F20000B700131DEE700BF1E9EFF1F67666666BD
:106F300094230100164B1B880BB31BB230B583EAB8
:106F4000E374A4EBE374002BA0B21CDB012300E08C
:106F5000134603EB830252009442F9DA0D4D90FB85
:106F6000F3F285FB03E403FB1200DB173032D3EBB3
:106F7000A40380B201F8012BF1D10B7030BD064B98
:106F80001868086070472D230B700131DEE700BFE1
:106F9000389EFF1F6766666694230100174B1B88A7
:106FA0001BB31BB270B583EAE375A5EBE375002B49
:106FB000ACB21EDB012300E0034603EB830040007C
:106FC0008542F9DA0E4E94FBF3F086FB03E503FBF2
:106FD0001044DB173030D3EBA503A4B201F8010B4A
:106FE000F1D108480B70106070BD074B186808603D
:106FF00070472D230B700131DCE700BF1C9EFF1F83
:10700000676666660C24010094230100074B1B8809
:10701000022B06D0012B0CBF054B064B18680860ED
:107020007047054B18680860704700BF889DFF1FB8
:10703000142401001824010010240100054B1B88B2
:107040001BB1054B186808607047044B186808604E
:10705000704700BF629CFF1F202401001C24010018
:1070600038B5FAF751FD0D4B1B7833B90C4B102096
:10707000198801F01FFE012038BD0A4D0A4C2B78FB
:107080002288B3FA83F382F008025B09114642209A
:107090002B70228001F00EFE002038BDDA9BFF1F0E
:1070A0009C9DFF1F789DFF1FF89BFF1F184B1A88A0
:1070B00052B3184A128830B50A80B3F90030002B59
:1070C00083EAE374A4EBE374BCBF2D238B70A0B2FE
:1070D000ACBF02310331012300E0134603EB83020E
:1070E00052009442F9DA0C4D90FBF3F285FB03E475
:1070F00003FB1200DB173032D3EBA40380B201F89C
:10710000012BF1D10B7030BD044B1868086070473B
:10711000229CFF1F242401006766666694230100F9
:1071200070B53C4D2B780646002B35D11C46737844
:107130000BB9204670BDFAF7E7FC374A374B3848A1
:10714000127831781B78007802EB43034A1E03EB78
:1071500080030E2AEDD801A050F822F0C57100007E
:10716000E771000033710000C57100003371000049
:107170003371000033710000B371000033710000FF
:10718000337100003371000033710000337100006F
:1071900033710000AF710000AE21224803F0CEFD34
:1071A000204804F01BF800232B700124BFE706F0F1
:1071B000B1FAAF211B4803F0C1FD1B4A0123137034
:1071C0002B70B6E783B91948038804294FF6FF717D
:1071D00003F1FF320CBF01230B46134403F07F037E
:1071E000013303800FE073B1013B114A32F81330D1
:1071F0004BB10E4E0F481049104A33800123002630
:1072000006700B701370084A0221012311702B7055
:10721000204670BD0C8BFF1F219EFF1F229EFF1F6B
:10722000239EFF1F889EFF1F049FFF1F429EFF1F7C
:10723000549DFF1F4C9CFF1FDB9BFF1F079FFF1FE1
:1072400010B5064B064C1A882046012101F020FD9E
:1072500021884220BDE8104001F02CBD389CFF1F62
:10726000F89BFF1F10B5064B064C1A8820460221DA
:1072700001F00EFD21884220BDE8104001F01ABD4A
:10728000729CFF1FF89BFF1F10B5064B064C1A8817
:107290002046042101F0FCFC21884220BDE810407A
:1072A00001F008BD8A9DFF1FF89BFF1F10B5064B1C
:1072B000064C1A882046002101F0EAFC2188422071
:1072C000BDE8104001F0F6BCDA9DFF1FF89BFF1FE0
:1072D00008B5122001F008FD054B1988884206D038
:1072E000122001F0E7FCBDE8084001F0FBBB08BD3F
:1072F000D09DFF1F08B5582001F0F6FC054B1988FA
:10730000884206D0582001F0D5FCBDE8084001F0C5
:10731000E9BB08BDDE9DFF1F08B5142001F0E4FCA9
:10732000054B1988884206D0142001F0C3FCBDE843
:10733000084001F0D7BB08BD769CFF1FF0B480EA7F
:10734000E075A5EBE0750028ACB21FDB1DBF2B2359
:107350000B704E1C0E46012300E0134603EB830224
:1073600052009542F9DA0B4F94FBF3F287FB0305C9
:1073700003FB1244DB173032D3EBA503A4B206F8AB
:10738000012BF1D133700846F0BC70472D230B70F0
:107390004E1CE0E767666666084B188828B10D2822
:1073A00007D00D3800B2FFF7C9BF054A1068086062
:1073B0007047044A10680860704700BF5C9EFF1F5A
:1073C0009423010028240100174B18880C2813D09F
:1073D000192815D01A2817D01B2819D01C281BD003
:1073E0001D281DD01E2803D00C3800B2FFF7A6BF01
:1073F0000E4A1068086070470D4A106808607047B0
:107400000C4A1068086070470B4A106808607047A3
:107410000A4A106808607047094A10680860704797
:10742000084A106808607047129EFF1F442401003C
:107430002C240100302401003424010038240100F0
:107440003C24010040240100034B1888A0EB80007D
:10745000400000B2FFF772BFE89EFF1F024B188882
:10746000033800B2FFF76ABFEC9DFF1F024B18887C
:107470000C3800B2FFF762BFD49BFF1F024B188885
:10748000183800B2FFF75ABF049CFF1F024B188840
:10749000183800B2FFF752BF029CFF1F024B18883A
:1074A000183800B2FFF74ABFFA9BFF1FC36818885D
:1074B000183800B2FFF742BF054B1B881BB9054BBC
:1074C00018680860704708460422034909F0B6BCF2
:1074D0000C9CFF1F942301009023010030B5134C36
:1074E00085B001252B463C2202212046009503F061
:1074F0009BFC204603F072FE0022402180232046A0
:107500000191009311460A4B029504F015FB2046A9
:1075100003F070FF07480849084A0023036083808E
:107520000B608B801360938005B030BD889EFF1F79
:10753000FC1E01006C9EFF1F809EFF1FF49EFF1F1C
:1075400010B500EBC00000F10F02D2B293B284B0CC
:107550009C1E981C3D2303918DE819003921024897
:1075600004F04EFA04B010BD889EFF1F014B0122AB
:107570001A707047799EFF1FF0B585B0634C644B5D
:107580000293644A019204230093634E634B644F59
:10759000644D20464022802103F04EFA2046624A84
:1075A0006249634C08F0B2FDB761624FF761624F08
:1075B000AF61624FEF61624FA7616248624FE7615E
:1075C000624F87616249634FC761634F8F61634A4E
:1075D000634FCF61634F9761634B644FD761644FD3
:1075E0009F61644E644FDF61644FB761644D654FC6
:1075F000F761654FAF61654C654FEF61654F664858
:10760000A761664FE761664F66498761664FC7614C
:10761000664F674A8F61674FCF61674F674B9761CE
:10762000674FD761674F684E9F61684FDF61684F52
:10763000684DB761684FF761684F694CAF61694F3A
:10764000EF61694FA7616948694FE761694F8761D9
:1076500069496A4FC7616A4F8F616A4A6A4FCF6151
:107660006A4F97616A4B6B4FD7616B4F9F616B4E4F
:107670006B4FDF616B4FB7616B4D6C4FF7616C4FB8
:10768000AF616C4C6C4FEF616C4FA7616C486D4FF4
:10769000E7616D4F87616D496D4FC7616D4F8F61B8
:1076A0006D4A6E4FCF616E4F6E4B97616E4FD761D3
:1076B0006E4F6F4E9F616F4FDF616F4F6F4DB761C0
:1076C0006F4FF7616F4F704CAF61704F70487149E9
:1076D000EF61714F714DA761E561714F714D724C52
:1076E000DFF8E8E1714A724B8761C5618C61714EC8
:1076F000C1F81CE0704F714D714C7248724997612E
:10770000D5619C61D861B16005B0F0BD889EFF1F56
:10771000A0860100801A0600708DFF1FA090FF1F39
:107720006D740000E48EFF1F1C89FF1F91AA0000EA
:10773000548EFF1F8D6200005D740000996200008E
:10774000D1640000508CFF1F41720000F9640000FA
:10775000088FFF1F65720000216500004C8DFF1F20
:1077600089720000BD6A0000BC8CFF1FA962000086
:1077700049650000288DFF1FAD72000049740000AC
:10778000048DFF1F8167000099670000C08EFF1FF6
:107790008D670000F16A0000088CFF1F096A000075
:1077A000256B0000708FFF1FD1720000256D000057
:1077B000988CFF1FF5720000F1670000C48BFF1F5B
:1077C000B962000071650000DC8FFF1F19730000B3
:1077D0008D6D0000748CFF1FC9620000F56D000004
:1077E000948DFF1FD9620000656E0000348BFF1F6F
:1077F000E9620000616B0000E08CFF1FF96200008D
:10780000AD7000009C8EFF1F09630000956B0000A7
:107810006090FF1F19630000CD6E0000308EFF1FC7
:1078200029630000356F0000588BFF1F396300008B
:10783000C96B0000948FFF1F296A00009D6F000034
:10784000788EFF1F49630000C97300007C8BFF1F07
:1078500059630000FD6B0000108BFF1F696300007F
:10786000656C00007C8AFF1F79630000997300003B
:107870003090FF1F89630000516800002C8CFF1FAF
:1078800099630000A9680000E88AFF1FA96300004F
:10789000A08BFF1F2C8FFF1F01690000B963000040
:1078A00059690000C9630000B1690000C48AFF1F64
:1078B000A08AFF1F5490FF1F0D700000E9630000B5
:1078C0003D700000F9630000857E0000D963000070
:1078D000F0B5461C83B00D460127032336B22AB209
:1078E000044631468DE888002448ADB204F01EF805
:1078F0000C23AA1C12B200930197052321B21F4842
:1079000004F014F81E4A1F4B12881B68BA422AD092
:1079100023D3022A10D11C4CA3F6CA0384FB0324F0
:107920001C44DB17C3EB24140A2CA8BF0A2424EA46
:10793000E474A2B223B202E000231A461C460D35BD
:10794000AA1A01200093019012B2314603230B487A
:1079500003F06AFF204603B0F0BD0C4CA3F6FC0315
:1079600084FB0324DDE7084CA3F6980384FB03247F
:107970001C44DB17C3EBE404D6E700BF889EFF1F5F
:10798000749DFF1FFC9DFF1F898888881F85EB5110
:107990002DE9F0438FB283B0DFF84C80BD1D461D4A
:1079A0002DB204B236B24FF001090AB22346314675
:1079B00040460095CDF8049003F068FF2A46334610
:1079C000214640468DE8200203F060FF07F10C02DB
:1079D0000095334612B22146CDF80490404603F09C
:1079E00055FF03B0BDE8F083889EFF1F2DE9F043EB
:1079F000804685B0002956D10121304804F0DCFAD8
:107A00002F4998F8062098F8083011F80290994507
:107A100022DA4FEA89064D460C24D8F80C30274864
:107A20009B595F6822B2002104F0C2FA384609F07F
:107A300047F939460246214804F054FC1F4804F037
:107A400067FC98F8083001350934AB42A4B206F15E
:107A5000040601DD422CE0D1B9F1000F13D109F188
:107A6000060999450CDA3C2301213B22039102933C
:107A70000093019239233F223A21104803F0C0FFBE
:107A800005B0BDE8F0830F2301213B22039102934F
:107A90000093019239230C223A21084803F0B0FFE9
:107AA00098F80830DBE700213423009301913F234D
:107AB0000C22024803F0B8FE9EE700BF889EFF1F1D
:107AC000809EFF1F10B5104C0121204604F07AFA69
:107AD0002046012104F070FA20463422552104F09A
:107AE00067FA20460222094904F0FCFB20460522E1
:107AF000074904F0F7FB204604F00AFC2046BDE8E5
:107B0000104003F077BC00BF889EFF1F482401008F
:107B10004C24010070B50D46064609F0D1F800EB83
:107B200040008400002D36D0284609F0C9F800EB4B
:107B30004000400023185B1003F16001091A28225D
:107B400009B21748C3F1600404F032FA0121144865
:107B500004F032FA284609F0B3F8294602461048E4
:107B600004F0C0FB0E4804F0D3FB02210C4804F0E3
:107B700023FA21B221220A4804F01AFA304609F009
:107B80009FF831460246064804F0ACFB0448BDE8C5
:107B9000704004F0BDBB6410C4F16004E5E700BFB1
:107BA000889EFF1F10B50D4B1B5C51F823402378B6
:107BB00084B013B1012004B010BD04AA01A942F899
:107BC000103D2046A3699847A38A9B07F2D401A8D9
:107BD0000099FFF79FFF012004B010BD6C9EFF1FAE
:107BE0002DE9F04F2F4DDFF8CCB0DFF8C4A0DFF85F
:107BF000C8900FCD91B003AC0FC40FCD0FC40FCD03
:107C00000FC42B6823600025A8462F462E4600E0AF
:107C10009846BAF8003024495BF8232028461123FF
:107C2000F8F70AFF00EBC00400EB840089FB003486
:107C30000444C017C0EB6434C4F13C00C6F13C02FC
:107C400007F14101012600B208F1410300901BB287
:107C5000019612B209B2154803F018FE08EB0603AC
:107C600005F211153C2B2646ADB24746D0D1342241
:107C70006B210E4804F09CF900210C4804F09CF99B
:107C80000B4B1B8810AA02EB830353F8344C20469D
:107C900009F016F802460548214611B0BDE8F04F3C
:107CA00004F020BB841C0100FC150100889EFF1F0E
:107CB000E89BFF1F6014010009000280214B70B592
:107CC000B3F9003083EAE374A4EBE374002B82B0D1
:107CD000A1B22FDB68466D46012300E0134603EB9B
:107CE000830252009442F9DA174E91FBF3F286FBBD
:107CF00003E403FB1211DB173032D3EBA40389B288
:107D000005F8012BF1D119462B70FFF703FF0F4B3C
:107D10001B786BB101210E4804F04EF93322742117
:107D20000B4804F045F901220A49094804F0DAFA3F
:107D300002B070BD2D238DF800300DF101056846AD
:107D4000CAE700BF9C9DFF1F67666666789DFF1FA0
:107D5000889EFF1F5C28010010B5424C424882B04B
:107D600003F03CFA2378C3B906213F4804F024F914
:107D70002378012B37D90A22022B11463A486BD0BF
:107D800004F016F939490322374804F0ABFA3648B3
:107D900002B0BDE8104004F0BBBA354B1A7801219F
:107DA0000523002A35D10191009311462E4803F096
:107DB000BDFD304B1A78002A36D0052301220192EE
:107DC000009300220A21284803F02EFD2A4B1A783E
:107DD000002A35D101210523019100931421224865
:107DE00003F0A4FDC0E7254C2388092B32D9632B6F
:107DF0008CBF0A211F210A221B4804F0D9F82188D0
:107E0000194804F0D5FA184802B0BDE8104004F053
:107E10007FBA0022019100931146134803F004FD3C
:107E2000144B1A78002AC8D105230121019100932F
:107E30000A210D4803F07AFD0F4B1A78002AC9D0A9
:107E4000012205230192009300221421064803F029
:107E5000EBFC89E73021CEE704F0AAF803220849B9
:107E600092E700BF079FFF1F889EFF1F5824010055
:107E7000219EFF1F229EFF1F239EFF1F429EFF1F6A
:107E800054240100F8B56D4D287840B96C4B1B683F
:107E900099425CD36B4A012313702B70F8BD0C46DA
:107EA00000266948664F03F099F904F6AC53324650
:107EB00065483B6031212E7004F07AF80121624858
:107EC000624D04F07FF831465F4804F075F80522F2
:107ED0005F495D4804F006FA5B4804F019FA0C2289
:107EE0001021594804F064F80B225A49564804F00E
:107EF000F9F905225849544804F0F4F9524804F0BD
:107F000007FA564B50481C68A4F69803C3EB0313BA
:107F100085FB03251D441021DB172022C3EB6525BB
:107F200004F046F840F6CC339C4205F124054FF0AE
:107F300022014FF004000BDCFFF7CAFC484B1C8801
:107F4000064674B3012C46D0022C41D00120F8BD66
:107F5000FFF71EFD092243493B4804F0C3F92A22DA
:107F60001021394804F024F83F4C374884FB05348D
:107F7000EB17C3EBA404214604F01AFA01223B4993
:107F8000314804F0AFF904EB8401A5EB41012E4820
:107F900004F00EFA012236492B4804F0A3F901201F
:107FA000F8BD34491022284804F09CF9264804F012
:107FB000AFF92A221021244803F0FAFF3146224863
:107FC00004F0F6F907222C491F4804F08BF9CBE79F
:107FD0000C222A49E7E70C2229491B4804F082F9C0
:107FE000194804F095F92A221021174803F0E0FF00
:107FF000314615481C4E04F0DBF907221E49124891
:1080000004F070F986FB0536EB17C3EBA606314684
:108010000D4804F0CDF9224614490B4804F062F9EA
:1080200006EB8601A5EB4101074804F0C1F92246A1
:108030000F49054804F056F92046F8BD0C8BFF1F88
:10804000F09EFF1F049FFF1F889EFF1F3B773B98FA
:108050005C240100642401004C240100FC9DFF1FEE
:10806000749DFF1F7024010067666666782B01000F
:10807000E82A01007C24010090240100A8240100CA
:10808000982401002DE9F041754C2278002A05461C
:108090000F4614BF4FF001084FF000084ED1714E4B
:1080A0003368CB1AB3F5FA6F04D86B78A3B940469E
:1080B000BDE8F0816C4B6D486D49DFF8D0E11A7076
:1080C000012303700988237026208EF8002000F019
:1080D000F1FD6B78002BEAD03760F9F715FD654AA2
:1080E000654B6649127828781B78097802EB4303C0
:1080F000421E03EB81030E2AD9D801A151F822F0C8
:10810000F1810000BD810000AF800000F18100001E
:10811000AF800000AF800000AF800000A5810000AC
:10812000AF80000057810000AF800000AF800000EA
:10813000AF800000AF80000053810000AF215048A5
:10814000484E02F0FBFDFFF707FE00233760237067
:10815000ABE705F0DFFA4A4803F040F8022148484F
:1081600003F02AFF0F222321454803F021FF0522B7
:108170004449434804F0B6F8414804F0C9F81E22C7
:1081800023213F4803F014FF05223F493C4804F0F7
:10819000A9F83B4804F0BCF8394803F02BF900F08B
:1081A000ADFC84E7394D2B78012B50D9304B26207C
:1081B000198800F07FFD00232B7078E7002B3FF437
:1081C00076AF013B324A32F81330002B3FF46FAFE9
:1081D000274C304825492D4A23804FF001080023C1
:1081E000037081F8008082F80080FFF7B5FD5EE73C
:1081F00093B1013B264A32F8131019B31C4B254D9D
:108200001A4C224A19800026012326202E70237042
:10821000137000F04FFD15E0154C1E4922880B70BD
:1082200004284FF6FF7002F1FF310CBF0122024615
:108230000A440E4E154D02F07F02013201212280C8
:1082400031702B70FFF788FD4FF001082FE70649CA
:10825000064A01230020087013702370A6E700BFB0
:108260000C8BFF1F009FFF1F049FFF1FDB9BFF1F47
:10827000429EFF1F219EFF1F229EFF1F239EFF1F66
:10828000889EFF1FB8240100C0240100079FFF1F24
:10829000549DFF1F4C9CFF1F2DE9F04F05468BB0EE
:1082A0000F46AD480121164603F08CFEAA8812F055
:1082B000010440F0B080DFF8CC8298F80030002B49
:1082C0007DD1AB79A54AD15CA1B9DFF8BCA27978A0
:1082D0001AF8039041B339780139072900F2B780C1
:1082E000DFE811F0F1005401B5006C01B500B500F4
:1082F000B500E9007C78002C00F0CA800139EC68F8
:10830000387854F82170FC68411EB4F800800729C1
:1083100000F2A780DFE811F074015901A5006C019B
:10832000A500A500A5009F00DFF854A2DAF8002000
:10833000B21AB2F5967F75D9894A107801281ABF0A
:10834000012010701170874A18BF0146D05CC0EB45
:108350000900C0B2FFF7F4F80124CAF80060AB8846
:108360009B0770D57B78002B6DD0F9F7CDFB7E4B4A
:108370007E4A7F481B78127839780078022515FBF1
:1083800002330A2903EB800300F04E810C295AD1F5
:10839000002B58D003F11900764E774A013B00219B
:1083A000400080B226F813100123157088F80030C1
:1083B00000F080FC714B032220461A702FE06648C3
:1083C00002F00CFF0121644803F0F6FD62482246EA
:1083D000214603F0EDFDAB88580725D42C682046D4
:1083E00008F06EFC214602465B4803F07BFF5A48CA
:1083F00003F08EFF092201238DE80C0000217F236A
:10840000554803F043FA00212846FFF7EFFA00230E
:1084100088F8003055E7AB683146384698470BB0CE
:10842000BDE8F08F0846FAE72B6804A8984704A82F
:1084300008F046FC04A90246474803F053FF4648AB
:1084400003F066FFD6E720460BB0BDE8F08F0024AE
:108450000AF8039083E70021D1543846FB69984716
:10846000FC68A4F80080002725223C238DE88400C6
:1084700041211822384803F0D7F9E968A879FFF7B5
:1084800091FB374A3E4B17701E600BB0BDE8F08F72
:108490003B490A68B21AB2F5967FD4D9304F0E60C4
:1084A0003E78012E00F0B480E968184601233B7045
:1084B000FFF778FBB3E7304AE9791170012288F8B9
:1084C00000200024C4E72A7A013A4A45BFDD09F1B9
:1084D0000104E4B2A145BAD0224E16F803B0CBEBAA
:1084E0000900C0B20021FFF72BF82B7A052BD946E3
:1084F0001BD9CBEB0402042A40F3AE80A4F1040B99
:10850000BBF1000FC0F2B080063B5B45A8BF5B46E5
:108510005FFA83F9AA791348B15C994205D000F853
:10852000029001212846FFF761FAC9EB0400C0B2AE
:1085300001210B4EFFF704F8002134230191009331
:108540000548317040230B223F21A14603F06CF90E
:108550000124AB797CE700BF889EFF1FF49EFF1FBC
:10856000059FFF1F809EFF1F219EFF1F229EFF1F52
:10857000239EFF1F549DFF1F049FFF1F079FFF1F88
:10858000EC9EFF1F0C8BFF1F6C9EFF1F0FFA89F1E3
:10859000E868604C50F821602168049134785E49A5
:1085A00004980860002C71D0012C7FF450AF5B4A16
:1085B000317A88F800401170002449E7B9F1000FC2
:1085C00050D009F1FF34E4B284E7B98A01F0040124
:1085D00089B200293FF440AF3B6A03929847039A5F
:1085E00000283FF43DAFAB79FC680021D15438E757
:1085F0007B8A43453CD908F101081FFA88F830E727
:108600003B8A43453BD208F1FF381FFA88F828E738
:1086100025238DE8180042483C703C231822412154
:1086200003F002F93046FAE6002B3FF40CAF3D4A66
:108630003D4E1188394A03F11900013B400080B2D8
:1086400026F81310012388F80030157000F032FB73
:10865000364B20461D70E2E6002A3FF755AF04F185
:10866000FF3B4DE74C46F3E64FF000094B4651E720
:10867000BB8ADA077FF5F5AEB7F81080F1E6BB8A62
:10868000D9077FF5EEAEB7F81280EAE62849C85C54
:10869000C0EB090009F1010EC0B201214FF0340B0B
:1086A00002F803E0FEF74CFFB6681D480194402332
:1086B0000B223F210124CDF800B003F0B5F8402390
:1086C0000B223F211648CDF800B0019403F02EF99B
:1086D0002146134803F070FC304608F0F1FAA0EB95
:1086E000800000F15F0109B20F220D4803F060FC29
:1086F000304608F0E5FA31460246094803F0F2FD3B
:10870000074803F005FEE968A879FFF74BFAAB7953
:108710009EE600BF449FFF1FEC9EFF1F049FFF1FAC
:10872000889EFF1F429EFF1F549DFF1F079FFF1F34
:10873000809EFF1F2DE9F047DFF808926D4B99F8F6
:1087400000601B68DFF800A282B0003601934FF092
:10875000030018BF0126019F9AF8008004F092FCE4
:108760000546042004F08EFC0446052004F08AFC33
:10877000800040EA4404062004F084FC2C4364B2E8
:108780005D4944EAC0000A7880F00F03DBB29A42E8
:108790005A4A3CD01760002259480B7003788DF874
:1087A00000808DF8012053B3564A12684EF66021BE
:1087B000BA1A8A4219D8022B59D0012B5FD0062B46
:1087C00048D0032B63D0042B69D0052B77D0072B1F
:1087D0007DD0082B00F08380092B68D016B14A4861
:1087E00002F008FE02B0BDE8F087484A484C00237A
:1087F0000121237003701360938089F800103A46BA
:1088000069464448FFF748FD3043C6B2E6E71268C0
:10881000BA1A1E2A6BD99AF80020934222D0394CFA
:108820003D488AF80030012B276082EA0302076086
:108830009846B1D0042BAFD137480068381AB0F54C
:10884000C87FA9D9354C2068381A3228A4D92760A6
:108850001A46A1E73A4669463148FFF71DFD304305
:10886000C6B2BBE7012B4FF00002E3D1E4E73A4682
:1088700069462C48FFF710FD3043C6B2AEE73A46D2
:1088800069462948FFF708FD3043C6B2A6E73A46D5
:1088900069462648FFF700FD3043C6B29EE73A46D8
:1088A00069462348FFF7F8FC3043C6B296E73A46DC
:1088B00069462048FFF7F0FC3043C6B28EE73A46DF
:1088C00069461D48FFF7E8FC3043C6B286E73A46E2
:1088D00069461A48FFF7E0FC3043C6B27EE73A46E5
:1088E00069461748FFF7D8FC3043C6B276E7002246
:1088F00052E700BF449FFF1F089FFF1F749EFF1F8A
:10890000049FFF1FFC9EFF1F889EFF1FF49EFF1FFA
:10891000069FFF1FCC1E01000C9FFF1F7C9EFF1FA8
:10892000FC220100241E01004C1D0100C41C01009A
:10893000382A01003C1D0100A41D0100081E010091
:108940005490FF1F0C8BFF1F789EFF1F28B110282B
:10895000044BA8BF102018607047024B012018601C
:10896000704700BF109FFF1F38B50F4D2B78013B9C
:1089700001381B02C4B203F47063200443F4404383
:1089800043F00C0300F4FE00184305F0E3FC2868F4
:10899000013860F03F00C0B204F00AFD2046BDE897
:1089A000384004F005BD00BF109FFF1F70B5124D89
:1089B0002B78013B1B0203F47063064643F43043FB
:1089C0000806320400F0FE4043F00B03034302F4B8
:1089D000FE0018430C4605F0BDFC2868013860F025
:1089E0004F00C0B204F0E4FC304604F0E1FC204645
:1089F000BDE8704004F0DCBC109FFF1F70B5124D45
:108A00002B78013B1B0203F47063064643F41043CA
:108A10000806320400F0FE4043F00903034302F469
:108A2000FE0018430C4605F095FC2868013860F0FC
:108A30006F00C0B204F0BCFC304604F0B9FC204624
:108A4000BDE8704004F0B4BC109FFF1F38B5104D56
:108A50002B78013B1B0203F47063044643F410437C
:108A6000000443F0090300F4FE00184305F072FC13
:108A70002868013860F06F00C0B204F099FC20460D
:108A800004F096FC0020BDE8384004F091BC00BF23
:108A9000109FFF1F38B50E4D2B78013B1B0203F4CE
:108AA0007063044643F45043000443F00D0300F4A4
:108AB000FE00184305F04EFC2868013860F02F00D6
:108AC000C0B204F075FC2046BDE8384004F070BC2C
:108AD000109FFF1F08B5002005F006FD0028FAD101
:108AE00008BD00BF08B564210720FFF75FFF7F21A5
:108AF0000B20BDE80840FFF759BF00BF10B50021AB
:108B00007B20FFF753FF0024E0B2FFF79FFF013403
:108B1000022004F0EDFA802CF6D110BD10B5044609
:108B20004FF4406004F0F4FB04F04CFC2CB1102C2A
:108B3000044BA8BF10241C6010BD024B01241C6014
:108B400010BD00BF109FFF1F10B5044641F0E000AC
:108B500004F02EFC04F07F0004F02AFCC4F3C610DD
:108B6000BDE8104004F024BC38B5134D2B78044602
:108B700041F6FF72A0F50050824203F1FF33A8BF17
:108B800002461B0202F5005203F47063100443F422
:108B9000604343F00E0300F4FE005204184302F059
:108BA000FE42104305F0D6FB296801392046C9B2C0
:108BB000BDE83840FFF7C8BF109FFF1F38B5044617
:108BC0000D46F02004F0F4FB35B1254414F8010BF8
:108BD00004F0EEFBAC42F9D1F720BDE8384004F0D8
:108BE000E7BB00BF00B50B4B83B0024699881868FD
:108BF0000090032AADF8041002D903B05DF804FB1D
:108C0000684606218DF80520FFF7D8FF03B05DF810
:108C100004FB00BFA82A010000B50B4B024683B03D
:108C2000186899880090131F4C2BADF8041002D9D6
:108C300003B05DF804FB684606218DF80520FFF7B8
:108C4000BDFF03B05DF804FBB02A0100030203F48A
:108C5000FE43C0F3C6101843704700BF0378407846
:108C6000DB0103F47E5300F07F001843704700BF20
:108C700082B002AA114642F8040D002012F8013B0E
:108C800003F07F03914243EA0020F7D102B070471E
:108C9000003210B403884FF0010404FA01F418BF45
:108CA000012202FA01F123EA04020A43028010BC05
:108CB000704700BF70B5CEB20C46054603F0AAFD62
:108CC000864203D03146284603F0BEFD01352846D2
:108CD00003F0A0FD240A844205D021462846BDE8C1
:108CE000704003F0B1BD70BD38B5054603F092FD8C
:108CF0004FF0000460F30704681C03F08BFD60F381
:108D00000F24A0B238BD00BFF8B504460020FFF71D
:108D1000EBFF002C00F0F4844FF4AF610220FFF76A
:108D2000C9FF4FF47A610420FFF7C4FF4FF4966146
:108D30000620FFF7BFFF4FF4FA610820FFF7BAFFE4
:108D40004FF4AF610A20FFF7B5FF40F6FC010C209D
:108D5000FFF7B0FF4FF496612220FFF7ABFF4FF40F
:108D600016612420FFF7A6FF7D212A20FFF7A2FF2E
:108D70000C210E20FFF79EFF01211020FFF79AFF24
:108D800002211220FFF796FF00211420FFF792FF27
:108D900000211620FFF78EFF02211820FFF78AFF1F
:108DA00001211A20FFF786FF02211C20FFF782FF16
:108DB00004211E20FFF77EFF14212020FFF77AFFF9
:108DC00001212620FFF776FF03212820FFF772FFFD
:108DD00004212C20FFF76EFF0F212E20FFF76AFFE2
:108DE00000213020FFF766FF0C213220FFF762FFE1
:108DF00000213420FFF75EFF00213620FFF75AFFE5
:108E000000213820FFF756FF00213A20FFF752FFDC
:108E100000213C20FFF74EFF00213E20FFF74AFFD4
:108E200000214020FFF746FF00214220FFF742FFCC
:108E30001F214420FFF73EFF13214620FFF73AFF92
:108E40000E214820FFF736FF11214A20FFF732FF9D
:108E50000A214C20FFF72EFF00214E20FFF72AFFAA
:108E600006215020FFF726FF02215220FFF722FFA4
:108E70000C215420FFF71EFF00215620FFF71AFF98
:108E800000215820FFF716FF01215A20FFF712FF9B
:108E900003215C20FFF70EFF0A215E20FFF70AFF87
:108EA00000216020FFF706FF04216220FFF702FF88
:108EB00001216420FFF7FEFE00216620FFF7FAFE85
:108EC0000B216820FFF7F6FE7F216A20FFF7F2FEF4
:108ED00000216C20FFF7EEFE00216E20FFF7EAFE76
:108EE00000217020FFF7E6FE00217220FFF7E2FE6E
:108EF00000217420FFF7DEFE1F217620FFF7DAFE47
:108F000013217820FFF7D6FE0E217A20FFF7D2FE3C
:108F100011217C20FFF7CEFE0A217E20FFF7CAFE3A
:108F20001F218020FFF7C6FE13218220FFF7C2FE1B
:108F30000E218420FFF7BEFE11218620FFF7BAFE26
:108F40000A218820FFF7B6FE00218A20FFF7B2FE33
:108F500001218C20FFF7AEFE00219620FFF7AAFE2C
:108F600000219820FFF7A6FE00219A20FFF7A2FE1D
:108F700005219C20FFF79EFE26210020FFF79AFE88
:108F80000220FFF7B1FEB0F5805F034680F0228536
:108F9000D24A04201380FFF7A7FEB0F5805F034696
:108FA00080F00F85CE4A06201380FFF79DFEA0F5C6
:108FB0002F739BB2B3F57A6F024606D940F628218B
:108FC0000620FFF777FE40F62822C64B08201A80BD
:108FD000FFF78AFEA0F52F739BB2B3F57A6F0246B6
:108FE00006D940F6E4410820FFF764FE40F6E4426B
:108FF000BD4B0A201A80FFF777FEA0F5FA739BB2EB
:1090000040F6AC518B42024606D94FF4AF610A20BC
:10901000FFF750FE4FF4AF62B44B0C201A80FFF7FD
:1090200063FEA0F5FA739BB240F6AC518B42024648
:1090300006D940F6FC010C20FFF73CFE40F6FC028E
:10904000AB4B0E201A80FFF74FFE1828034600F2A4
:10905000B184A84A10201380FFF746FE431E9BB23E
:109060000F2B024604D901211020FFF723FE012215
:10907000A14B12201A80FFF737FE0A28034600F2A0
:1090800092849E4A14201380FFF72EFE0128034687
:1090900004D900211420FFF70DFE0023984A162062
:1090A0001380FFF721FE7F28034600F27584954A5E
:1090B00018201380FFF718FE0428034600F2658489
:1090C000914A1A201380FFF70FFE0C28034600F286
:1090D00055848E4A1C201380FFF706FE04280346A1
:1090E00000F245848A4A1E201380FFF7FDFD0928FF
:1090F000034600F23584874A20201380FFF7F4FDF1
:109100004628034600F22584834A22201380FFF775
:10911000EBFDA0F5FA739BB240F6AC518B420246D0
:1091200006D94FF496612220FFF7C4FD4FF49662F2
:109130007A4B24201A80FFF7D7FDA0F5FA739BB273
:1091400040F6AC518B42024606D94FF416612420FA
:10915000FFF7B0FD4FF41662714B26201A80FFF71F
:10916000C3FD7F28034600F2EE836E4A2820138059
:10917000FFF7BAFD0628034600F2DF836A4A2A2079
:109180001380FFF7B1FDA0F132039BB2B3F5967FD8
:10919000024604D97D212A20FFF78CFD7D22634BF6
:1091A0002C201A80FFF7A0FD0C28034600F2BF8395
:1091B0005F4A2E201380FFF797FD1E28034600F21A
:1091C000B0835C4A30201380FFF78EFD09280346E8
:1091D00000F2A183584A32201380FFF785FD1E2834
:1091E000034600F29283554A34201380FFF77CFD3A
:1091F0007F28034600F28383514C36202380FFF7FB
:1092000073FD7F28034600F2748338206380FFF7E4
:109210006BFD7F28034600F266833A20A380FFF7A8
:1092200063FD7F28034600F258833C20E380FFF76C
:109230005BFD7F28034600F24A833E202381FFF72F
:1092400053FD7F28034600F23C8340206381FFF7F3
:109250004BFD7F28034600F22E834220A381FFF7B7
:1092600043FD384D28804420FFF73EFD302803465B
:1092700000F21B83344A46201380FFF735FD302867
:10928000034600F20C83314C48202380FFF72CFD6D
:109290003028034600F2FD824A206380FFF724FD58
:1092A0003028034600F2EF824C20A380FFF71CFD1C
:1092B0003028034600F2E1824E20E380FFF714FDE0
:1092C0000128034604D900214E20FFF7F3FC0023B8
:1092D0001F4A50201380FFF707FD3BE07E9CFF1FD5
:1092E000329EFF1F3A9CFF1F109EFF1FE09DFF1F35
:1092F000009CFF1FD49BFF1F9C9DFF1FD09DFF1F45
:10930000769CFF1FD89BFF1F829CFF1F229CFF1F84
:109310001A9CFF1FE49BFF1F1C9EFF1F969DFF1FB3
:109320008C9DFF1F429EFF1FEC9DFF1F2C9EFF1F69
:10933000E89BFF1F709CFF1FC49BFF1F129EFF1F17
:10934000549DFF1FF89BFF1FFA9BFF1FF09DFF1FFF
:10935000189CFF1F431E9BB20B2B024604D906210B
:109360005020FFF7A7FC0622C14B52201A80FFF7BE
:10937000BBFC0428034600F27A82BE4A54201380C4
:10938000FFF7B2FC431E9BB21D2B024604D90C21F1
:109390005420FFF78FFC0C22B74B56201A80FFF7A2
:1093A000A3FC0128034604D900215620FFF782FCC4
:1093B0000023B24A58201380FFF796FC7F2803460B
:1093C00000F24F82AE4A5A201380FFF78DFC431EF5
:1093D0009BB2092B024604D901215A20FFF76AFCEF
:1093E0000122A84B5C201A80FFF77EFC431E9BB233
:1093F000102B024604D903215C20FFF75BFC0322FB
:10940000A14B5E201A80FFF76FFC431E9BB21D2B01
:10941000024604D90A215E20FFF74CFC0A229B4B2E
:1094200060201A80FFF760FC0228034600F21382D6
:10943000974A64201380FFF757FC0128034604D99C
:1094400001216420FFF736FC0123924A6220138039
:10945000FFF74AFCC31E9BB2012B024604D904212C
:109460006220FFF727FC04228B4B66201A80FFF74F
:109470003BFC7F28034600F2E881884A682013807D
:10948000FFF732FC7F28034600F2D981844A6A2024
:109490001380FFF729FC7F28034600F2CA81814A26
:1094A0006C201380FFF720FC0428034600F2BB81E8
:1094B0007D4A6E201380FFF717FC1928034600F23F
:1094C000AC817A4A70201380FFF70EFC0228034615
:1094D00000F29D81764A72201380FFF705FC062872
:1094E000034600F28E81734A74201380FFF7FCFB61
:1094F0000428034600F27F816F4A8A201380FFF719
:10950000F3FB0A28034600F270816C4A8C2013801A
:10951000FFF7EAFB0428034600F26181684A9820BD
:109520001380FFF7E1FB0128034604D900219820AE
:10953000FFF7C0FB0023634A9A201380FFF7D4FB98
:109540000128034604D900219A20FFF7B3FB00232A
:109550005D4A96201380FFF7C7FB0B28034600F2F5
:1095600038815A4A9C201380FFF7BEFB831E9BB2B2
:10957000032B024604D905219C20FFF79BFB052203
:10958000534B76201A80FFF7AFFB3028034600F2DA
:109590001A81504A78201380FFF7A6FB3028034633
:1095A00000F20B814C4C7A202380FFF79DFB302882
:1095B000034600F2FC807C206380FFF795FB302897
:1095C000034600F2EE807E20A380FFF78DFB30285B
:1095D000034600F2E0808020E380FFF785FB30281F
:1095E000034600F2D2803D4A82201380FFF77CFBC5
:1095F0003028034600F2C380394C84202380FFF7D3
:1096000073FB3028034600F2B48086206380FFF7A6
:109610006BFB3028034600F2A6808820A380FFF76A
:1096200063FB302800F299802B88DFF8CCC02D4FE7
:10963000E08003F00100DFF8C4E02B4EACF800003E
:10964000C3F340003880294D29492A4AC3F38000DA
:10965000C3F3C007C3F30014AEF800003770C3F3C0
:109660004010C3F380132C8008801380F8BD00BF26
:10967000108AFF1F5E89FF1F128AFF1F629CFF1F57
:10968000DE9DFF1FD09BFF1F608AFF1F5C89FF1FAD
:10969000889DFF1FE89DFF1F289CFF1F1E9EFF1F28
:1096A000549CFF1F0E9CFF1FC09BFF1F5C9EFF1F53
:1096B000749DFF1F389EFF1F089EFF1F9E9DFF1F6A
:1096C000829DFF1F0C9CFF1F689CFF1FD89DFF1FE2
:1096D000EE9BFF1F029CFF1F649DFF1F049CFF1F4A
:1096E0006C9DFF1F389CFF1F789DFF1F8A9DFF1FE9
:1096F000EA9DFF1FA29DFF1FDA9DFF1F729CFF1FA7
:109700004FF6FF7398423FF407AB26283FF438AC7E
:1097100017287FF601AB19287FF66AAB1B287FF666
:1097200087AB1C283FF49CAB1E287FF6A1AB1F28FB
:109730003FF4A6AB20283FF4BFAB21283FF4C8ABD1
:1097400022283FF4CDAB23283FF4D6AB24283FF4A6
:1097500007AC25287FF410AC0AE488200A21FFF723
:10976000A9FA0A2060E711218620FFF7A3FA112346
:1097700053E70E218420FFF79DFA0E2345E71321BE
:109780008220FFF797FA132336E71F218020FFF787
:1097900091FA1F2327E70A217E20FFF78BFA0A237D
:1097A00019E711217C20FFF785FA11230BE70E2121
:1097B0007A20FFF77FFA0E23FDE613217820FFF7CA
:1097C00079FA1323EEE61F217620FFF773FA1F23A1
:1097D000DFE600219620FFF76DFA0023C1E60121A4
:1097E0008C20FFF767FA012398E600218A20FFF713
:1097F00061FA002389E600217420FFF75BFA002359
:109800007AE600217220FFF755FA00236BE600216B
:109810007020FFF74FFA00235CE600216E20FFF76F
:1098200049FA00234DE600216C20FFF743FA00239C
:109830003EE67F216A20FFF73DFA7F232FE60B21CA
:109840006820FFF737FA0B2320E600216620FFF798
:1098500031FA002311E600216020FFF72BFA0023E4
:10986000E6E500215820FFF725FA0023AAE50221AA
:109870005220FFF71FFA02237FE50A214C20FFF751
:1098800019FA0A2318E511214A20FFF713FA1123C8
:109890000AE50E214820FFF70DFA0E23FCE4132100
:1098A0004620FFF707FA1323EDE41F214420FFF7BA
:1098B00001FA1F23DEE400214020FFF7FBF900231B
:1098C000CBE400213E20FFF7F5F90023BDE40021A1
:1098D0003C20FFF7EFF90023AFE400213A20FFF727
:1098E000E9F90023A1E400213820FFF7E3F9002380
:1098F00093E400213620FFF7DDF9002385E4002101
:109900003420FFF7D7F9002376E40C213220FFF74B
:10991000D1F90C2367E400213020FFF7CBF90023B5
:1099200058E40F212E20FFF7C5F90F2349E4042145
:109930002C20FFF7BFF904233AE403212820FFF786
:10994000B9F903231AE401212620FFF7B3F9012313
:109950000BE414212020FFF7ADF91423FFF7D4BB4B
:1099600004211E20FFF7A6F90423FFF7C4BB022140
:109970001C20FFF79FF90223FFF7B4BB01211A2037
:10998000FFF798F90123FFF7A4BB02211820FFF786
:1099900091F90223FFF794BB00211620FFF78AF903
:1099A0000023FFF784BB02211220FFF783F9022373
:1099B000FFF767BB0C210E20FFF77CF90C23FFF7A4
:1099C00048BB4FF47A610420FFF774F94FF47A63CF
:1099D000FFF7E8BA4FF4AF610220FFF76BF94FF4DD
:1099E000AF63FFF7D5BA00BFF8B5AF2006F0C8FBEC
:1099F000204B214A054603CB1368C5F803001A0C17
:109A00009E20C5F807102B80AA70FFF71FF92E467D
:109A1000002426F80B0FA0B2FFF766F9FFF716F93E
:109A200002349E2C26F8020FF5D16C1E05F1AA0611
:109A30004FF0FF3014F8013F082758400F4B40F318
:109A400000017A1E0B4012F0FF0783EA5000F5D1A7
:109A5000B442EFD1C043FFF70BF93A46C5F8AB006B
:109A6000AF21284604F0C4FC2846BDE8F84006F0C3
:109A70008FBB00BFBC2A0100B82A01002083B8EDCB
:109A8000F0B50E4B0E4C054693E8070085B02468F0
:109A90002E88AD7801AB83E80700270C184600221A
:109AA0000B21ADF804408DF80670ADF80C608DF810
:109AB0000E5004F09DFC05B0F0BD00BFC82A0100A7
:109AC000B82A0100F0B5124B124D1E68124F0FCD8F
:109AD00087B06C460FC495E8030044F8040B38685F
:109AE0003B79CDF80D00320C262021808DF8022024
:109AF0008DF81130ADF80060FFF7A8F80022ADF83E
:109B00000B001221684604F073FC07B0F0BD00BFE3
:109B1000B82A0100D42A01004C240100002004F0DE
:109B2000E3BC00BF02F02EBE70B5124C82B000251F
:109B30004023064629462046009301958023202293
:109B400001F072FE20222946204602F031FA20461A
:109B5000012102F037FA304607F0B2F831460246EA
:109B6000204602F0BFFB204602B0BDE8704001F085
:109B700041BC00BF889EFF1FF0B5AE2983B075D9E8
:109B80000546441E00F1AA064FF0FF3014F8012FDD
:109B900008275040404A40F300017B1E0A4013F062
:109BA000FF0782EA5000F5D1B442EFD1C043FFF77E
:109BB0005FF80146D5F8AB000190019A914202D0BE
:109BC000B2F17F2F0BD105F10B00FFF747F89E286C
:109BD0000BD03248FFF7A8FF002003B0F0BD30489B
:109BE000FFF7A2FF384603B0F0BD05F10D00FFF707
:109BF00035F8262840D1002440F6AC5613E004285E
:109C00001AD0062821D008281FD00A2828D00C28CE
:109C100022D1A1F5FA7292B2B24201D8FFF74AF806
:109C200002349E2C0ED004F10D002844FFF716F8E4
:109C3000022C0146A0B2E2D1B1F5805FEED302342E
:109C40009E2CF0D1012003B0F0BDA1F52F7292B28D
:109C5000B2F57A6FE4D8E1E7222801D0242811D1A7
:109C6000A1F5FA7292B2B242DAD8D7E70D48FFF7FF
:109C70005BFF002003B0F0BD0B48FFF755FF00204D
:109C800003B0F0BD2A28C9D1A1F1320292B2B2F5D7
:109C9000967FC5D8C2E700BF2083B8ED182B01001E
:109CA000042B0100EC2A01002C2B010003290CD904
:109CB00070B5461C82B005460C46304603222A4940
:109CC00007F06CF810B102B070BD70470B2C05D9CD
:109CD00005222649281D07F061F840B12448FFF706
:109CE00023FF244802B0BDE87040FFF7C9BE05F16C
:109CF0000901032201A807F0A1F801A803221E49C7
:109D000007F04CF8D8B103221C4901A807F046F827
:109D100008B301A803221A4907F040F8B0B919485E
:109D2000FFF702FFA11E89B23046FFF725FF00288A
:109D3000C9D0154802B0BDE87040FFF7F5BE134822
:109D4000FFF7F2FEFFF750FE1148F3E71148FFF767
:109D5000EBFE1148C6E71148FFF7E6FE02B0BDE88A
:109D60007040FFF7AFBE00BFB82A0100442B0100CE
:109D70004C2B0100602B0100642B01008C2B010097
:109D8000A42B0100A82B0100BC2B0100682B0100B3
:109D90007C2B0100D02B0100E42B0100902B010053
:109DA0002DE9F043174D2B6883B081460F4690464E
:109DB000F3B1154E34880A1992B218461146328012
:109DC00006F05CFD28603A464946204402F06CFDEE
:109DD000B8F1000F09D031882868FFF767FF2868BD
:109DE00006F0D6F900232B60338003B0BDE8F08382
:109DF000054E01930846318006F0C2F9019B2860A8
:109E00001C46E0E7189FFF1F149FFF1F10B51F4C53
:109E10004FF4FA70FCF7C4F8204601F0DFF9002295
:109E20001146204602F0C4F82046012102F0CAF88B
:109E30002046002102F0C0F80B221549204602F00E
:109E400051FA204602F064FA0F221249204602F02D
:109E500049FA204602F05CFA0F490722204602F038
:109E600041FA204602F054FA204601F0C3FA0B4BA7
:109E70000B4A1A604FF4FA70FCF792F8FFF722FED3
:109E80000848BDE81040FFF74FBE00BF889EFF1F87
:109E9000E82B0100F42B0100042C0100D0A0FF1FCF
:109EA000A19D00000C2C01000020704790F8392083
:109EB00090F83800101A704790F8383090F8392030
:109EC0009A4205D95A1C034480F83820187E7047FE
:109ED0004FF0FF30704700BF90F8383090F83920CD
:109EE0009A4286BF1B18187E4FF0FF30704700BFA4
:109EF000704700BF38B50546B0F85E0090B195F8E0
:109F00005D301446C3F1210294420CD805F13B00A8
:109F10001844224602F0C8FC95F85D30234485F8C9
:109F20005D30204638BD012014462871EEE700BFA1
:109F3000B0F85E306BB190F85D30202B07D8C218B6
:109F4000013380F85D30012082F83B107047012317
:109F500003710020704700BF0023426980F8383049
:109F600080F8393080F85C3080F85D3080F85E3001
:109F700080F85F3006CA30B40D68046943662A432E
:109F800083660A60A370426990F8613016491468CC
:109F900013441D7A5B7B01EBC5051B026D6803F45E
:109FA000E06343F064032B6090F8623013449D7CBF
:109FB000DB7D01EBC5011B02496803F4E06343F05C
:109FC00064030B6021685368194205D00369272296
:109FD0005A70036904229A71036920225A71036935
:109FE00080229A7030BC70474037010043690CCB27
:109FF00012681A420CD0094B99420AD9084B99426F
:10A00000036994BF1A220D225A70036904229A71BF
:10A010007047036927225A70F7E700BF7F1A0600CE
:10A020003F420F0010B50269D378DBB2D90604466F
:10A030003DD510215806D17038D503F0040303F044
:10A04000FF02002B51D03D49626E00230B7084F853
:10A050005D30002A5BD0904794F85D30002B56D0DD
:10A060002369D0229A70236994F83B201A712369DE
:10A07000012284F85C200222DA7010BD304B84F893
:10A0800060009C424AD02F4B9C4252D094F8391029
:10A0900013791F29DBB207D82848007820B160184F
:10A0A000013184F8391003760223D37010BD5906AC
:10A0B000C3D4917801F0100101F0FF000029DDD038
:10A0C00013F001031ED194F85C1094F85D008842EF
:10A0D00081BF4B1C091984F85C3091F83B30137137
:10A0E0002369D0229A702269DEE7236984F8392037
:10A0F000C0229A702369114A197901211170022234
:10A10000DA7010BDC023937022691379CCE7012265
:10A11000002384F85D2084F83B30A1E7626994F85D
:10A120006130094913440322187A02F043FD226981
:10A13000ACE7626994F861300449F3E71C9FFF1FA4
:10A14000A090FF1F0C91FF1FADA10000B9A100005E
:10A150000369DB7803F0200373B190F860300133BA
:10A16000DBB2012B80F860301AD9426990F8613077
:10A170001344187A02F09ABD70B5426903F0FF05E6
:10A1800090F8613013440446187A02F08FFDA36EF4
:10A190005BB184F8385094F83900BDE87040184736
:10A1A00090F85F30002BE0D0704770BD0148FFF79A
:10A1B000CFBF00BFA090FF1F0148FFF7C9BF00BF7E
:10A1C0000C91FF1F2DE9F047374FDFF8E0903B6817
:10A1D000026982B006460093DDF800800021A025C8
:10A1E000D3789B065BD53B680193019BC8EB0303C7
:10A1F0000F2BF5D949B1102BF2D0002090703369A4
:10A2000080229A7002B0BDE8F087726996F86130DA
:10A2100013440521187A02F043FF726996F8613001
:10A220001344012193F812A0504602F039FF09248B
:10A230000021504602F020FF2B46013BFDD10121B9
:10A24000504602F019FF2B46013BFDD1013CEFD1F6
:10A25000706996F8611001444FF4A0720C7A4B7B40
:10A2600009EBC4011B02496803F4E06343F0640393
:10A270000B6096F862300344997CDB7D09EBC101E9
:10A280001B02496803F4E06343F064030B60013A86
:10A29000FDD13269D3789B064FF00101A3D4012090
:10A2A00002B0BDE8F08700BF449FFF1F40370100A8
:10A2B000F0B503691222DA700269937803F0200383
:10A2C00085B004460D46002B5ED0B42393703C4904
:10A2D00022690B680093009E05E00B680193019BC7
:10A2E0009B1B042B42D8D37803F0200303F0FF001C
:10A2F000002BF2D094F85D30002B31D04FF0000EDF
:10A300004FF0020C04EB0E0393F83B3013710B6813
:10A310000393039F206907E09B060DD50B6802930A
:10A32000029BDB1B052B28D8C378DBB203F00202AB
:10A3300002F0FF06002AEFD080F803C02669F37808
:10A34000DBB2DF0632462DD49F062BD5DB0731D496
:10A350000EF1010E94F85D305FFA8EFE7345D1D890
:10A3600000201DBB002384F85E3004E09070236958
:10A3700080229A70042005B0F0BD86702369802287
:10A3800004209A7005B0F0BD03F0FF06FFF71AFF36
:10A3900010B9042005B0F0BD236984F85F60B022D5
:10A3A0009A7094E78023B3700420DAE7266980234B
:10A3B000B370D7E7BEF1000F0CBF02200320F6E711
:10A3C000449FFF1F2DE9F04106690025122780F800
:10A3D000385080F83950F770D0F810C09CF802E07F
:10A3E0000EF0200E88B00446884615461E46BEF183
:10A3F000000F49D0B4238CF80230784B21691A68D9
:10A400000092DDF800E006E01A6801920198CEEBB8
:10A410000000042830D8C87800F0200000F0FF07C2
:10A420000028F1D04FEA480242F00102D2B20A718C
:10A430001A680292DDF808E0206906E01A680392C3
:10A440000399CEEB010105292AD8C17801F0020158
:10A4500001F0FF070029F1D04FF0020C80F803C093
:10A460002269D17811F0110722D12DBB002E0CBF2B
:10A47000A0238023937003E08F70236980229A7059
:10A48000384608B0BDE8F0810EF0FF07FFF79AFEEE
:10A490000028F5D0236984F85F70B0229A70ACE789
:10A4A00087702369802238469A7008B0BDE8F08131
:10A4B000802393700027E3E7012D75D0A0219170D0
:10A4C00021690A79BE4667464FF0A80C1A680492C3
:10A4D000049805E01A680592059A121A052A4AD8C6
:10A4E000CA7802F0020202F0FF08002AF2D0CF7010
:10A4F0002169CA78D2B212F0100F08465AD19206DA
:10A5000058D5013DEDB2012D49D0BEF11F0F3BD909
:10A510000A79012DDAD11A680692069D05E01A68BB
:10A520000792079A521B052A46D8C27802F0020207
:10A5300002F0FF01002AF2D00223C3702269D3780F
:10A54000DBB2D9063AD49B0634D5B023BEF11F0F37
:10A5500093703FD8226904EB0E0312791A760EF13C
:10A56000010E5FFA8EFE16B1236980229A7084F87C
:10A5700039E0774684E781F80280236980229A7067
:10A58000774684F839E07BE704EB0E0291F804800B
:10A5900082F818800EF1010E5FFA8EFEB9E781F89D
:10A5A00002C021690846B0E7A82191702069BE4623
:10A5B0000279B0E7774663E78170DEE71021A023D8
:10A5C000D170013BFDD12269937803F0F703774600
:10A5D000937055E723691B79C5E700BF449FFF1FB0
:10A5E0000148FFF71FBD00BFA090FF1F0148FFF704
:10A5F00019BD00BF0C91FF1F704700BF38B5144C48
:10A60000037801225B000546204684F83B3084F83D
:10A610005E2084F85D20FFF78BFC20460021FFF7C9
:10A6200047FE0B4C2978012320461A46FFF7CAFE45
:10A630000128F6D194F8383094F839209A4205D997
:10A64000E218013384F83830107E38BDFF2038BD61
:10A65000A090FF1F38B51B4C037801225B00054614
:10A66000204684F83B3084F85E2084F85D20FFF7B4
:10A670005FFC20460021FFF71BFE124C2978204684
:10A6800001230222FFF79EFE0228F6D194F838201B
:10A6900094F839108A420FD2531CDBB2A0189942A9
:10A6A00084F83830007E0AD9234402321B7E84F8B5
:10A6B000382040EA032038BD4FF6FF7038BD40F423
:10A6C0007F4038BDA090FF1F0C2901D900207047A2
:10A6D0000231490001F0FE01FFF7BCBF70B50C4C20
:10A6E0000378164601255B00204684F83B3084F849
:10A6F0005E5084F85D50FFF71BFC31462046FFF7A3
:10A7000017FC29462046BDE87040FFF7D1BD00BFC9
:10A71000A090FF1FF8B505460F4616464124214676
:10A720003A462846FFF7DAFF611C0234C9B23246C6
:10A730002846E4B2FFF7D2FF592CF0D1F8BD00BF94
:10A7400038B504460D463548FFF706FC63228021E4
:10A7500020462570FFF7C2FF012002F0C9FC204609
:10A7600000225E21FFF7BAFF20465D21FFF746FF7A
:10A77000242801D0002038BD204606220C21FFF7F6
:10A78000C9FF204601222B21FFF7A8FF2046012206
:10A790002C21FFF7A3FF20460E222D21FFF79EFF5D
:10A7A000204600222E21FFF799FF204601222F216B
:10A7B000FFF794FF204605223021FFF78FFF204648
:10A7C00001223121FFF78AFF204600223221FFF7C4
:10A7D00085FF204600223321FFF780FF204600221C
:10A7E0003421FFF77BFF204600223521FFF776FF5B
:10A7F000204600225B21FFF771FF204610225C21DA
:10A80000FFF76CFF204620225D21FFF767FF2046FF
:10A810008F225E21FFF762FF012038BDA090FF1F4D
:10A8200010B4047F4160022CC26002D010BC01F061
:10A83000D7BB836810BC184790E80C00F0B41C68C4
:10A8400059682568164F174E29432160164D174940
:10A850001760D66015611160417A154A5C180A319B
:10A8600094F8244053F8215002EBC40149680D606C
:10A87000017A5C1803EB8101247ECD6902EBC401EF
:10A8800049680D60817A581803EB810390F8300015
:10A89000596B02EBC002F0BC53681960704700BFEF
:10A8A00001401F00011000380110007800001F80D7
:10A8B00040370100704700BFF0B50C1EBDF81460B2
:10A8C00034DBB0F906701919B942C4BF3B1B1BB287
:10A8D000002BA6461CDD002A1146B8BFD11D02F090
:10A8E0000705CC10826A012007FB04E1A840012E75
:10A8F0000A44C0B21ED00CD3022E09D1013B12FA79
:10A9000083F3013A12F8011F41409A421170F9D1C4
:10A91000F0BDC043013B12FA83F3C0B2013A12F812
:10A92000011F014093421170F9D1F0BD23441BB2C5
:10A930000024C6E7013B12FA83F3013A12F8011F23
:10A9400001439A421170F9D1F0BD00BFF8B50D1E58
:10A950000EDB14461F46064601F03AFBA84207DD0F
:10A96000002C05DB304601F037FBA04201DCF8BDCE
:10A97000F8BD304601F02AFB022853D003284BD003
:10A98000012806D16540F3886C406540013B5D1BA2
:10A990002DB2012F03D02AD3022F14D0F8BD002CE2
:10A9A0002246B6F90630B06AB8BFE21D42F3CF02C4
:10A9B00002FB035504F00704435D012101FA04F48E
:10A9C0001C434455F8BD002C2246B6F90630B06A47
:10A9D000B8BFE21D42F3CF0202FB035504F00704A7
:10A9E000435D012101FA04F45C404455F8BD002C9C
:10A9F0002246B6F90630B06AB8BFE21D42F3CF0274
:10AA000002FB035504F00704435D012101FA04F43D
:10AA100023EA04044455F8BD3389013B591B2546FC
:10AA20000CB2B6E7F18832890139013A4D1B141B8B
:10AA30002DB224B2ADE700BF2DE9F041079E9DF98C
:10AA40001880089D04461F4600F0C0FF0D4B0E48BD
:10AA50000E4984F83380FF22002F08BF1F4684F878
:10AA60002F20002384F8302084F8312084F832200D
:10AA70002060A665E565676261652362A362204682
:10AA8000BDE8F081A090FF1F982C01000110013853
:10AA900010B50446806A034B236008B105F078FBCB
:10AAA000204610BD982C0100F8B5436ADBB190F840
:10AAB0002C200125AA4083F83B2083F85E5083F8C0
:10AAC0005D500446406A03680E461B6800219847A3
:10AAD000606A036831461B6898472946606ABDE88A
:10AAE000F840FFF7E5BBC26BC56C1368046A23EA44
:10AAF000050313604CB122684FF00043D3625163E9
:10AB0000D36A002BFCDA936BF8BD836B466B082588
:10AB1000802410E03768426C3A4332601F68826CD0
:10AB20003A431A601A68876C013D22EA07024FEA2D
:10AB300054041A6007D02142ECD13268476C22EAF3
:10AB400007023260EAE7F8BD70B50446406A0D4678
:10AB500000282BD0A16DFFF749FA002D20460CBF2D
:10AB6000A621A721FFF7A0FF606A20B1E16DBDE833
:10AB70007040FFF73BBA216C226D0868236A0243DC
:10AB80000A6093B1DA7A82B1D00703D5224A996973
:10AB90001160DA7A910703D5204AD9691160DA7A0F
:10ABA000520702D51E4A1B6A136070BD236A002B30
:10ABB0002BD0D97A626DE1B172B6D97ACE0706D5BB
:10ABC0001848D9680668314099610160D97A8807C8
:10ABD00006D51548196906683140D9610160D97AEE
:10ABE0004E0705D511485969066831401962016060
:10ABF00062B61B68D968914207D00D4818600D49AC
:10AC0000DA6042F0804018611960226C216D13688F
:10AC100023EA01031360A0E700E100E004E100E0A3
:10AC200008E100E080E100E084E100E088E100E08C
:10AC300001403F0000003F80436A2DE9F041054696
:10AC40000E469046002B3ED090F82C100124A140D7
:10AC500083F83B1083F85E4083F85D40406A0368E8
:10AC600000211B6808F1FF379847FFB2B8F1000FC9
:10AC700023D03744A046013E686A16F8011F0368D6
:10AC80001B6898470134B742E4B216D0202CF3D1A8
:10AC90000121686AFFF70CFB95F82C206B6A5200C3
:10ACA00083F83B2083F85E8083F85D80686A0368E0
:10ACB00000211B6898470124DEE7686A0121BDE88E
:10ACC000F041FFF7F5BAC26BC16C136823EA0103C8
:10ACD00006EB080413604FF00048A6420ED02B6A22
:10ACE00016F801EB63B11A68C2F82C80C2F834E0A0
:10ACF000D36A002BFCDAA642936BF0D1BDE8F08159
:10AD0000AB6BD5F834C008208021DCF800206F6CD4
:10AD10001EEA010F14BF3A43BA43CCF800201A6868
:10AD2000AF6C3A431A601A68AF6C013822EA070226
:10AD30004FEA51011A60E8D1CFE700BF70B5044671
:10AD4000406A0D46002828D0A16DFFF74FF9204634
:10AD50002946FFF7A9FE606A20B1E16DBDE87040A9
:10AD6000FFF744B9216C226D0868236A02430A6028
:10AD700093B1DA7A82B1D00703D5234A9969116079
:10AD8000DA7A910703D5214AD9691160DA7A520734
:10AD900002D51F4A1B6A136070BD236A002B2BD09B
:10ADA000D97A626DE1B172B6D97ACE0706D5194863
:10ADB000D9680668314099610160D97A880706D55B
:10ADC0001548196906683140D9610160D97A4E0782
:10ADD00005D512485969066831401962016062B6AA
:10ADE0001B68D968914207D00D4818600D49DA6098
:10ADF00042F0804018611960226C216D136823EACB
:10AE000001031360A3E700BF00E100E004E100E0FC
:10AE100008E100E080E100E084E100E088E100E09A
:10AE200001403F0000003F802DE9F041044686B01C
:10AE3000806A9DF830801E460F461546B4F90830EA
:10AE4000002800F04281DA1D48BF03F10E02B4F978
:10AE50000630D21003FB02F2002105F0BDFCB4F96C
:10AE60000820202A00F39280B4F90610A34B012099
:10AE7000203A733902EBD27201EBD1714FF0200E00
:10AE8000029073208DE8014042F34F0241F34F01DD
:10AE9000204600F051FE606A84F82D70002800F012
:10AEA0004D81002D40F08A80B4F90830202B14BF6A
:10AEB0003D253C2584F82C50B8F1000F40F08580EA
:10AEC00006B394F93300002818DBC0B2012102F068
:10AED000E7F8012194F8330002F0CEF8012002F0E7
:10AEE00007F9002194F8330002F0C6F80A2002F0B6
:10AEF000FFF8012194F8330002F0BEF8606A0028E0
:10AF000000F08280A16DFFF771F804227C49204691
:10AF1000FFF792FE217A0139C9B22046FFF7C4FD3E
:10AF2000784904222046FFF787FE94F92D30012B43
:10AF300014BF142110212046FFF7B6FD04227249E8
:10AF40002046FFF779FEB4F90630802B00F092809E
:10AF5000602B00F0A680D9212046FFF7A5FD94F9CB
:10AF60002D30012B14BFF12122212046FFF79CFD3B
:10AF7000204606226549FFF75FFE606A50B3E16D27
:10AF8000FFF734F8012006B0BDE8F081B4F90610EF
:10AF90005F4B0120403A52394FF0400E029002EBD5
:10AFA000D272522001EBD1718DE8014042F34F0281
:10AFB00041F34F01204600F0BFFD6CE76DB284F80D
:10AFC0002C50B8F1000F3FF47BAFFEF7C5FF002E09
:10AFD00094D076E7216C226D0868236A02430A60E8
:10AFE00073B1DA7A62B1D00703D54A4A9969116020
:10AFF000DA7A91077CD4520702D5474A1B6A13605C
:10B00000012006B0BDE8F081236A002B2BD0D97A4D
:10B01000626DE1B172B6D97ACF0706D53F48D968DB
:10B020000568294099610160D97A8E0706D53C48A8
:10B03000196905682940D9610160D97A4D0705D59C
:10B0400038485969056829401962016062B61B6871
:10B05000D968914207D0344818603449DA6042F028
:10B06000804018611960226C216D136823EA010386
:10B0700013604AE7B4F90830202B00F08680402B9B
:10B080007FF469AF2A4920460322FFF7D5FD94F9E2
:10B090002D30012B14BFCF219F212046FFF704FD47
:10B0A00059E7B4F90830102B7FF455AF21492046F9
:10B0B0000322FFF7C1FD94F92D30012B14BFAF21FE
:10B0C00010212046FFF7F0FC45E7DA1D48BF03F1E9
:10B0D0000E02B4F90630D21003FB02F210460592BC
:10B0E00005F04EF8A06200283FF44DAF059AB3E694
:10B0F000114AD9691160DA7A7DE700BFF02C0100AE
:10B10000D02E0100D42E0100D82E0100DC2E01002B
:10B11000E42E010000E100E008E100E080E100E051
:10B1200084E100E088E100E001403F0000003F8052
:10B13000EC2C0100A431010004E100E0012194F8AD
:10B140003100244F01F0ACFF94F83200012101F0EE
:10B15000A7FF94F9312094F9323057F83220E26396
:10B1600057F83330206A23640125E56425651A68A1
:10B170002A431A6078B1B8F1000F3FF428AFFFF707
:10B180005BFB002E3FF4BAAE9BE604221249204638
:10B19000FFF752FDDFE6294694F82F0001F080FF0B
:10B1A000294694F8300001F07BFF94F92F2094F9A0
:10B1B000303057F83220626357F833306564A56445
:10B1C0001A68A36322F001021A60002E3FF496AEC3
:10B1D00077E600BF40370100E82C0100B0F90820F5
:10B1E000D31D48BF02F10E03B0F90620806ADB10C0
:10B1F00002FB03F2002105F0EFBA00BFF0B5002911
:10B20000BDF814502EDBB0F90660B1422ADA002AEC
:10B2100059DBB0F9087014461C44BC42C4BFBB1AC9
:10B220001BB2002B1EDDD2B2D408D0F828E016FBEA
:10B23000041112F00702DBB20EEB010421D0C2F1BF
:10B240000807FAB2374F9342BF5C0CD2C3EB020C33
:10B25000FF2646FA0CF6012D07EA06073FD005D374
:10B26000022D36D0F0BD012D39D030D21EF801604C
:10B2700026EA07070EF801709342F3D3B0F90610DF
:10B280000C449A1AD2B2072A10D9022D36D0002DBA
:10B2900014BFFF26002613462670083BB0F906109F
:10B2A000DBB2072B0C44F7D802F00702002AD9D0F2
:10B2B0001D4B012D9B5C1DD017D3022DD2D12278BE
:10B2C00053402370F0BD13441BB20022A1E7022DAE
:10B2D00025D11EF8016077400EF80170CCE71EF80A
:10B2E000016037430EF80170C6E7227822EA0303B3
:10B2F0002370F0BD227813432370F0BD11462378EC
:10B30000DB4323700839B0F90630C9B207291C4461
:10B31000F5D812F00702A5D0034B9B5CCFE734446D
:10B32000AFE700BF882C0100782C010070B4C47D09
:10B33000BDF80C50022C18D0032C1FD0012C0BD0C0
:10B34000002A03DBB0F90840944201DC70BC70476E
:10B35000039570BCFFF7B0BAC4880395013CA41AEA
:10B360000A4621B270BCFFF749BF0689C488013E76
:10B37000641AB21AE41A12B221B2E1E70489039501
:10B38000E41A641A114622B270BCFFF737BF00BF3F
:10B3900070B4C57DBDF80C60022D1AD0032D12D0FB
:10B3A000012D03D0039670BCFFF728BFC488E41AB0
:10B3B000A41A0A4621B2002A03DBB0F908409442DD
:10B3C00013DC70BC70470489013C641A114622B238
:10B3D000F1E7C48805890396013CAD1AED1A621A9B
:10B3E00011B22AB270BCFFF709BF039670BCFFF719
:10B3F00063BA00BF2DE9F8430446406A002863D0D1
:10B40000A16DFEF7F3FD052274492046FFF714FCF9
:10B41000A1790139C9B22046FFF746FBB4F90820EB
:10B42000E588A66AD31D48BF02F10E03DB10626AED
:10B4300015FB03F51FFA85F8002A7BD094F82C3011
:10B440000125AB4082F83B3082F85E5082F85D50B7
:10B45000606A036840211B6808F1FF379847BFB254
:10B46000B8F1000F23D03744A846013E606A16F8B1
:10B47000011F03681B6898470135B742EDB216D02B
:10B48000202DF3D10121606AFEF712FF94F82C20E1
:10B49000636A520083F83B2083F85E8083F85D8006
:10B4A000606A036840211B6898470125DEE7012197
:10B4B000606AFEF7FDFE606A002800F08D80E16D95
:10B4C000BDE8F843FEF792BD236A002B2BD0D97A52
:10B4D000626DE1B172B6D97ACE0706D54048D96817
:10B4E0000568294099610160D97A8D0706D53D48E4
:10B4F000196905682940D9610160D97A480705D5DD
:10B5000039485969056829401962016062B61B68AB
:10B51000D968914207D0354818603549DA6042F061
:10B52000804018611960226C216D136823EA0103C1
:10B53000136068E7E26BE36C1168276A0B4306EB64
:10B54000080913604FF0004E4E450DD016F801CBA0
:10B550002FB33A68C2F82CE0C2F834C0D36A002B8B
:10B56000FCDA4E45936BF1D1226C236D11680B43CD
:10B57000136097B1FB7A83B1D90703D51D4BBA6924
:10B580001A60FB7A9A0703D51B4BFA691A60FB7A9B
:10B590005B0702D5194B3A6A1A60BDE8F883A36BC2
:10B5A000D4F8348008208021D8F80020656C1CEA8B
:10B5B000010F14BF2A43AA43C8F800201A68A56CDB
:10B5C0002A431A601A68A56C013822EA05024FEA7C
:10B5D00051011A60E8D1B7E7276AC5E7802C01005E
:10B5E00080E100E084E100E088E100E001403F000C
:10B5F00000003F8000E100E004E100E008E100E03D
:10B600002DE9F04F85B09946BDF93870BDF83CA0E2
:10B61000BB1AC1EB090B002BB8BF5B42BBF1000F9B
:10B62000B8BFCBF1000B5B450D4616460093804634
:10B6300048DC4D453A4633464CDC194613460A462B
:10B64000C5EB09019B1A89B2002B0CB2B8BF5B4253
:10B6500004EBD474BE42ACBF4FF0FF3201224D4523
:10B66000039102924FEA640429DC9BB201930DE03E
:10B67000D8F80070BF69B847019BE41AA3B21CB2A6
:10B680000135002C2DB211DBA94518DB009B5B4571
:10B690002A46534631464046EADCD8F80020534655
:10B6A0009769294632464046B847E5E7029A16446C
:10B6B000039AA94502EB030436B224B2E6DA05B0D8
:10B6C000BDE8F08F4A462B46B94635464D451746EC
:10B6D0001E46B2DD304629463E464D46074689465F
:10B6E000AEE700BF10B404682469A44610BC6047EC
:10B6F00030B40468BDF808500295A46BA44630BC71
:10B70000604700BF30B40468BDF808500295E46B90
:10B71000A44630BC604700BF70B40468BDF90C603B
:10B72000BDF8105003960495246CA44670BC604785
:10B73000704700BF10B582B0B0F90C2001910168CC
:10B74000009200220C6CB0F90A301146A04702B0FA
:10B7500010BD00BF704700BF01F003010129C17592
:10B7600006D0032904D0C2880389428183817047AF
:10B770000289C38842818381704700BF2DE9F0416F
:10B780000568134E6F6986B0B7420446BDF8308035
:10B7900010D1013B13441BB20093CDF804800B463B
:10B7A000AD6A2046A8472368DB6AB3420AD106B0D7
:10B7B000BDE8F081059304920391B84703A9256879
:10B7C0000EC9E6E7204606B0BDE8F041184700BFC5
:10B7D00031B700002DE9F0410568124E6F6986B05F
:10B7E000B7420446BDF830800FD1013BCDF804804C
:10B7F0000B4400921BB2AD6A2046A8472368DB6A5F
:10B80000B3420AD106B0BDE8F081059304920391DA
:10B81000B84703A925680EC9E7E7204606B0BDE88A
:10B82000F041184731B700002DE9F04F0568DFF807
:10B8300058B06F6985B05F450646BDF93890BDF8D0
:10B840003CA00C46904615D11F19BC420CDACDF82D
:10B8500000A0214601342D6A4B464246304624B2B0
:10B86000A847BC423568F2DBEB6A5B4507D105B0FF
:10B87000BDE8F08F0393B8473568039BE4E7304693
:10B8800005B0BDE8F04F184731B700002DE9F0438F
:10B8900087B099420546BDF93840BDF83C6025D0D7
:10B8A000A24212D00768DFF88080D7F81490C14513
:10B8B00032D18DE850002846BC6AA0472B68DB6A6D
:10B8C000434524D107B0BDE8F083994202DD084624
:10B8D0001946034628680E96C46B01335B1A1BB2E7
:10B8E0002846A44607B0BDE8F0436047A24202DD07
:10B8F000134622461C4628680E96631C846B9B1ACE
:10B900001BB22846A44607B0BDE8F043604728466E
:10B9100007B0BDE8F0431847059304920391C84768
:10B9200003A92F680EC9C4E731B700002DE9F04F15
:10B93000D0F800E0DFF89090DEF814B083B0CB458B
:10B940000446BDF93080BDF834A00D4617461E46AA
:10B9500031D1CDF800A0DEF824B0294633463A466E
:10B960002046D8472368CDF800A008F1FF323A44BA
:10B97000D3F824B0294612B233462046D84723686C
:10B98000CDF800A02946D3F820B03A4643462046D9
:10B99000D8472068CDF800A0711E29444346056AA7
:10B9A00009B23A462046A8472368DB6A4B4506D1D0
:10B9B00003B0BDE8F08FD847D4F800E0C9E72046CF
:10B9C00003B0BDE8F04F184731B70000F0B40024D1
:10B9D00001264FF6FF75094F07600471C475C481D5
:10B9E00004824476C4618675067685824582C1806C
:10B9F000028141818281F0BC704700BFB0310100FB
:10BA00002DE9F04F85B00668BDF84450BDF9388087
:10BA1000CDF8008004460195D6F848B00392BDF9F0
:10BA20003C60BDF9407089469A46D8472368019525
:10BA3000009742465146D3F8488020463346C047D7
:10BA40002068039B0E930F95856C4B463A46314612
:10BA50002046AC4605B0BDE8F04F60472DE9F04FF9
:10BA600087B01746BDF9404000912546E91D059372
:10BA700044BF2B4603F10E010268BDF848605369CC
:10BA80000294C91003912B49BDF9444001968B42A1
:10BA9000824645D1002C3CDD029B3C445E1EB6B282
:10BAA0004FF0000923B2049301364D46029B002B50
:10BAB00028DD059B002403EB090806E0EDB22B0608
:10BAC00004F1010411D4A6421CD0A1B211F0070F59
:10BAD00023B24FEA4505F1D1002BB8BF0733DB1085
:10BAE000013418F803502B06EDD5009BD2F818B09E
:10BAF00019443A4609B2019B5046D847A642DAF8A3
:10BB00000020E2D1039B01379944049B3FB2BB4222
:10BB1000CCD1D36A074A934206D107B0BDE8F08F73
:10BB20009847DAF80020B5E7504607B0BDE8F04F77
:10BB3000184700BF31B7000070B4BDF90C60BDF903
:10BB40001050BDF8144003960495059470BCFFF79F
:10BB500085BF00BF2DE9F04F93B090460591C169B4
:10BB60001090BDF870000790BDF874909DF878A013
:10BB70000493002900F0CD800A7A0AC98946049905
:10BB80008A1AD2B203EBC203BAF1010FDA780B9230
:10BB900093F905201E8893F802B00F9293F906409E
:10BBA00079D913B2099323B20C93109B1A68A94B4D
:10BBB0001193194653698B4240F0A6800B9B002BD2
:10BBC00055D01FFA88F300210D93C8462344DDF8B1
:10BBD000409006910E930F460C46BBF1000F3FD0EC
:10BBE000BDF818100C9B03971FFA8AF0CB1813FBB3
:10BBF00000F304900E9801440D98034409B21BB25F
:10BC00000A910893002505E00135EBB264009B45DD
:10BC1000E4B222D9039B2B44590703D1731C18F8B3
:10BC200006409EB22306EFD5099BBDF81000E91827
:10BC300011FB00F10598BAF1010F0FFA8AF30144E4
:10BC40001CD0079801900093D26909B21746484664
:10BC5000089AB847D9F80020D6E7039F5F44FFB29F
:10BC6000069B0B9901330693DBB29942B5D8D36A90
:10BC7000119A934243D113B0BDE8F08F0F9B19186E
:10BC800093690A9A29441F4609B2079B4846B84758
:10BC9000D9F80020B8E700230C93099385E70A9AA6
:10BCA0000D9B0132013B52B213F0FF030A920D9338
:10BCB0006FD1DDF81890079BDDF83C80DDF820A0FF
:10BCC0004B4517D0BAF1010F00F0C8800B9A109DB8
:10BCD000CDF804900BEB8B014FEACB030A440093A1
:10BCE0001146DEF81C405346424609B22846A0479A
:10BCF000D5F800E0DEF82C30119A9342BBD01098B2
:10BD000013B0BDE8F04F1847109D284698472A68A1
:10BD100054E7109A0598B2F90A308342ABDDB2F9C4
:10BD20000C304345A7DD062313FB0A03002BA2DDDD
:10BD300008EBCA03002B9EDD537E2BB9049BAF2B6F
:10BD400002D90133DBB20493109BD3F800E0414BDE
:10BD500011931A46DEF81430934240F08E801FFA99
:10BD600088F30E9308339BB2BDF814200593052386
:10BD70000D9300230A93CDF83C800FFA8AF3DDF887
:10BD80004080CDF818900B921FFA8AFBCDF820A0C6
:10BD900099460A9ABDF810000B9C0E9D0523194682
:10BDA00011FB00232C481146C75C039702FB0B4292
:10BDB00014FA81F312B21BB209920C932C462E4650
:10BDC0001CE0089B0999012B2AB24B4640462DD016
:10BDD000079F0197CDF80090DEF81CA0D047D8F857
:10BDE00000E0039B5B0801340393059BA4B25D4410
:10BDF0005E44A342ADB2B6B23FF451AF039BD80745
:10BE0000DFD4079B069A9342EBD0089B012B16D0F8
:10BE1000069B0193CDF80090DEF81CA009994B46D3
:10BE200032B24046D047D8F800E0DAE7DEF818A092
:10BE3000079B0C9922B2D047D8F800E0D1E7DEF892
:10BE400018A00C991346404622B2D047D8F800E01B
:10BE5000C7E700BF31B70000003201000B99109D09
:10BE6000CDF800900531DEF8204009B242460823A3
:10BE70002846A047D5F800E03CE7109C20469847AC
:10BE8000D4F800E06BE700BFF0B5C36985B00446A5
:10BE90002BB30A2968D00D294AD01A7A914247D388
:10BEA000587A884244D35D688A1A05EBC205AA789D
:10BEB000002A50D0E87800284DD0207E00283AD0C3
:10BEC00095F905E0B4F90E00A67DB4F90A70724444
:10BED00006FB0202BA4262DCB4F9102030E00A2903
:10BEE00056D00D2924D0027E002A4BD0B0F90E0086
:10BEF000A57DB4F90A60062212FB0502B2423EDDBE
:10BF0000228AE38102EBC50212B218462282A78A76
:10BF1000668A02950B468DE8C00001462046FFF771
:10BF200019FEA37DE28903EB430302EB4303E381A4
:10BF3000012005B0F0BDA67DB4F90E00B4F91020C3
:10BF4000B4F814E0678A02960B468DE880400146FB
:10BF50002046FFF7FFFD2979E389A27D012001FB3F
:10BF60000233E38105B0F0BD0022C2819A7A817D5F
:10BF7000038A01FB02330382012005B0F0BDB4F94E
:10BF80001020C4E7857DB4F91020B0F90E00BEE79B
:10BF9000028A817DC38102EBC1030382C8E70020CE
:10BFA000E0819B7A228A03FB062212B22282C7E733
:10BFB000C1810282704700BF002908BF012181753D
:10BFC000704700BF81824182704700BFC07D7047CB
:10BFD000B0F90A00704700BFB0F90C00704700BF0D
:10BFE00010B4EFF3108272B6437F33B9017F012999
:10BFF00007D003290FD00123437702B962B610BCE2
:10C000007047124C2168A1B1114943610B688361EB
:10C0100008605861EFE70F4C216881B10E49436118
:10C020000B688361086058610C4B4FF080511960B8
:10C03000E1E7074B4161816120601860DBE7064B57
:10C040004161816120601860EEE700BF309FFF1FF3
:10C050002C9FFF1F209FFF1F249FFF1F04ED00E068
:10C0600070B5EFF3108272B60C4C206880B10C4EA4
:10C0700000254369236073B19D6102B962B64577BB
:10C0800083689847EFF3108272B620680028F0D1D9
:10C0900002B962B670BD3360EFE700BF209FFF1F9B
:10C0A000249FFF1FFFF7DCBF184A30B41468002C30
:10C0B00027D0036821688B420ED2CB1A00218460FE
:10C0C000C1602360E06010600223037530BC7047DC
:10C0D00011688B42144608D3A2685B1A0360002AD9
:10C0E000F6D18260C460A060EEE7D268C26084606E
:10C0F000E060C568CB1A0222A8602360027530BCDC
:10C1000070478460C4601060DEE700BF289FFF1F97
:10C11000F8B5224E34682CB32368002B3AD1204F57
:10C120001D4604E03468ECB12368002B32D1A368CB
:10C1300003B1DD6020693360036825751B68BB426D
:10C1400021D1037F4560022BC46020D0FFF748FF58
:10C150006368002BE6D023602046FFF7A5FF346814
:10C16000002CE1D1EFF3108372B60E4A0021106863
:10C17000116003B962B628B18468FFF795FF2046C5
:10C180000028F9D1F8BD224600219847E0E78368EE
:10C190009847DDE7013B2360E4E700BF289FFF1FCE
:10C1A00021A80000389FFF1F024A13680133136063
:10C1B000FFF7AEBF449FFF1F704700BF0368F0B496
:10C1C000FBB1002501249D60DC601B4C1A601C44FF
:10C1D000241104F144056A11032692009E60174F52
:10C1E0000679174B47F8241002F1604202F56142CC
:10C1F00005F01F05012000FA05F5E6541560F0BCB6
:10C200007047104C236843F40003236000BF0E4BBB
:10C210000E4DA4F58734A4F59E7401261E602346B6
:10C2200004609C68002CD0D01033AB420360F8D17E
:10C23000002303601846E2E7008FFCBF7891FF1FE0
:10C2400044E400E03C80044000700340407103403F
:10C250000168A9B10B4BF0B40B441B110A4E0B4FF4
:10C260000B4D46F8237003F1440202F01F04012332
:10C270005211A340002445F822308C600460F0BCC9
:10C28000704700BF008FFCBF7891FF1FB9C100004D
:10C2900080E100E0024A034B012111601B6818474E
:10C2A0000C7103407891FF1F024A034B012111607A
:10C2B0005B6818471C7103407891FF1F024A034BCB
:10C2C000012111609B6818472C7103407891FF1F72
:10C2D000024A034B01211160DB6818473C7103409F
:10C2E0007891FF1FF8B50E4671B17AB10746144632
:10C2F00000253B6816F8011B1B6838469847013C2F
:10C300000544F6D12846F8BD0846F8BD1046F8BDEC
:10C3100000B5064A036812885B6883B001A9ADF8CE
:10C3200004200222984703B05DF804FB00370100A7
:10C33000F0B507468BB0002A33D0012A08BF0A2285
:10C3400051B3212400E0F4B2B1FBF2F502FB151168
:10C35000C8B2092900F1300198BFC8B20AA988BF44
:10C360003730214488BFC0B201F8240C661E29462C
:10C37000002DE8D133B1013CE4B20AAB23442D22B5
:10C3800003F8242C3B6801AA11195B683846C4F1F4
:10C39000220298470BB0F0BD30228DF825202124D1
:10C3A000E8E70368C9B21B6898470BB0F0BD00BF4F
:10C3B0000029BABF49422D2300230A22FFF7B8BF44
:10C3C000374A384913681B06FCD40B6813F0800306
:10C3D000F8D172B634490A78002A5FD0334A34481B
:10C3E000F0B4344C176806682568D4680C303E44B5
:10C3F000143200681268304F35442C442044024403
:10C40000C2F34E022D4E2E482E4D2F4C42F40042C8
:10C410003A60376806682D682C4A24680C303E4420
:10C42000006812682A4F35442C4420440244C2F369
:10C430004E02284E2848294D294C42F400423A60C9
:10C44000376806682D68274A24680C303E44006827
:10C450001268254F35442C4420440244C2F34E0256
:10C46000224E2348234D244C42F400423A60376860
:10C4700006682D68214A24680C303E440068126822
:10C4800035442C4420440244C2F34E021C4842F47A
:10C49000004202600B7062B6F0BC704762B6704733
:10C4A00024B0034024B00B403D9FFF1F38B0034031
:10C4B0003CB0034040B003402CB0034058B00340B0
:10C4C0005CB0034060B0034064B003406CB0034014
:10C4D00030B0034038B00B403CB00B4040B00B4094
:10C4E00044B00B404CB00B402CB00B4058B00B404C
:10C4F0005CB00B4060B00B4064B00B406CB00B40C4
:10C5000030B00B4030B42948294A2A4B2A4D6024C8
:10C51000E121047011701B78284C082B30D00A2BB5
:10C520002748284937D00C2B0CBF35223D22122337
:10C530002A60236002600B60234B24491B78244A45
:10C54000BBB101230B601360224B23491B78234AA4
:10C55000012B26D9042B0FD9082B1ED9102B94BFE1
:10C56000862387230B6013601D4B01221A7030BC99
:10C5700070470B601360E7E784230B601360F3E7F9
:10C5800000F58E200F490830012213232A60236012
:10C5900002600B60D0E73922F7E785230B60136058
:10C5A000E2E780230B601360DEE700BF0040074036
:10C5B000014007408891FF1F08B003400CB00340C2
:10C5C00008B00B400CB00B40409FFF1F20B0034051
:10C5D00020B00B408991FF1F24B0034024B00B40D2
:10C5E0003D9FFF1F0C2830B417D91023984228BF55
:10C5F00018461C46104A114D1178181A8C422870A2
:10C6000018D00F4913700B7823B10E490E4A00233E
:10C610000B60136030BCFFF775BF0A2802D90C23EA
:10C620001C46E7E7082802D90A231C46E2E708234C
:10C630001C46DFE730BC70478891FF1F3C9FFF1FFF
:10C640003D9FFF1F24B0034024B00B4028282FD863
:10C65000334B2DE9F0411E5CFF2E2BD0314B1B7864
:10C66000002B2AD132062CD472B62F4D2F4C2F46D8
:10C67000012326602B7062B672B623681B060CD4A9
:10C680003B781BB9F4E72B78002BF1D062B602F0AF
:10C690009BF972B623681806F5D5254B1B68002256
:10C6A0002A7062B6234A107843FA00F0BDE8F081A0
:10C6B000002070470020BDE8F081FFF781FE3206C0
:10C6C000D2D572B61C4DDFF87C801C4C06F04007BA
:10C6D000FFB206F03F06D8F80030DFB123F01003B8
:10C6E000C8F8003001232660134A2B7062B672B678
:10C6F000236819060CD413781BB9ECE72B78002BB0
:10C70000E9D062B602F060F972B623681B06F5D56F
:10C710000B4BC3E743F01003C8F80030E2E700BF5B
:10C72000043701003D9FFF1F3F9FFF1F00B00340E4
:10C7300010B003403C9FFF1F3E9FFF1F00B00B4007
:10C7400010B00B400CB00B400A4A0B49136843F47D
:10C75000805313600B7843B9084BC0221A70084B02
:10C7600080F30C0000B218807047044B80221A70CE
:10C77000F5E700BF2C800440409FFF1F21C00C4004
:10C7800000C00C40F0B51B4B1B4E596818689A68E6
:10C79000DB6885B06C460FC4337899071DD5174AFE
:10C7A000174C1378174913F0700318BF1370164A0B
:10C7B000164B8027177000263320032226706D4603
:10C7C00008701A7072B6043C45F001052046A8476F
:10C7D00062B6237813F0700309D10D4B064901E0CE
:10C7E000013B02D00A78D207FAD505B0F0BD23701C
:10C7F00005B0F0BD303701000100024000000240EA
:10C80000040002400B000240070002400A00024000
:10C81000410D0300B0F5006F0AD210B5094B1B782B
:10C82000DB07044606D504F1A0500078C0B210BD65
:10C8300000207047FFF7A6FF04F1A0500078C0B2B7
:10C8400010BD00BF01000240B0F5006F17D238B52F
:10C850000F4B1B78DA070D46044611D504F1A050A2
:10C860000378AB420AD00B4A137813F0700318BF59
:10C870001370074A05701378DB07FCD538BD704785
:10C88000FFF780FF04F1A0500378AB42EBD1F5E74E
:10C89000010002400000024008B5F3F705FFF5F77C
:10C8A0000FFE02F091F8FAE7844641EA000313F024
:10C8B00003036DD1403A41D351F8043B40F8043BA7
:10C8C00051F8043B40F8043B51F8043B40F8043B6A
:10C8D00051F8043B40F8043B51F8043B40F8043B5A
:10C8E00051F8043B40F8043B51F8043B40F8043B4A
:10C8F00051F8043B40F8043B51F8043B40F8043B3A
:10C9000051F8043B40F8043B51F8043B40F8043B29
:10C9100051F8043B40F8043B51F8043B40F8043B19
:10C9200051F8043B40F8043B51F8043B40F8043B09
:10C9300051F8043B40F8043B403ABDD2303211D3A9
:10C9400051F8043B40F8043B51F8043B40F8043BE9
:10C9500051F8043B40F8043B51F8043B40F8043BD9
:10C96000103AEDD20C3205D351F8043B40F8043BA9
:10C97000043AF9D2043208D0D2071CBF11F8013BA7
:10C9800000F8013B01D30B8803806046704700BF6D
:10C99000082A13D38B078DD010F003038AD0C3F17C
:10C9A0000403D21ADB071CBF11F8013B00F8013B5E
:10C9B00080D331F8023B20F8023B7BE7043AD9D31D
:10C9C000013A11F8013B00F8013BF9D20B780370F2
:10C9D0004B7843708B7883706046704708B5104C75
:10C9E00008E0236859050DD423681A050FD423687D
:10C9F000DB0411D423685803F3D500F08DFE2368BF
:10CA00005905F1D502F044F823681A05EFD502F074
:10CA1000D5F82368DB04EDD500F0F0FCEAE700BFB1
:10CA20003480044008B5FFF7D9FF00BF014B102246
:10CA30001A80704700200540704700BF094908B5BB
:10CA40000B6830B16A461844A2F58052904202D277
:10CA50000860184608BD03F065FB0C2303604FF027
:10CA6000FF3008BD8C91FF1FFEE700BFEFF313807E
:10CA700070B9EFF310836BB9EFF305825AB94FF435
:10CA80008070EFF311832BB1984228BF184670478E
:10CA90004FF0FF3070470F2A01D81846F1E7014BDD
:10CAA000D05CEEE7F0E300E0F0B44D1E2E4600242B
:10CAB00000E00134B0FBF2F302FB1300092800F19F
:10CAC00030078ABF3730F8B2C0B206F8010F1846F7
:10CAD000002BEED10A1953704CB1107815F8016F84
:10CAE00028700133E01A834202F80169F5DB084639
:10CAF000F0BC7047704700BF10B40F4B53F83020A4
:10CB000092F880422CB1012369B182F8803010BCC8
:10CB1000704703EBC0035B681A6841B922F0020258
:10CB20001A6010BC704782F8003110BC704742F0A8
:10CB300003021A6010BC7047403701001C4A02EB28
:10CB4000C00301295B6811D004291BD052F83000C2
:10CB5000002280F8802229B1022920D0032922D086
:10CB60001A6070474FF480721A60704752F83000B4
:10CB70004FF4A27280F880121A601A6822F0200224
:10CB80001A60704752F830104FF4A272012081F8F9
:10CB900080021A601A6842F020021A60704740F260
:10CBA00003121A6070474FF481721A60704700BF19
:10CBB00040370100212848D8F8B5042A44D8DFE8D6
:10CBC00002F0484B4E0345004FF410262B4B03EB6D
:10CBD000C0030D465C68216811F4E06148D0284B21
:10CBE000284A2949C3F89C2104F140422748C3F848
:10CBF000A411A2F59221264FC3F8A0017C29254853
:10CC0000C3F8A871C3F8AC012CD9A2F594237C2BEE
:10CC10002AD9A2F596237C2B28D9A2F598237C2B20
:10CC200029D9A2F59A227C2A27D81B4872B62368F4
:10CC300023F4702343F08072C4F38401164323600D
:10CC400040F82150266062B6F8BD70474FF4302698
:10CC5000BCE74FF40026B9E74FF44026B6E74FF49F
:10CC60002026B3E70D48E1E70D48DFE70D48DDE793
:10CC7000FFF764FFB3E70C48D8E7F8BD4037010081
:10CC80000082FF1FF188FF1F9988FF1FC588FF1FC3
:10CC90006D88FF1F4188FF1F6892FF1F9091FF1F43
:10CCA000C891FF1F1892FF1F4892FF1F1A4B03EBFA
:10CCB000C00010B4426802F14043A3F592217C29E0
:10CCC00023D9A3F594217C290DD9A3F596217C299C
:10CCD0001FD9A3F598217C2919D9A3F59A237C2B78
:10CCE00011D80E4C00E00E4C72B613680D4823F0BC
:10CCF0008773C2F3840123F4803343F0807313609D
:10CD000044F8210062B610BC7047074CECE7074CB2
:10CD1000EAE7074CE8E700BF403701006892FF1FD1
:10CD2000C891FF1FF5CA00009091FF1F4892FF1F96
:10CD30001892FF1F30B4054B054D064C0022102100
:10CD40001A602A602060196030BC704714D003401C
:10CD500004D0034000D00340282838B52ED0002945
:10CD600004464FDD5F4B1B78012505FA03F28A422A
:10CD700002D8212837D938BD0338C2B2012A3AD99E
:10CD8000202C4AD0192C48D0574A126802FB0112B5
:10CD900022FA03F31D2800F29B80DFE800F0928B5B
:10CDA000847D9999766F99999999999999999968A2
:10CDB000615A53994C99999999999945494B1B787E
:10CDC0000B2B08D90C2B1CBF0C3B19410846BDE8A6
:10CDD0003840FFF7B9BCC3F10C0399400846BDE8E1
:10CDE0003840FFF7B1BC2946FFF786FE2946BDE86B
:10CDF0003840FFF7A3BE3D4A126802FB011222FA37
:10CE000003F3C7E72128B6D80021FFF775FE2046B7
:10CE10000121BDE83840FFF791BE354A126802FB98
:10CE2000011222FA03F3B5E73249334A0B604FF49B
:10CE30005173136038BD3149314A0B604FF451735F
:10CE4000136038BD2F49304A0B6040F244431360F1
:10CE500038BD2E492E4A0B6040F24443136038BD62
:10CE60002C492D4A0B6040F24443136038BD2B49D6
:10CE70002B4A0B6040F24443136038BD29492A4ACB
:10CE80000B6040F24443136038BD2849284A0B60C8
:10CE900040F24443136038BD2649274A0B6040F2F4
:10CEA0004443136038BD2549254A0B6040F2444392
:10CEB000136038BD2349244A0B604FF4517313604B
:10CEC00038BD2249224A0B604FF45173136038BDBC
:10CED000212C3FF650AF7F29D4BF002101212046ED
:10CEE00093E700BF7092FF1F088003400890034043
:10CEF00008800B4010800B4048A0044018800B4075
:10CF00004CA004401880034008B004401080034047
:10CF100004B004404080034018C0044038800340FF
:10CF200014C004402880034010B004402080034017
:10CF30000CB004403080034010C0044048800340DF
:10CF40001CC00440189003403490044010900340EB
:10CF50003090044038B1102828BF1020044AC3B2D2
:10CF6000107813707047024A0123107813707047CD
:10CF70007092FF1F2DE9F8430E4680463249334D2B
:10CF8000304603F055F847F6122300281ABF1D4615
:10CF90004FF002094FF00109002425FA04F002F0D5
:10CFA00051FE4FF05E51074602F0A4FE01463046A6
:10CFB00003F052F830B90134072CEED1E80902F041
:10CFC00041FE07463146384602F048FF4FF07C519B
:10CFD00002F086FD03F07AF84FF6FF729042A8F156
:10CFE000030328BF1046012B29D9B8F1170F17D812
:10CFF000174B23FA08F303F0010383F0010223B96E
:10D00000B8F1190F0FD0BDE8F883124B124D134938
:10D010001A6044EAC9042A6008601C60BDE8F8830D
:10D02000B8F1200FECD10E4B0E4D0F49002244EA0F
:10D03000C9041A602A6008601C60BDE8F8830B4BC5
:10D040000B4D0C49F2E700BF001BB740006CDC023F
:10D050006006F00000800340048003400880034025
:10D0600000800B4004800B4008800B400090034080
:10D070000490034008900340212801D8FFF73CBDED
:10D08000704700BF212806D8044B53F8303093F87E
:10D090000002C0B270470020704700BF4037010057
:10D0A000212801D8FFF74ABD704700BF72B60C496E
:10D0B0000C4B0D4A1B680868126862B6520102D513
:10D0C000322B88BF01300949C3F5BB334FF47A7264
:10D0D000FF33A1FB031302FB00F000EB931070473A
:10D0E000449FFF1F18E000E004ED00E0ABAAAAAAED
:10D0F0002DE9F843054672B6204F214B214A1B68A3
:10D100003C68126862B6520102D5322B88BF0134E6
:10D1100095B3C3F5BB331C4EDFF86490DFF8648031
:10D12000FF334FF47A72A6FB031302FB04F404EB03
:10D13000931472B6D9F800103A68D8F800E062B6D5
:10D14000C1F5BB33FF33A6FB03031EF0806FC4EBB6
:10D1500093134FF47A7002D0322988BF013200FB5A
:10D160000233B3F57A7F04D3013D05D004F57A7418
:10D17000DFE701F029FCDCE7BDE8F883449FFF1FEF
:10D1800018E000E004ED00E0ABAAAAAAF8B52D4B28
:10D190002D49DFF8D0E0DFF8D0C02C4E2C4D2D4CBF
:10D1A0002D4A2E4F4FF4000018604FF08070186029
:10D1B0004FF0007018604FF0806018604FF0006012
:10D1C00018600020086028234BF6FF71CCF800108F
:10D1D000CEF80030336013602B6023603B60B36295
:10D1E0009362092245F8242CC4F8D80F05F57F6511
:10D1F000C7F8D41F07F5FF2707F5FA67C6F8F83F09
:10D200002B6006F5FF26C4F8D42F05F5FD2504F59F
:10D21000FF24386006F2F4761148316005F5FF65A9
:10D2200004F5FD642B6023600260FFF76BF91920A1
:10D23000FFF75EFF00F0B6FF40F21310BDE8F840C4
:10D24000FFF756BF08E100E004800340148003406C
:10D25000248003402C8003401C8003403480034022
:10D2600000800B400C800340088003402DE9F84FFC
:10D27000214B1B6807460BB101221A70DFF888901A
:10D280001E4D99F80040DFF884801D4E0134272C94
:10D290008ABF4FF0000A5FFA84FA5446AB462B78F7
:10D2A000A34216D1FFF7E2FB40281FDC33791B06AF
:10D2B000F5D59BF800300133272B86BF002213469B
:10D2C000DAB218F80330DBB2F3712A702B78A3427C
:10D2D000E8D00C490A4BFFB208F804700120AC22D8
:10D2E000087089F800A0DA70BDE8F88FFF28D6DD55
:10D2F00001F06AFBD3E700BFBC9FFF1FB99FFF1F70
:10D3000000C00640B89FFF1FC09FFF1F509FFF1F18
:10D310001C4BDFF894C01A681B49F0B542F48052E8
:10D320001A4D1A60DFF884E0194F1A4E1A4C002388
:10D330008CF800304FF451722B701F2840F21335D7
:10D340008EF800303B70337025600A6012D81946A1
:10D350000124124A124D11701248547000212C27DA
:10D36000402693724FF4003491701174D7702E7070
:10D370000460F0BDC0F34431C0F3471400F01F0354
:10D38000E7E700BF348004400CC004404D9FFF1FFE
:10D39000B99FFF1FB89FFF1F08C0044000C0064090
:10D3A00031E400E004E100E04C9FFF1FC09FFF1F3D
:10D3B000034B1B68DB0401D5FFF758BF704700BF64
:10D3C0003480044010B5044C237823B101F0FCFAFA
:10D3D0002378002BFAD110BDB89FFF1F054A064BDA
:10D3E00010781B78C0B2DBB2984238BF4030C01A08
:10D3F000704700BF4C9FFF1F4D9FFF1F30B42B4B4A
:10D400001A7994061FD52A48DA7903782949013315
:10D410003F2B0978C8BF00238B42D2B203D0264CE1
:10D42000D9B2E2540170254A116861B1244A1278D8
:10D43000D2B2934236BFC2F140029B1A9B18272BEF
:10D44000C4BF01230B70194AD378DBB2180611D47C
:10D450005A060DD5154B1B795B0609D5194B1A4990
:10D460001B6800220A7003B11A70104B2C22DA706C
:10D4700030BC704711790906EAD5144910480C7878
:10D480000178C9B28C420DD04A1C272A84BF0021E2
:10D490000A460F4D054C98BFD1B2AA5CD2B2E271D8
:10D4A0000170D5E76C21D170D2E700BF00C0064003
:10D4B0004C9FFF1F4D9FFF1F789FFF1F489FFF1F1F
:10D4C000B99FFF1FBC9FFF1FB89FFF1FC09FFF1F7B
:10D4D000509FFF1F21282FD8184B195CFF292BD0F4
:10D4E000174B184ADFF870C003EBC000F0B5436873
:10D4F000DFF868E0144F154D154E00241C60DEF86F
:10D500000030012043F020038840CEF80030146042
:10D510004FF4A07338602E60C2F800C0013BFDD10B
:10D5200013689B05FCD42023013BFDD1094B09B2B4
:10D5300033F8110080B2F0BD002070475038010070
:10D54000403701000050044008500440045004409B
:10D55000000002030051044080014A00388004406A
:10D56000431E032B14D872B60A4951F8230068B140
:10D5700070B4094C058834F81320466841F82360DC
:10D58000521B24F8132062B670BC704762B6704715
:10D59000002070471CA0FF1F60A2FF1F0138032856
:10D5A0000BD872B6074B53F8203043B100205B68AC
:10D5B0000130002BFBD162B670470020704718463F
:10D5C000F9E700BF70A0FF1F30B472B62B4A137882
:10D5D0001D0706D52A4B196A002936D0996A0029F9
:10D5E00041D053781C0706D5254B196C00293ED035
:10D5F000996C002939D09378190705D5204B196EFD
:10D60000002936D0996E89B1D3781B0707D51C4BFA
:10D61000D3F880207AB3D3F8882011213AB162B6CA
:10D62000184B00221A7030BC00F04ABE0D21154C78
:10D63000154D227843F8315003EBC1030830013A0D
:10D640005860227062B630BC704704220D4C0F4DFA
:10D65000217843F8325003EBC20308304A1E586069
:10D66000227062B6EFE70521E1E70921DFE7082232
:10D67000ECE70C22EAE71022E8E700BF743801006B
:10D680000080FF1F99A0FF1FC800400088004000D5
:10D69000431E032B1DD81B4A400140F0100030B43C
:10D6A000104472B6184CE25C032A1BD8DFE802F083
:10D6B0000212151703220D88E25410F0080F14BF50
:10D6C000C823882343EA054308310360416062B6FA
:10D6D00030BC704708300222EDE70522EBE7083046
:10D6E0000422E8E7094A52F8230038B1084A52F800
:10D6F0002300416042F8231062B6E9E742F82310A4
:10D70000034AF7E70080FF1FA8A0FF1F70A0FF1FBC
:10D7100080A0FF1F00BE70472DE9F04FDFF818B35F
:10D72000DFF818A387B044E0AD4F4FEA930807EB4A
:10D73000C809013ED9F8042003F00803F6B2A2F1AB
:10D74000080003F0FF04002B40F0018157F8383047
:10D750001B0C99B222F8081C002B00F0EF80A14BA3
:10D7600022F8064C42F8044C53F82620002A00F018
:10D77000CF819D4D55F8263058609C4C45F82600C9
:10D7800034F81630194424F8161000F079FD0028FA
:10D7900000F0C281964A974B19F0080F00F108007B
:10D7A00018BF1346C9F8040047F8383008238BF82F
:10D7B00000309BF80040E4B265071CD58E4B1B7807
:10D7C000B3B18E490A7802F0FF0322B1013BDBB20C
:10D7D0000B7003B900BE8A490A7802F0FF032AB130
:10D7E000013BDBB20B70002B00F0688100F066FE9D
:10D7F00004238BF8003004F0080303F0FF02002B31
:10D8000000F0C9809AF80030DBB21E098CD19A086A
:10D81000DFF8CC9159F8321009EBC200C1F3830153
:10D82000013940680C2900F28580DFE801F07A7A3E
:10D830008383838383834683838307000168714DD9
:10D840004068714F714E6860296088B240F2816112
:10D850000024674B49F832304FF0010E88423C609B
:10D86000C9F81040C9F8184086F800E05C4A00F298
:10D87000E780B0F5D06F80F01B82B0F5817F00F0BB
:10D88000D98100F26981802800F02A82822840F044
:10D89000D781A98801F07F01042900F2D1815C4879
:10D8A0005C4A890008441470547001788C0740F178
:10D8B000608382F800E0022173E1534F3A682AB393
:10D8C000554B524E554819883478057840298E4674
:10D8D00045F0020828BF4FF0400E002C84F00104F0
:10D8E0003470CEEB01010CBF8824C82409EBC806B4
:10D8F00089B285F0010544EA0E447260198049F846
:10D90000384072440570002965D03A603D4B1A8852
:10D91000B2F5A06F0ED100219A785970404B1A7061
:10D9200008E038493F4C0D68A54200F09880304926
:10D9300049F832103C4A0123137037E72C4A2D4B2B
:10D9400019F0080F18BF134647F838302EE700F0DB
:10D95000B7FC364A364952F82630002B00F0E380F7
:10D9600058688C5D42F8260003F10802C9F80420CB
:10D97000032C05D8DFE804F02C02292602228A5560
:10D980001A8819F0080F0CBF8823C82343EA024302
:10D9900047F838300AE7E00700F19380210600F1EC
:10D9A000D180A20706D5234A234913780220DBB28F
:10D9B00013700870E30602D51F4B10221A7007B0CF
:10D9C000BDE8F08F04228A55DAE705228A55D7E7A9
:10D9D00003228A55D4E7BEF1400F18BF002294E716
:10D9E0000080FF1F1CA0FF1FC89FFF1F60A2FF1F1A
:10D9F000C800400088004000A4A0FF1F2DA0FF1F0A
:10DA000018A1FF1F90A0FF1FC49FFF1F2CA0FF1F86
:10DA1000C02007409CA0FF1FD89FFF1F98A0FF1F9A
:10DA200098200740210900039420074070A0FF1FA1
:10DA3000A8A0FF1F882007408020074090200740B3
:10DA4000B0F5106F00F07C8140F2A38040F6211207
:10DA5000904240F07B82A54A012313706AE74C682C
:10DA6000A3498C427FF463AF0178A9297FF45FAFAB
:10DA7000417845297FF45BAF8178C2297FF457AFA5
:10DA8000C1786B297FF453AF9A489B4E0178347864
:10DA900081F00105002C41F0020105700CBF8820C7
:10DAA000C82084F0010449F8310009EBC101934812
:10DAB0003470002505244D60047038E700F064FFE1
:10DAC00094E68F4B89488B491A614FF0020E80F81B
:10DAD00000E08C4F0A708C49196099608B4E8C4D18
:10DAE0008C4C9A610D213970FF213170DFF84CE2C6
:10DAF00029702270884D894A8EF800109F270124D2
:10DB000006F8047C5D600470DA6007B0BDE8F08F51
:10DB100043F82600824D30E6824A47F838001378F1
:10DB20000133137042E68B5D032B00F2BA8001A231
:10DB300052F823F0ADD70000ADD700008DDB000018
:10DB400087DB00006F49724B80220D2008701A702D
:10DB5000A2077FF52FAF26E740F20232904240F055
:10DB6000ED81AA8802F07F02042A69D86D88002D11
:10DB700066D16449CDF804E0920011440A7842F07D
:10DB800002020A70C1E101238B550FE600238B5579
:10DB90000CE6B0F5086F53D16349644A09781170F7
:10DBA0007146ED888D4280F0E88252480478402D1D
:10DBB000AE4644F0020C28BF4FF0400E02EB0E03BD
:10DBC00009EBCC01029301234A604FEA0E48CEEBE9
:10DBD000050101930025C82242EA080384F00102EE
:10DBE00049F83C3035700270DFF814C1424BDFF861
:10DBF000048149BBBEF1400F7FF42DAF42F0020C0F
:10DC000009EBCC03029ADFF8F8E05A608DBB0D04F3
:10DC100045F088059DF804304EF83C500A443370B6
:10DC20000470134640297FF416AF0021404A3B6040
:10DC3000118010E7AA8802F07F02042A40F28B814B
:10DC4000304A0F23137006E74029D7D942F0020269
:10DC50000CEBC200029E4660BDB19DF804503548F1
:10DC60001D703346403988F8004040334CF832008C
:10DC7000DCE79DF8043033700D04029B047045F01E
:10DC8000C8050B444EF83C50CCE79DF804501D707D
:10DC9000029B1D4888F80040403940334CF8320060
:10DCA000C4E719F0080F0CBF022303238B557DE551
:10DCB00021494A68002AC3D06C88B5F804E003E023
:10DCC0000C314A68002ABBD00B88A342F8D14B889C
:10DCD0007345F5D1240A032C0CBF1178098960E73C
:10DCE000124A0221147054705BE700BF9420074071
:10DCF0000100040098A0FF1F2CA0FF1F2DA0FF1FF4
:10DD00000080FF1FC0200740880040008820074097
:10DD10008020074098200740DC9FFF1F30A0FF1F96
:10DD2000C89FFF1F99A0FF1FA4A0FF1F9CA0FF1F5B
:10DD3000D89FFF1FC8004000783801008C200740A2
:10DD4000B248116AAC7804700C0600F19881D9F8D9
:10DD50002820AF49100600F1DB81D9F83020AC490A
:10DD6000120600F1D081D9F83820A949130600F134
:10DD7000C581D9F84020A649150600F1BA81D9F825
:10DD80004820A349140600F1AF81D9F85020A049DA
:10DD9000100600F1A481D9F858209D49120600F11F
:10DDA0009981D9F860209A49130600F18E81D9F83B
:10DDB00068209749150600F18381D9F870209449AD
:10DDC000140600F17881D9F878209149100600F105
:10DDD0006D81D9F880208E49120600F16181D9F851
:10DDE00088208B49130600F15581D9F89020884985
:10DDF000150600F14981D9F898208549140600F1EB
:10DE0000FF808448844A854901908548854D864C29
:10DE1000049700230596029580460F4616461D4638
:10DE20000394306828B1446800F04AFA2046002C78
:10DE3000F9D100233360029B38681A46002342F868
:10DE4000253028B1446800F03BFA2046002CF9D177
:10DE500000223A60019A98F800301146002241F8F9
:10DE6000042B039A0191023B4FF0000122F8151098
:10DE7000032B07D8DFE803F05D025D024FF00103DA
:10DE800088F800300135042D06F1040607F1040777
:10DE900008F10108C5D1654C654D2278654B049F9A
:10DEA000059E0021100729701A7000F192806249C6
:10DEB00062780A700021C9F83010C9F838101107CB
:10DEC000DFF84C816ED4A2785C49DFF844810A7097
:10DED00000211207C9F85010C9F858104BD4E27845
:10DEE00057494B4C0A7013074FF00001C9F87010E6
:10DEF000C9F8781000F1AE8033780193002283F0E6
:10DF00000105C9F89020C9F898200021029188469F
:10DF10008E460A464B48047844F0020C09EBCC03C9
:10DF20000393019B002B039B5A600CBF8822C822DD
:10DF300052E64FF0000388F80030A3E7B0F5A06F79
:10DF40007FF47EAE012300250193DEE740F6212217
:10DF50009042F7D074E66D88002D7FF471AE3A4997
:10DF6000CDF804E0920011440A7822F002020A700F
:10DF7000CBE7022115E600F083F9002800F0EB80E2
:10DF80000830324AC8F86400C8F8602000F078F918
:10DF9000002800F0DA8008302D4AC9F86C00C9F872
:10DFA00068209CE700F06CF9002800F0E080083061
:10DFB000264AC8F84400C8F8402000F061F900285B
:10DFC00000F0CF800830224AC9F84C00C9F8482038
:10DFD00079E700F055F9002800F0A58008301B4AC9
:10DFE000C9F82400C9F8202000F04AF9002800F000
:10DFF00094800830164AC9F82C00C9F8282056E742
:10E00000D1F89C00083800F05BF9FAE6A4A0FF1FE5
:10E010000080FF1F80A0FF1F1CA0FF1F70A0FF1F1C
:10E02000A8A0FF1FC89FFF1F60A2FF1F7438010038
:10E0300099A0FF1FC4200740C8200740CC200740FC
:10E04000D020074098A0FF1FC02007408800400054
:10E05000C800400000F014F9002870D008304F4A82
:10E06000C4F88400C4F8802000F00AF9002860D0C9
:10E0700008304B4AC9F88C00C9F888203CE7506A40
:10E08000083800F01DF962E6D1F89400083800F075
:10E0900017F9B0E6D1F88C00083800F011F9A4E6C1
:10E0A000D1F88400083800F00BF998E6C86F0838FA
:10E0B00000F006F98DE6486F083800F001F982E6B5
:10E0C000C86E083800F0FCF877E6486E083800F0B3
:10E0D000F7F86CE6C86D083800F0F2F861E6486DB4
:10E0E000083800F0EDF856E6C86C083800F0E8F89B
:10E0F0004BE6486C083800F0E3F840E6C86B083897
:10E1000000F0DEF835E6486B083800F0D9F82AE66A
:10E11000C86A083800F0D4F81FE62A78C9F8280041
:10E1200001322A70C3E62A78C9F8200001322A7029
:10E130005AE72A78C9F8880001322A70DCE62A7882
:10E14000C4F8800001322A708EE72A78C9F8680086
:10E1500001322A70C3E62A78C8F8600001322A70BA
:10E1600014E72A78C9F8480001322A70ABE62A7809
:10E17000C8F8400001322A701FE740298E4628BFA8
:10E180004FF0400E02EB0E0302930123CEEB010190
:10E190004FEA0E4800250193BCE600BF880040000E
:10E1A000C8004000F8B500F08FFD294B29482A4CE3
:10E1B0002A4F2B4DDFF8BCC0DFF8BCE0294E00220F
:10E1C0001A605A609A60DA601A615A619A61DA617B
:10E1D0001A625A629A62DA621A635A639A63DA635B
:10E1E0001A645A649A64DA641A655A659A65DA653B
:10E1F0001A665A669A66DA661A675A679A67DA671B
:10E20000C3F880200168C3F8842041F480210160B4
:10E21000C3F307212170C3F30740134938701B0E65
:10E220002B70FF238CF80030104D8EF80030104812
:10E230000B700123337084F8642070264FF400744F
:10E24000102207F82C3C2E70046081F8F820F8BDED
:10E250000080FF1F348004409C200740B02007400E
:10E26000B4200740942007401020074049E400E014
:10E2700008E100E08020074088200740704700BF89
:10E2800072B60D480268B2FA82F30F2B10DC4FF021
:10E290000041D94022EA0102026062B6074803EB5E
:10E2A000C303DB00C2180021C15010465160704703
:10E2B00062B60020704700BF7492FF1FBC83FF1F2F
:10E2C0000D4B0E4AC31AA2FB03231B090F2B0CD8BC
:10E2D0000B4A127852B972B60A484FF000410268F0
:10E2E00021FA03F31A43026062B67047064A1278B5
:10E2F000002AF0D0FFF768B9BC83FF1F398EE338DE
:10E3000099A0FF1F7492FF1FA4A0FF1F38B50E4BEA
:10E310000E4C1B68218805468BB1B1F5917F05D263
:10E320000B4A4B1C55549BB2238038BD0022084831
:10E3300098470021064A55540123238038BDB1F582
:10E34000917FEDD338BD00BFD0A0FF1F6AA2FF1F91
:10E3500070A2FF1F2DE9F843214E224F316801239F
:10E3600080463B70B1B1204D4B8801EB83020133F5
:10E3700000240F2BC2F808802C7004D84B80002397
:10E380003B70BDE8F88340230B800320FFF780F942
:10E390003460F4E7DFF8549099F80030002BF0D0A7
:10E3A000114D45F6215408E0013C12D02B7883B979
:10E3B00000F00AFB99F800307BB10320FFF7EEF87C
:10E3C0000528F1D8FFF75CFF014630600028EBD04C
:10E3D000CAE701232B70BDE8F883BDE8F88300BFCE
:10E3E000ECA0FF1FC0A0FF1FF0A0FF1FA4A0FF1FF5
:10E3F0001201F8B5D5B2A1B3012943D04378044640
:10E4000000781B0643EA004040F4704045F00406E3
:10E410008F1E3043FFF79EFF022F04F1020314D931
:10E42000053414F8023C14F8032C14F8010C1B04F6
:10E4300043EA0223334343EA0060033FFFF78AFFC6
:10E44000022F234604F10304EBD8022F23D0012F1F
:10E450000DD045F4774040F00500BDE8F840FFF7E7
:10E4600079BF14482843BDE8F840FFF773BF187818
:10E4700045F4770545F0060545EA0020BDE8F8407B
:10E48000FFF768BF03780C4845EA03452843BDE819
:10E49000F840FFF75FBF1A78587845F0774545F0A8
:10E4A000070545EA022545EA0040BDE8F840FFF7C8
:10E4B00051BF00BF06F0F70007F000F738B5084B72
:10E4C0001C7824B9074D296809B14B8803B938BDB8
:10E4D0009B000B800320FFF7DBF82C6038BD00BFEA
:10E4E000C0A0FF1FECA0FF1F2DE9F041AD4E336827
:10E4F0000746002B00F092801D885A88910803EB94
:10E5000081010432AA428C6842D25A8004F00F067C
:10E510004FEA1428A449A6F1080208F00F00C4F33A
:10E520000313062A00F101050B701AD9B31E012B43
:10E530005FFA88F04ED9052E48D0042E00F0A48151
:10E54000731F022B7FD90F2E0ED1F72842D8F02847
:10E5500002D0964B1B883BB1FFF7D8FE0020BDE8E8
:10E56000F08127B1BD4202D00020BDE8F081082E25
:10E57000C4F3033300F08780092E11D00A2E40F037
:10E5800094800A2BF0D18A4B8A4A1B68A02181E033
:10E590001846FFF795FE0420FEF7E2FF3060B5E76E
:10E5A000092BE1D1270E00F07B81834B814A1B6848
:10E5B0009021C4F307461170EDB2FCB2002B00F0BD
:10E5C0009D80224631462846984797E0F02843D957
:10E5D000F72841D0F1380E28C6D801A353F820F00F
:10E5E00097E700007BE7000069E7000069E50000AD
:10E5F00069E500005BE7000069E500003BE800001A
:10E6000069E5000005E800001FE8000043E700009E
:10E6100069E500002BE700000FE70000674B1B785F
:10E62000002BA1D00420FEF79BFF0346306000289A
:10E630009AD00588002D7FF460AFFFF741FE35606A
:10E640002846BDE8F081FFF761FEC4F30740FFF7FD
:10E650005DFE072E02D1200EFFF758FE534B584A9D
:10E66000198858481468584D524A017000270E0AFC
:10E67000F0201F802E7010700CB301225348A04769
:10E680000120BDE8F081082B7FF46EAF504B494A62
:10E690001B688021C4F307461170EDB2240E6BB3E2
:10E6A000284622463146984728E00B2E11D10B2BE5
:10E6B0007FF45AAF474B3F4A1B68B021EAE7464B0D
:10E6C0001B68002B00F0FB80404898470120BDE804
:10E6D000F0810C2E40F000810C2B7FF445AF3F4BB6
:10E6E000344A1B68C0211170EDB2C4F30746002BF9
:10E6F00000F0C88028463146240E98473849314AF0
:10E70000314B0D7016701C700120BDE8F081354B47
:10E710001B68002B00F0D6809847C4F30746254BB2
:10E72000EDB2240E83F80080E8E72F4B1B68002B26
:10E73000F2D12E4B1B68A3B1FE209847C4F30746C5
:10E74000EDE72B4B1B68002BE6D1284B1B6843B130
:10E75000FC209847C4F30746E1E7264B1B68002BD3
:10E76000DAD1C4F30746DAE7234B1B68C4F3074644
:10E77000002BD4D030469847D1E7204B1A68002AA6
:10E78000EFD0260C630C06F07F0003F47E53184391
:10E79000F6B29047C3E71A4B1B68C4F30746002B39
:10E7A000E8D1BCE7F8A0FF1F6EA2FF1F6AA2FF1FFF
:10E7B000D4A0FF1F68A2FF1F08A1FF1FA4A0FF1F76
:10E7C000D0A0FF1F6CA2FF1F6DA2FF1F70A2FF1F32
:10E7D00000A1FF1F04A1FF1FE8A0FF1FC4A0FF1F8F
:10E7E0006FA2FF1FB0A0FF1FB4A0FF1FB8A0FF1FA4
:10E7F000F4A0FF1FE4A0FF1FFCA0FF1FCCA0FF1F81
:10E80000E0A0FF1F3F4B1B68002B85D13E4B1B68D0
:10E81000002BA6D0FA209847C4F307467FE73B4B6E
:10E820001B68002B7FF478AF374B1B68002B98D008
:10E83000FB209847C4F3074671E7354B1B68002B54
:10E840007FF46AAF304B1B68002B8AD0F8209847C2
:10E85000C4F3074663E70E2B7FF486AE2D4A2E4B9A
:10E860001268E0211970002A47D0260C610C06F0CE
:10E870007F0301F47E511943EDB2A1F50051284602
:10E880009047F6B2240E39E7FFF740FDC4F3074086
:10E89000FFF73CFD200EFFF739FD0020BDE8F081B9
:10E8A0001E4B1D4A1B6880211170EDB2C4F3074650
:10E8B00083B1314628463A4698473C461EE7012038
:10E8C000BDE8F081104B1B68002B3FF44AAFFF20DE
:10E8D000984746E71C4611E70D2EBCD10D2B7FF45F
:10E8E00043AE0F4B0C4A1B68D0211170EDB2C4F33C
:10E8F0000746002B7FF4FEAEC4E7C4F30746EDB233
:10E90000240EFBE6DCA0FF1FB8A0FF1FBCA0FF1F6A
:10E91000ACA0FF1FC8A0FF1F68A2FF1F00A1FF1F20
:10E92000D8A0FF1F38B5164D2868E0B1018844888B
:10E93000A14213DD03191B7A83B104F10803C21845
:10E940000C1B002302E012F8011F21B10133A34286
:10E95000F9D1204638BD1C46204638BDFFF7B0FC33
:10E960000020286038BD074B1B780BB9002038BD4C
:10E970000220FEF7F5FD28600028D7D1F6E700BF9A
:10E9800014A1FF1FA4A0FF1F0D4B1B78BBB910B52E
:10E990000C4C216803F0FF024B883F2B07DC073348
:10E9A0000B4401F1470003F8012F8342FBD14023C0
:10E9B0000B800120FEF76CFE0023236010BD704722
:10E9C0000CA1FF1F10A1FF1F38B5224C237803B103
:10E9D00038BD01232370FFF7A5FF70BB00F048F896
:10E9E00040BB00F0DBF810BBFEF7F8FCE0B90023F9
:10E9F0002370EFF30583002BEAD1EFF3108172B699
:10EA0000154B1868E0B1154C2278CAB945691D60EC
:10EA100001232370C5B1AA6101B962B6002545770B
:10EA2000836898472570D3E700F020F8DFE700F00F
:10EA30001BF8D9E700F016F8D3E7FFF71FFCCDE786
:10EA40000029C5D162B638BD054B1D600029E5D14E
:10EA5000E3E700BF19A1FF1F309FFF1F349FFF1F77
:10EA60002C9FFF1F704700BF704700BF704700BF5B
:10EA7000054A064B10781B78C0B2DBB2984238BF0B
:10EA80004030C01A704700BF20A1FF1F21A1FF1F07
:10EA9000F0B4384B1A7912F0300F2CD072B6997D41
:10EAA00001F0FF0200293DD062B6334F3349387878
:10EAB0000D78334E1C46C0B2EDB2431C402BE179B9
:10EAC00028BF0023AB4202F1FF32C9B21CBFF15490
:10EAD000184612F0FF02F0D12A4B1B68C2B23A70FE
:10EAE0004BB1A84236BFC5F14005401B401927284D
:10EAF000C4BF01221A701F49CA78D2B2150616D4B3
:10EB000052060DD51B4B1B795B0609D51E4B1F49C1
:10EB10001B6800220A7003B11A70164B3C22DA708F
:10EB2000F0BC70474022D9795A7462B6E3E70B799A
:10EB30001C06E5D5164B174E1C783378E4B2DBB2D1
:10EB40009C420ED0144D01E0A3420AD00133402B69
:10EB500028BF00230879E85CC0B2C871087D072887
:10EB6000F2D9DBB2034933700B79180644BF7C231A
:10EB7000CB70C5E700A0064020A1FF1F21A1FF1F09
:10EB800064A1FF1F1CA1FF1FA8A1FF1FA4A1FF1FBD
:10EB9000ACA1FF1FA5A1FF1F24A1FF1F054A064B23
:10EBA00010781B78C0B2DBB2984238BF4030C01A30
:10EBB000704700BF20A2FF1FB5A1FF1FF0B4384B64
:10EBC0001A7912F0300F2CD072B6997D01F0FF0245
:10EBD00000293DD062B6334F334938780D78334E33
:10EBE0001C46C0B2EDB2431C402BE17928BF002384
:10EBF000AB4202F1FF32C9B21CBFF154184612F009
:10EC0000FF02F0D12A4B1B68C2B23A704BB1A84246
:10EC100036BFC5F14005401B40192728C4BF01225B
:10EC20001A701F49CA78D2B2150616D452060DD5ED
:10EC30001B4B1B795B0609D51E4B1F491B68002225
:10EC40000A7003B11A70164B3C22DA70F0BC7047A0
:10EC50004022D9795A7462B6E3E70B791C06E5D5F0
:10EC6000164B174E1C783378E4B2DBB29C420ED0C0
:10EC7000144D01E0A3420AD00133282B28BF002302
:10EC80000879E85CC0B2C871087D0728F2D9DBB208
:10EC9000034933700B79180644BF7C23CB70C5E75A
:10ECA00000B0064020A2FF1FB5A1FF1FE0A1FF1F7B
:10ECB000B0A1FF1F24A2FF1FB4A1FF1F28A2FF1FA6
:10ECC00021A2FF1FB8A1FF1F70B584B072B6194B07
:10ECD000194D1A48702241260F2480211A702E7077
:10ECE0001A460470197013781B06FCD5144B18686B
:10ECF00062B6144B144C984298BF00EB800001A9F7
:10ED000098BF40000A22FDF7CFFE01A9204600234C
:10ED100011F8012B01333AB10A2B20F8022FF7D159
:10ED20001623237004B070BD5B00DBB2237004B007
:10ED300070BD00BF00000240070002400600024014
:10ED4000080002407F9698004093FF1FFFFFFFFFDF
:10ED50002DE9F043DFF8EC808BB006460F4600F05B
:10ED600073F898F90030013304460D4637D0304629
:10ED7000394600F0DFF9002831D02BA3D3E9002376
:10ED80003046394600F026FE814668BB28A3D3E909
:10ED900000233046394600F0FFFD00B398F90030FB
:10EDA000254ACDF82090042400200021022BCDE933
:10EDB0000467CDE9026700940192CDE906012CD0E9
:10EDC000684600F0BDF940B3089B1BB101F0AAF9F9
:10EDD000089B0360DDE906010BB0BDE8F083204627
:10EDE00029460BB0BDE8F083134A98F90030019230
:10EDF00003210022CDE90467CDE902670091089262
:10EE00002BB90E4B4FF06042CDE90623D8E70C49F1
:10EE10000020022BCDE90601D2D101F083F9222393
:10EE20000360D1E7AFF30080EF39FAFE422E86404F
:10EE300051302DD5104987C0E4380100FFFFEF475E
:10EE40000000F07F5693FF1F2DE9F04FB04F21F0E7
:10EE50000042BA4283B00C464FEAD17605460DD93E
:10EE6000AC4FBA4225D9C1F31303034340F0EF80FE
:10EE70000EB10020014603B0BDE8F08FA64B9A42C8
:10EE800000F2CC80A54B9A4200F2DE808AA3D3E93F
:10EE9000002300F05DF90022A14B00F09BFD00284B
:10EEA00000F005812846214600229D4B00F050F9D4
:10EEB000E1E783A3D3E9002300F08CFD002840F0B4
:10EEC000CB802846214680A3D3E9002300F064FDCF
:10EED0000028CED1934B284603EBC60821467CA3DD
:10EEE000D3E9002300F0E6FAD8E9002300F030F976
:10EEF00000F07AFD804600F077FA77A3D3E900238B
:10EF000006460F4600F0D6FA02460B462846214632
:10EF100000F01CF972A3D3E90023CDE900013046CB
:10EF2000394600F0C7FA82468B4652465B46DDE919
:10EF3000000100F00BF905460C462A4623462846F8
:10EF4000214600F0B7FA68A3D3E9002306460F462E
:10EF500000F0B0FA66A3D3E9002300F0F7F83246D8
:10EF60003B4600F0A7FA64A3D3E9002300F0F0F8D1
:10EF700032463B4600F09EFA61A3D3E9002300F03D
:10EF8000E5F832463B4600F095FA5FA3D3E900234B
:10EF900000F0DEF832463B4600F08CFA02460B46A3
:10EFA0002846214600F0D2F806460F46284621465C
:10EFB00032463B46B8F1000F56D000F07BFA32469D
:10EFC00004460D463B4600204FF0804100F0BEF85D
:10EFD00002460B462046294600F096FB02460B46A9
:10EFE0005046594600F0B2F8DDE9002300F0AEF8D3
:10EFF0000B4602464A49002000F0A8F86FF47F73E0
:10F0000098454FDA08F57A7801EB085100224FF065
:10F01000B87300F04FFA03B0BDE8F08F424B9A424C
:10F020003FF658AF414BF4002344D3E9002300F0EE
:10F030008DF83F4BC6F101081C44CDE90001D4E92D
:10F0400000ABC6EB080870E74FF0000875E7024612
:10F050000B4600F07DF80EE717A3D3E90023104616
:10F06000194600F027FA06E700F024FA002280464D
:10F0700089464FF080433046394600F067F8024633
:10F080000B464046494600F03FFB2A46234600F027
:10F090005DF802460B460020214900F057F803B006
:10F0A000BDE8F08F01EB085103B0BDE8F08F80465A
:10F0B00043E700BFAFF300809C7500883CE4377ED7
:10F0C000EF39FAFE422E864051302DD5104987C0C7
:10F0D000FE822B654715F73F0000E0FE422EE63F1B
:10F0E000763C7935EF39EA3DD0A4BE726937663E89
:10F0F000F16BD2C541BDBB3E2CDE25AF6A56113F38
:10F1000093BDBE166CC1663F3E5555555555C53F1E
:10F11000412E8640FFFFEF7F422ED63FFFFF2F3E5E
:10F120000000F03FE8380100B1A2F03F08390100CB
:10F13000F838010041F0004101F58010C00F704720
:10F140000020704781F0004102E000BF83F00043DF
:10F1500030B54FEA41044FEA430594EA050F08BF72
:10F1600090EA020F1FBF54EA000C55EA020C7FEA36
:10F17000645C7FEA655C00F0E2804FEA5454D4EBB3
:10F180005555B8BF6D420CDD2C4480EA020281EA7D
:10F19000030382EA000083EA010180EA020281EAB5
:10F1A0000303362D88BF30BD11F0004F4FEA013107
:10F1B0004FF4801C4CEA113102D0404261EB410116
:10F1C00013F0004F4FEA03334CEA133302D052429C
:10F1D00063EB430394EA050F00F0A780A4F1010458
:10F1E000D5F1200E0DDB02FA0EFC22FA05F2801892
:10F1F00041F1000103FA0EF2801843FA05F3594178
:10F200000EE0A5F120050EF1200E012A03FA0EFCF6
:10F2100028BF4CF0020C43FA05F3C01851EBE37120
:10F2200001F0004507D54FF0000EDCF1000C7EEB3D
:10F2300000006EEB0101B1F5801F1BD3B1F5001F7B
:10F240000CD349085FEA30004FEA3C0C04F101049A
:10F250004FEA445212F5800F80F09A80BCF1004FC3
:10F2600008BF5FEA500C50F1000041EB045141EA45
:10F27000050130BD5FEA4C0C404141EB010111F446
:10F28000801FA4F10104E9D191F0000F04BF0146F1
:10F290000020B1FA81F308BF2033A3F10B03B3F1CF
:10F2A00020020CDA0C3208DD02F1140CC2F10C025F
:10F2B00001FA0CF021FA02F10CE002F11402D8BFBD
:10F2C000C2F1200C01FA02F120FA0CFCDCBF41EA89
:10F2D0000C019040E41AA2BF01EB0451294330BD58
:10F2E0006FEA04041F3C1CDA0C340EDC04F1140435
:10F2F000C4F1200220FA04F001FA02F340EA03000C
:10F3000021FA04F345EA030130BDC4F10C04C4F151
:10F31000200220FA02F001FA04F340EA0300294631
:10F3200030BD21FA04F0294630BD94F0000F83F47B
:10F33000801306BF81F480110134013D4EE77FEA5E
:10F34000645C18BF7FEA655C29D094EA050F08BFAA
:10F3500090EA020F05D054EA000C04BF194610468B
:10F3600030BD91EA030F1EBF0021002030BD5FEACF
:10F37000545C05D14000494128BF41F0004130BDF7
:10F3800014F580043CBF01F5801130BD01F000454B
:10F3900045F0FE4141F470014FF0000030BD7FEABE
:10F3A000645C1ABF194610467FEA655C1CBF0B46B9
:10F3B000024650EA013406BF52EA033591EA030FD0
:10F3C00041F4002130BD00BF90F0000F04BF0021C8
:10F3D000704730B54FF4806404F132044FF00005FB
:10F3E0004FF0000150E700BF90F0000F04BF002174
:10F3F000704730B54FF4806404F1320410F00045DA
:10F4000048BF40424FF000013EE700BF42004FEAD4
:10F41000E2014FEA31014FEA02701FBF12F07F4351
:10F4200093F07F4F81F06051704792F0000F14BF4E
:10F4300093F07F4F704730B54FF4607401F0004592
:10F4400021F0004120E700BF50EA010208BF7047E9
:10F4500030B54FF000050AE050EA010208BF7047DE
:10F4600030B511F0004502D5404261EB41014FF447
:10F47000806404F132045FEA915C3FF4DCAE4FF04B
:10F4800003025FEADC0C18BF03325FEADC0C18BF32
:10F49000033202EBDC02C2F1200300FA03FC20FA83
:10F4A00002F001FA03FE40EA0E0021FA02F11444D0
:10F4B000C1E600BF70B54FF0FF0C4CF4E06C1CEAE5
:10F4C00011541DBF1CEA135594EA0C0F95EA0C0F5A
:10F4D00000F0DEF82C4481EA030621EA4C5123EACD
:10F4E0004C5350EA013518BF52EA033541F48011FC
:10F4F00043F4801338D0A0FB02CE4FF00005E1FBAF
:10F5000002E506F00042E0FB03E54FF00006E1FBF8
:10F5100003569CF0000F18BF4EF0010EA4F1FF043B
:10F52000B6F5007F64F5407404D25FEA4E0E6D417B
:10F5300046EB060642EAC62141EA55514FEAC5208C
:10F5400040EA5E504FEACE2EB4F1FD0C88BFBCF508
:10F55000E06F1ED8BEF1004F08BF5FEA500E50F1B9
:10F56000000041EB045170BD06F0004646EA01017F
:10F5700040EA020081EA0301B4EB5C04C2BFD4EBB1
:10F580000C0541EA045170BD41F480114FF0000EAA
:10F59000013C00F3AB8014F1360FDEBF002001F018
:10F5A000004170BDC4F10004203C35DA0C341BDC92
:10F5B00004F11404C4F1200500FA05F320FA04F064
:10F5C00001FA05F240EA020001F0004221F0004198
:10F5D00010EBD37021FA04F642EB06015EEA430E0B
:10F5E00008BF20EAD37070BDC4F10C04C4F120053B
:10F5F00000FA04F320FA05F001FA04F240EA0200EE
:10F6000001F0004110EBD37041F100015EEA430EBE
:10F6100008BF20EAD37070BDC4F1200500FA05F2DE
:10F620004EEA020E20FA04F301FA05F243EA02035D
:10F6300021FA04F001F0004121FA04F220EA02006C
:10F6400000EBD3705EEA430E08BF20EAD37070BDB2
:10F6500094F0000F0FD101F00046400041EB010192
:10F6600011F4801F08BF013CF7D041EA060195F074
:10F67000000F18BF704703F00046520043EB03032E
:10F6800013F4801F08BF013DF7D043EA060370471B
:10F6900094EA0C0F0CEA135518BF95EA0C0F0CD026
:10F6A00050EA410618BF52EA4306D1D181EA03016C
:10F6B00001F000414FF0000070BD50EA410606BF66
:10F6C0001046194652EA430619D094EA0C0F02D1AB
:10F6D00050EA013613D195EA0C0F05D152EA0336F0
:10F6E0001CBF104619460AD181EA030101F000410E
:10F6F00041F0FE4141F470014FF0000070BD41F057
:10F70000FE4141F4780170BD70B54FF0FF0C4CF430
:10F71000E06C1CEA11541DBF1CEA135594EA0C0F4F
:10F7200095EA0C0F00F0A7F8A4EB050481EA030E9C
:10F7300052EA03354FEA013100F088804FEA033383
:10F740004FF0805545EA131343EA12634FEA022251
:10F7500045EA111545EA10654FEA00260EF0004112
:10F760009D4208BF964244F1FD0404F5407402D264
:10F770005B084FEA3202B61A65EB03055B084FEAF5
:10F7800032024FF480104FF4002CB6EB020E75EBF2
:10F79000030E22BFB61A754640EA0C005B084FEA1A
:10F7A0003202B6EB020E75EB030E22BFB61A754697
:10F7B00040EA5C005B084FEA3202B6EB020E75EBE2
:10F7C000030E22BFB61A754640EA9C005B084FEA5A
:10F7D0003202B6EB020E75EB030E22BFB61A754667
:10F7E00040EADC0055EA060E18D04FEA051545EA56
:10F7F00016754FEA06164FEAC30343EA52734FEAFF
:10F80000C2025FEA1C1CC0D111F4801F0BD141EA77
:10F8100000014FF000004FF0004CB6E711F4801FDC
:10F8200004BF01430020B4F1FD0C88BFBCF5E06FBC
:10F830003FF6AFAEB5EB030C04BFB6EB020C5FEACC
:10F84000500C50F1000041EB045170BD0EF0004E21
:10F850004EEA113114EB5C04C2BFD4EB0C0541EA53
:10F86000045170BD41F480114FF0000E013C90E650
:10F8700045EA060E8DE60CEA135594EA0C0F08BF14
:10F8800095EA0C0F3FF43BAF94EA0C0F0AD150EA13
:10F8900001347FF434AF95EA0C0F7FF425AF1046A6
:10F8A00019462CE795EA0C0F06D152EA03353FF4CE
:10F8B000FDAE1046194622E750EA410618BF52EA4B
:10F8C00043067FF4C5AE50EA41047FF40DAF52EA1F
:10F8D00043057FF4EBAE12E74FF0FF3C06E000BFBC
:10F8E0004FF0010C02E000BF4FF0010C4DF804CDC9
:10F8F0004FEA410C7FEA6C5C4FEA430C18BF7FEA89
:10F900006C5C1BD001B050EA410C0CBF52EA430CB6
:10F9100091EA030F02BF90EA020F0020704710F136
:10F92000000F91EA030F58BF994208BF90422CBFC5
:10F93000D8176FEAE37040F0010070474FEA410CBE
:10F940007FEA6C5C02D150EA013C07D14FEA430CDC
:10F950007FEA6C5CD6D152EA033CD3D05DF8040B4D
:10F96000704700BF8446104662468C46194663467F
:10F9700000E000BF01B5FFF7B7FF002848BF10F156
:10F98000000F01BD4DF808EDFFF7F4FF0CBF01209B
:10F9900000205DF808FB00BF4DF808EDFFF7EAFF17
:10F9A00034BF012000205DF808FB00BF4DF808EDD2
:10F9B000FFF7E0FF94BF012000205DF808FB00BFC7
:10F9C0004DF808EDFFF7CEFF94BF012000205DF851
:10F9D00008FB00BF4DF808EDFFF7C4FF34BF01205E
:10F9E00000205DF808FB00BF4FEA410212F500124B
:10F9F00015D211D56FF47873B3EB625212D94FEA76
:10FA0000C12343F0004343EA505311F0004F23FA5F
:10FA100002F018BF404270474FF00000704750EAB4
:10FA2000013005D111F0004008BF6FF00040704771
:10FA30004FF00000704700BF4FEA4102B2F1E043CF
:10FA400024BFB3F5001CDCF1FE5C0DD901F0004CC5
:10FA50004FEAC0024CEA5070B2F1004F40EB830015
:10FA600008BF20F00100704711F0804F21D113F141
:10FA70003872BCBF01F00040704741F480114FEA7A
:10FA80005252C2F11802C2F1200C10FA0CF320FA03
:10FA900002F018BF40F001004FEAC1234FEAD32320
:10FAA00003FA0CFC40EA0C0023FA02F34FEA43038A
:10FAB000CCE77FEA625307D150EA01331EBF4FF013
:10FAC000FE4040F44000704701F0004040F0FE402E
:10FAD00040F40000704700BF80F0004002E000BF2B
:10FAE00081F0004142001FBF5FEA410392EA030F29
:10FAF0007FEA226C7FEA236C6AD04FEA1262D2EB73
:10FB00001363C1BFD218414048404140B8BF5B4277
:10FB1000192B88BF704710F0004F40F4000020F010
:10FB20007F4018BF404211F0004F41F4000121F026
:10FB30007F4118BF494292EA030F3FD0A2F1010270
:10FB400041FA03FC10EB0C00C3F1200301FA03F1AE
:10FB500000F0004302D5494260EB4000B0F5000FD1
:10FB600013D3B0F1807F06D340084FEA310102F190
:10FB70000102FE2A51D2B1F1004F40EBC25008BF42
:10FB800020F0010040EA03007047490040EB00000C
:10FB900010F4000FA2F10102EDD1B0FA80FCACF13B
:10FBA000080CB2EB0C0200FA0CF0AABF00EBC2503A
:10FBB00052421843BCBFD0401843704792F0000F28
:10FBC00081F4000106BF80F400000132013BB5E77B
:10FBD0004FEA41037FEA226C18BF7FEA236C21D0F1
:10FBE00092EA030F04D092F0000F08BF0846704756
:10FBF00090EA010F1CBF0020704712F07F4F04D124
:10FC0000400028BF40F00040704712F100723CBF36
:10FC100000F50000704700F0004343F0FE4040F460
:10FC2000000070477FEA226216BF08467FEA23631E
:10FC30000146420206BF5FEA412390EA010F40F409
:10FC4000800070474FF0000304E000BF10F0004355
:10FC500048BF40425FEA000C08BF704743F096433C
:10FC600001464FF000001CE050EA010208BF704757
:10FC70004FF000030AE000BF50EA010208BF7047DE
:10FC800011F0004302D5404261EB41015FEA010CF3
:10FC900002BF84460146002043F0B64308BFA3F1EB
:10FCA0008053A3F50003BCFA8CF2083AA3EBC253CD
:10FCB00010DB01FA02FC634400FA02FCC2F12002EC
:10FCC000BCF1004F20FA02F243EB020008BF20F023
:10FCD0000100704702F1200201FA02FCC2F1200289
:10FCE00050EA4C0021FA02F243EB020008BF20EA7E
:10FCF000DC7070474FF0FF0C1CEAD0521EBF1CEAAC
:10FD0000D15392EA0C0F93EA0C0F6FD01A4480EA99
:10FD1000010C400218BF5FEA41211ED04FF0006382
:10FD200043EA501043EA5111A0FB01310CF00040AE
:10FD3000B1F5000F3EBF490041EAD3715B0040EAD4
:10FD4000010062F17F02FD2A1DD8B3F1004F40EBA4
:10FD5000C25008BF20F00100704790F0000F0CF077
:10FD6000004C08BF49024CEA502040EA51207F3A3B
:10FD7000C2BFD2F1FF0340EAC250704740F4000016
:10FD80004FF00003013A5DDC12F1190FDCBF00F007
:10FD900000407047C2F10002410021FA02F1C2F1B5
:10FDA000200200FA02FC5FEA310040F1000053EA51
:10FDB0004C0308BF20EADC70704792F0000F00F09F
:10FDC000004C02BF400010F4000F013AF9D040EAA5
:10FDD0000C0093F0000F01F0004C02BF490011F439
:10FDE000000F013BF9D041EA0C018FE70CEAD15337
:10FDF00092EA0C0F18BF93EA0C0F0AD030F0004CB7
:10FE000018BF31F0004CD8D180EA010000F000406A
:10FE1000704790F0000F17BF90F0004F084691F028
:10FE2000000F91F0004F14D092EA0C0F01D1420262
:10FE30000FD193EA0C0F03D14B0218BF084608D12B
:10FE400080EA010000F0004040F0FE4040F4000075
:10FE5000704740F0FE4040F4400070474FF0FF0C08
:10FE60001CEAD0521EBF1CEAD15392EA0C0F93EA4F
:10FE70000C0F69D0A2EB030280EA010C49024FEAA1
:10FE8000402037D04FF0805343EA111143EA10135A
:10FE90000CF000408B4238BF5B0042F17D024FF412
:10FEA000000C8B4224BF5B1A40EA0C00B3EB510FED
:10FEB00024BFA3EB510340EA5C00B3EB910F24BFD6
:10FEC000A3EB910340EA9C00B3EBD10F24BFA3EB5B
:10FED000D10340EADC001B0118BF5FEA1C1CE0D123
:10FEE000FD2A3FF650AF8B4240EBC25008BF20F0D6
:10FEF000010070470CF0004C4CEA50207F32C2BF2A
:10FF0000D2F1FF0340EAC250704740F400004FF0C6
:10FF10000003013A37E792F0000F00F0004C02BFF7
:10FF2000400010F4000F013AF9D040EA0C0093F0C1
:10FF3000000F01F0004C02BF490011F4000F013B1B
:10FF4000F9D041EA0C0195E70CEAD15392EA0C0F83
:10FF500008D142027FF47DAF93EA0C0F7FF470AFBB
:10FF6000084676E793EA0C0F04D14B023FF44CAFFE
:10FF700008466EE730F0004C18BF31F0004CCAD193
:10FF800030F000427FF45CAF31F000437FF43CAFCF
:10FF90005FE700BF4FF0FF3C06E000BF4FF0010CF1
:10FFA00002E000BF4FF0010C4DF804CD4FEA4002D3
:10FFB0004FEA41037FEA226C18BF7FEA236C11D01D
:10FFC00001B052EA530C18BF90EA010F58BFB2EBD0
:10FFD000030088BFC81738BF6FEAE17018BF40F050
:10FFE000010070477FEA226C02D15FEA402C05D104
:10FFF0007FEA236CE4D15FEA412CE1D05DF8040B89
:020000021000EC
:10000000704700BF844608466146FFE70FB5FFF71B
:10001000C9FF002848BF10F1000F0FBD4DF808EDD3
:10002000FFF7F4FF0CBF012000205DF808FB00BFC4
:100030004DF808EDFFF7EAFF34BF012000205DF81E
:1000400008FB00BF4DF808EDFFF7E0FF94BF01206B
:1000500000205DF808FB00BF4DF808EDFFF7D2FF68
:1000600094BF012000205DF808FB00BF4DF808EDAB
:10007000FFF7C8FF34BF012000205DF808FB00BF78
:100080004FEA4002B2F1FE4F0FD34FF09E03B3EBA5
:1000900012620DD94FEA002343F0004310F0004FE5
:1000A00023FA02F018BF404270474FF0000070473B
:1000B00012F1610F01D1420205D110F0004008BFDA
:1000C0006FF0004070474FF00000704742000ED2C2
:1000D000B2F1FE4F0BD34FF09E03B3EB126209D483
:1000E0004FEA002343F0004323FA02F070474FF039
:1000F0000000704712F1610F01D1420202D14FF0AE
:10010000FF3070474FF00000704700BF0B460146BC
:10011000184600F001B800BF13460A460146022007
:1001200000F0C0BE014B1868704700BF8097FF1FEA
:1001300070B50F4E0F4D761BB61018BF002405D0BA
:10014000013455F8043B9847A642F9D10A4E0B4DAD
:10015000761B03F0E3FBB61018BF002406D0013471
:1001600055F8043B9847A642F9D170BD70BD00BF59
:1001700028390100283901003C39010028390100E3
:10018000024B0146186800F00BB800BF8097FF1FB4
:10019000024B0146186800F049BF00BF8097FF1F5F
:1001A0002DE9F04F01F10B05162D83B0064640F204
:1001B0009F8035F0070500F1BF80A94200F2BC80A6
:1001C00000F058FBB5F5FC7FC0F09C826B0A00F094
:1001D000BA80042B00F28381A80900F1390E4FEA9E
:1001E0004E033830C44F07EB8303A3F108015C686A
:1001F000A14207D1ACE0002A80F2AC80E468A142C1
:1002000000F0A680636823F003035A1B0F2AF2DD77
:10021000B9493C6901F1080E744500F0B381636887
:1002200023F003035A1B0F2A00F39981002AC1F817
:1002300014E0C1F810E080F29E80B3F5007F80F0FA
:100240006781DB0803F1010C01229B1002FA03F322
:100250004A6851F83C80C4F8088001EBCC091A4385
:10026000A9F10803E3604A6041F83C40C8F80C403B
:10027000831001249C40944200F28A80144206D1EB
:1002800020F003006400144200F10400FAD007EBF0
:10029000C009CC468046DCF80C108C4507D173E1D0
:1002A000002A80F28181C9688C4500F06D814B681D
:1002B00023F003035A1B0F2AF2DD0C46D1F80CC0C1
:1002C00054F8088F4B1945F001054D6042F00101CB
:1002D000C8F80CC03046CCF808807B613B61C3F89D
:1002E0000CE0C3F808E059609A5000F0C5FA1FE02E
:1002F000102921D800F0BEFA1025062302207E4FD7
:1003000007EB8303A3F108025C68944200F0458187
:100310006368E168A56823F00303234430465A6804
:10032000E96042F001028D605A6000F0A5FA0834DD
:10033000204603B0BDE8F08F00240C232046336034
:1003400003B0BDE8F08F80234FF0400E3F2049E717
:1003500070465DE72344E1685A68A56842F00102EF
:10036000E96030468D605A6000F086FA0834204615
:1003700003B0BDE8F08F234430465A6842F00102D2
:100380005A6000F079FA0834204603B0BDE8F08FD7
:10039000BC68636823F00308A84504D3C5EB0803D1
:1003A0000F2B00F38C80554BDFF860911A68D9F859
:1003B000003001332A4404EB080A00F0608102F5A2
:1003C00080520F3222F47F6222F00F021146304633
:1003D000019200F04BFCB0F1FF3F8346019A00F020
:1003E0005881824500F2FC80454B1968DA4511447A
:1003F000196000F05381D9F80000DFF810E10130F6
:100400001BBFCAEB0B0A5144CEF800B019601BF0B9
:10041000070100F01781C1F10800C1F58051834444
:1004200008315A44C2F30B02C2EB01094946304677
:10043000019300F01BFC431C019B00F03F81CBEBC0
:1004400000024A4442F001021968C7F808B0494462
:10045000BC42CBF804201960DFF8A49016D0B8F1A4
:100460000F0F40F2FD806268A8F10C0323F0070330
:10047000E01802F001024FF0050E1A430F2B6260E4
:10048000C0F804E0C0F808E000F21C811D4BBC6815
:100490001A68914288BF19601B4B1A6891426268C2
:1004A00088BF196022F003029542A2EB050301D830
:1004B0000F2B04DC304600F0DFF9002438E7621926
:1004C00043F0010345F0010565603046BA605360B2
:1004D00000F0D2F90834204603B0BDE8F08F142BA9
:1004E00071D9542B00F2A480280B00F16F0E4FEA53
:1004F0004E036E3076E600BF8497FF1F34A2FF1FC5
:1005000038A2FF1F30A2FF1F2CA2FF1F909BFF1FCE
:100510005A0A042A5ED9142A00F2B38002F15C015F
:1005200049005B3207EB810C57F82110DFF8DC81C2
:10053000ACF1080C8C4500F088804A6822F0030278
:10054000934202D289688C45F7D1D1F80CC07A6801
:10055000C4F80CC0A160CCF80840CC6088E66319F0
:1005600042F0010745F00105656030464B610B61C3
:10057000C3F80CE0C3F808E05F609A50083400F05C
:100580007BF9D5E64A6873E608F1010818F0030F15
:100590000CF1080C7FF47FAE30E0DC68A34208BFAA
:1005A00002303FF435AEB3E60B440C465A68C968D6
:1005B00054F8085F42F001025A603046E9608D60ED
:1005C00000F05AF9B4E603F15C0E03F15B004FEA68
:1005D0004E0307E69A0902F1390149003832A1E7D2
:1005E000BC424A4B3FF400AF9C68626822F00302B1
:1005F0005AE759F80839994540F0828010F0030F06
:1006000000F1FF30F5D17B6823EA04037B606400CE
:100610009C423FF6BDAE002C3FF4BAAE1C424046B1
:100620007FF435AE64001C4200F10400FAD02EE6DF
:10063000B3F5AA7F18D8E80B00F1780E4FEA4E0305
:100640007730CFE54FF48051EBE60121D8F8043044
:10065000921001FA02F21A43C8F80420614677E7C3
:100660000123CBF8043025E740F25452934220D8BE
:10067000A80C00F17D0E4FEA4E037C30B2E510323B
:10068000A4E6542A26D81A0B02F16F0149006E32F3
:1006900048E7BC68626822F0030205E7CAF30B0072
:1006A00000287FF4A8AE4244BB6842F001025A60C1
:1006B000ECE6FE234FF07F0E7E2093E501224FF003
:1006C0000009C1E604F10801304600F0AFFCD9F89A
:1006D0000010DBE6B2F5AA7F05D8DA0B02F178014B
:1006E000490077321EE740F254518A4205D89A0CED
:1006F00002F17D0149007C3214E7FE217E2211E7E0
:100700007B6884E7E808431C5B00F8E58497FF1FDB
:100710008842F0B50DD98B1898420AD28118002A68
:1007200051D09A1A13F8014D01F8014D9342F9D1B5
:10073000F0BD0F2A48D941EA00039B0746D100F1DA
:10074000100401F11003154653F8106C44F8106CB6
:1007500053F80C6C44F80C6C53F8086C44F8086CB3
:10076000103D53F8046C44F8046C0F2D03F1100392
:1007700004F11004E8D8A2F1100323F00F0302F0F3
:100780000F0E1033BEF1030F1944034421D91E1F6D
:100790000D467446043C55F8047B46F8047F032C50
:1007A000F8D8AEF1040424F00304043423442144B3
:1007B00002F0030262B1013B0A4411F8014B03F855
:1007C000014F8A42F9D1F0BD0346F3E70346F2E751
:1007D000F0BD7246EEE700BF70B4840746D0541EE9
:1007E000002A41D0CDB2034602E0621EE4B31446B3
:1007F00003F8015B9A07F8D1032C2ED9CDB245EA54
:1008000005250F2C45EA054519D903F110022646A6
:10081000103E0F2E42F8105C42F80C5C42F8085C67
:1008200042F8045C02F11002F2D8A4F1100222F0A6
:100830000F0204F00F041032032C13440DD91E468E
:100840002246043A032A46F8045BFAD8221F22F013
:1008500003020432134404F003042CB1C9B21C4453
:1008600003F8011BA342FBD170BC7047144603463A
:10087000C2E700BF704700BF704700BF024B0A4687
:100880000146186800F002B88097FF1F2DE9F04F6D
:10089000174683B0002900F0C1800E46814607F15B
:1008A0000B05FFF7E7FF56F804EC162D2EF00304B6
:1008B000A6F1080840D810221546AF4241D894420C
:1008C00075DAC94B996808EB04008842416800F06A
:1008D000D98021F0010303445B68DB077DD51EF05E
:1008E000010F35D039464846FFF75AFC0746E0B1BC
:1008F00056F8043C23F001034344A0F108029A4255
:1009000000F04481221F242A00F23181132A00F2D0
:100910000481034632461168196051685960926833
:100920009A603146484600F081FB4846FFF7A4FF35
:10093000384603B0BDE8F08F25F00705002D2A46A4
:10094000BBDA0C230020C9F8003003B0BDE8F08FFB
:1009500056F8083CC3EB080ADAF8043023F0030C1D
:1009600004EB0C039342BDDB5746DAF80C1057F842
:10097000080F221F242AC160886000F21781132A01
:1009800040F212813168CAF808107168CAF80C1078
:100990001B2A00F22B8108360AF11002316811601F
:1009A00071685160B16891603E461C46D046631B39
:1009B0000F2B1DD8D8F8043003F00103234344441F
:1009C000C8F80430636843F0010363604846FFF7EA
:1009D00053FF304603B0BDE8F08F21F003012144FE
:1009E000914221DBC36882680C46D3609A60DEE7DF
:1009F000D8F8042008EB050102F00102154343F08A
:100A000001020B44C8F804504A605A6842F00102DF
:100A100008315A60484600F009FBD7E7114603B099
:100A2000BDE8F04FFFF7BCBB1EF0010F7FF45AAFDB
:100A300056F8083CC3EB080ADAF8043023F0030C3C
:100A400001EB0C0E96458BDBC36882685746D3607A
:100A50009A6057F8081FDAF80C30CB60221F242A5E
:100A6000996000F29980132A62D93368CAF8083075
:100A70007368CAF80C301B2A00F2A08008360AF10D
:100A8000100356E021F0030BA34405F11000834549
:100A900059DA1EF0010F7FF425AF56F8081CC1EBA0
:100AA000080ADAF8041021F0030CE34458453FF734
:100AB00057AF5746DAF80C1057F8080F221F242AB0
:100AC000C160886000F2B480132A40F2A5803168CA
:100AD000CAF808107168CAF80C101B2A00F2AF801F
:100AE00008360AF110023168116071685160B1680E
:100AF00091600AEB0501C5EB0B0242F0010299601F
:100B00004A60DAF8043003F001031D434846CAF88E
:100B10000450FFF7B1FE38465CE733680360736842
:100B200043601B2A27D800F1080306F10802F2E609
:100B30003B4632681A6072685A60B2689A603E46F4
:100B40007446D04633E708EB0501C5EB0B0B4BF0C1
:100B5000010299604A6056F8043C03F001031D430A
:100B6000484646F8045CFFF787FE304632E73146D8
:100B7000FFF7CEFDD5E6B3688360F368C360242A2F
:100B800028D000F1100306F11002C4E650F8043C2E
:100B900023F003031C440AE7314638467446D04626
:100BA000FFF7B6FD3E4602E73A46F7E631463846DD
:100BB0001C46D046FFF7ACFD3E46F8E6B368CAF8DF
:100BC0001030F368CAF81430242A1BD010360AF10A
:100BD0001803AEE7336903617369436106F11802D4
:100BE00000F1180397E600BF8497FF1FB168CAF8A9
:100BF0001010F168CAF81410242A0FD010360AF128
:100C00001802CBE63369CAF818307369CAF81C3089
:100C100018360AF120038CE73A4664E73269CAF8CD
:100C200018207269CAF81C2018360AF12002B5E6AD
:100C3000314638460193FFF76BFD019B59E7B168D8
:100C4000CAF81010F168CAF81410242A03D010361C
:100C50000AF1180247E73269CAF818207269CAF81F
:100C60001C2018360AF120023DE700BF38B5074CBA
:100C70000023054608462360FBF7E0FE431C00D036
:100C800038BD2368002BFBD02B6038BD94A3FF1F19
:100C9000FFFFFFFFFFFFFFFFFFFFFFFFFFFFFFFF64
:100CA000FFFFFFFFFFFFFFFFFFFFFFFFFFFFFFFF54
:100CB000FFFFFFFFFFFFFFFFFFFFFFFFFFFFFFFF44
:100CC00090F800F06DE9024520F007016FF0000C8C
:100CD00010F0070491F820F040F049804FF0000434
:100CE0006FF00700D1E9002391F840F000F108000F
:100CF00082FA4CF2A4FA8CF283FA4CF3A2FA8CF347
:100D00004BBBD1E9022382FA4CF200F10800A4FAAD
:100D10008CF283FA4CF3A2FA8CF3E3B9D1E9042301
:100D200082FA4CF200F10800A4FA8CF283FA4CF338
:100D3000A2FA8CF37BB9D1E9062301F1200182FAF2
:100D40004CF200F10800A4FA8CF283FA4CF3A2FAF8
:100D50008CF3002BC6D0002A04BF04301A4612BA06
:100D6000B2FA82F2FDE8024500EBD2007047D1E909
:100D7000002304F00305C4F100004FEAC50514F098
:100D8000040F91F840F00CFA05F562EA05021CBF69
:100D900063EA050362464FF00004A9E7002A41D048
:100DA00040EA010313F00303F0B425D1032A23D949
:100DB00004680D68AC421FD1043A35D0A4F1013566
:100DC00025EA040414F0803F31D1071D0D1D0DE00C
:100DD00057F8043B0E68A3F10134B34224EA03043C
:100DE0000AD1043A20D014F0803F23D1032A2946A7
:100DF000384605F10405EBD803780C789C4202F1E3
:100E0000FF320CD182B114B916E06AB17BB110F88F
:100E1000013F11F8014FA34202F1FF32F5D0181B38
:100E2000F0BC7047104670471046F0BC704718463B
:100E3000F0BC70470020F3E72046F1E740EA0103E9
:100E40009B0770B42BD1032A29D90C4603462146AF
:100E500054F8046BA6F1013525EA060515F0803F2C
:100E600006D1043A032A43F8046B2146EFD8A2B115
:100E70000C781C70013A013301313CB16AB111F8B0
:100E8000014B03F8014B013A002CF7D12AB11A4467
:100E9000002103F8011B9A42FBD170BC7047034646
:100EA000E5E700BF2DE9F047254C2568D5F8484116
:100EB0000646884692469946C4B360681F2817DCE8
:100EC000431C76B104EB80050122C5F888A0D4F854
:100ED000881182401143022EC4F88811C5F8089188
:100EE0001ED00230636044F820800020BDE8F08707
:100EF000144B03B34FF4C870FFF742F90446D0B166
:100F0000D5F84831002780E88800C5F848413846C0
:100F10000123C4F88871C4F88C71002EE1D0D1E7A8
:100F2000D4F88C110A43C4F88C21DAE705F5A674CD
:100F3000C5F84841C1E74FF0FF30BDE8F08700BF7A
:100F40001839010081010100024B13B1024800F081
:100F500005B8704700000000690F0100002301463A
:100F60001A461846FFF79EBF38B5074D074C2C1B95
:100F7000A41005D0013C55F8043D9847002CF9D148
:100F8000BDE8384002F0DABC0000000000000000BC
:100F9000F8B5234F0C460646FFF76CFCBB685D684E
:100FA00025F00305291B01F6EF7121F47F6121F083
:100FB0000F01A1F58054B4F5805F07DB00213046B6
:100FC000FFF754FEBB682B44984204D03046FFF72D
:100FD00053FC0020F8BD61423046FFF747FE013068
:100FE0000DD0104BBA6819682D1B45F0010530462D
:100FF000091B55601960FFF73FFC0120F8BD002177
:101000003046FFF733FEBA68831A0F2BDEDD064C3D
:101010000449246843F00103001B53600860D5E7CE
:101020008497FF1F38A2FF1F909BFF1F002945D008
:101030002DE9F0410D468046FFF71CFC55F8047C75
:101040006A4927F00103A5F10804E2188E68506888
:10105000B24220F0030062D0FE0750600BD455F876
:10106000087CE41B01F1080EA56875453B446FD070
:10107000E768EF60BD6015186D68ED0742D543F075
:1010800001026260E350B3F5007F18D2DB085A1CFE
:101090004D6851F83270A76001209B1000FA03F3ED
:1010A00001EBC2001D430838E0604D6041F832405A
:1010B000FC604046BDE8F041FFF7DEBB70475A0ACE
:1010C000042A53D89A0902F139077F0002F1380542
:1010D00001EB870051F827204449083890424DD051
:1010E000516821F003018B4202D292689042F7D1FD
:1010F000D068E060A2608460D4604046BDE8F04102
:10110000FFF7BABB95683A4FBD4203443FD0D06861
:10111000E86043F0010285606260E350B3E7FF07D7
:10112000034407D455F8082CA41A1344A068E268B5
:10113000C26090602F4A126843F0010093426060E1
:101140008C60B6D32C4B40461968FFF721FFB0E7FF
:1011500011184968C90744D49168D268CA60034429
:1011600043F0010091606060E350A2E7142A17D8B1
:1011700002F15C077F0002F15B05A9E7AA104B684A
:10118000012505FA02F213434B600246B1E743F032
:1011900001024C610C61E560A5606260E35088E784
:1011A000542A06D81A0B02F16F077F0002F16E0570
:1011B0008EE7B2F5AA7F06D8DA0B02F178077F0036
:1011C00002F1770584E740F25450824206D89A0C27
:1011D00002F17D077F0002F17C0579E7FE277E257D
:1011E00076E743F001026260E35062E78497FF1FF5
:1011F0008C97FF1F8C9BFF1F34A2FF1F00007805F8
:101200003408540B800C3C0F5C12E015FA19141EC4
:101210006022AC265C2B0C30BC34023AFF3FFFFF4F
:10122000FDFFFFFFFBFFFFFFF8FFFFFFFDFFFFFFDD
:10123000FBFFFFFFF8FFFFFFFDFFFFFFFAFFFFFFD0
:10124000F7FFFFFFFDFFFFFFFBFFFFFFF7FFFFFFC4
:10125000FCFFFFFFFBFFFFFFF7FFFFFFFDFFFFFFAF
:10126000FAFFFFFFF7FFFFFFFDFFFFFFFBFFFFFFA1
:10127000F8FFFFFFFDFFFFFFFBFFFFFFF8FFFFFF92
:10128000FDFFFFFFFAFFFFFFF7FFFFFFFCFFFFFF80
:10129000FBFFFFFFF7FFFFFFFDFFFFFFFBFFFFFF70
:1012A000F7FFFFFFFDFFFFFFFAFFFFFFF7FFFFFF65
:1012B000FDFFFFFFFBFFFFFFF7FFFFFFFDFFFFFF4E
:1012C000FBFFFFFFF7FFFFFFFDFFFFFFFAFFFFFF41
:1012D000F7FFFFFFFDFFFFFFFAFFFFFFF8FFFFFF34
:1012E000FDFFFFFFFAFFFFFFF7FFFFFFFDFFFFFF1F
:1012F000FAFFFFFFF7FFFFFFFDFFFFFFFAFFFFFF12
:10130000F8FFFFFFFDFFFFFFFAFFFFFFF8FFFFFF02
:10131000FDFFFFFFFAFFFFFFF7FFFFFFFCFFFFFFEF
:10132000FBFFFFFFF7FFFFFFFDFFFFFFFAFFFFFFE0
:10133000F7FFFFFFFDFFFFFFFAFFFFFFF7FFFFFFD4
:10134000FEFFFFFFFBFFFFFFF8FFFFFFFEFFFFFFBA
:10135000FBFFFFFFF8FFFFFFFDFFFFFFFAFFFFFFAF
:10136000F7FFFFFFFCFFFFFFFAFFFFFFF7FFFFFFA5
:10137000FCFFFFFFFAFFFFFFF7FFFFFFFDFFFFFF8F
:10138000FAFFFFFFF7FFFFFFFDFFFFFFF9FFFFFF82
:10139000F7FFFFFFFDFFFFFFF9FFFFFFF7FFFFFF75
:1013A000FDFFFFFFFAFFFFFFF7FFFFFFFDFFFFFF5E
:1013B000FAFFFFFFF7FFFFFFFDFFFFFFFAFFFFFF51
:1013C000F6FFFFFFFDFFFFFFFAFFFFFFF7FFFFFF45
:1013D000FEFFFFFFFBFFFFFFF7FFFFFFFEFFFFFF2B
:1013E000FBFFFFFFF7FFFFFFFDFFFFFFFAFFFFFF20
:1013F000F7FFFFFFFDFFFFFFFBFFFFFFF8FFFFFF12
:10140000FDFFFFFFFBFFFFFFF8FFFFFFFDFFFFFFFB
:10141000FAFFFFFFF7FFFFFFFCFFFFFFF9FFFFFFF2
:10142000F7FFFFFFFCFFFFFFF9FFFFFFF7FFFFFFE5
:10143000FDFFFFFFFAFFFFFFF7FFFFFFFDFFFFFFCD
:10144000FAFFFFFFF7FFFFFFFDFFFFFFF9FFFFFFC1
:10145000F6FFFFFFFDFFFFFFFAFFFFFFF7FFFFFFB4
:10146000101B0100EC1A0100C81A0100A41A0100A7
:10147000FC150100B8140100DC1401000015010086
:10148000D81501009414010020190100FC1101007D
:10149000501701000000580246056608540BD80E8C
:1014A0005C127017FC21F82A70305834DC37663A29
:1014B0008C3C803EFF3FFFFF000058024605660857
:1014C000540BD80E5C12E015FA19141E6022AC26DB
:1014D0005C2B0C30BC34023AFF3FFFFF0000900150
:1014E00020031405D0075A0AAC0DCC10B4146A18A6
:1014F000E81C342180252A2B70301437FF3FFFFF72
:101500000000C800F4018403140508072E091C0C10
:10151000D80EF811AE159619401F1C25F22B583421
:10152000FF3FFFFFFBFFFFFFF8FFFFFFF4FFFFFFA1
:10153000FAFFFFFFF7FFFFFFF4FFFFFFFDFFFFFFD5
:10154000F9FFFFFFF4FFFFFFFAFFFFFFF7FFFFFFC9
:10155000F4FFFFFFFCFFFFFFF7FFFFFFF4FFFFFFBC
:10156000FBFFFFFFF8FFFFFFF4FFFFFFFDFFFFFFA3
:10157000FAFFFFFFF4FFFFFFFDFFFFFFF9FFFFFF93
:10158000F4FFFFFFFDFFFFFFF8FFFFFFF4FFFFFF8A
:10159000FCFFFFFFF7FFFFFFF4FFFFFFFBFFFFFF75
:1015A000F8FFFFFFF4FFFFFFFCFFFFFFF7FFFFFF68
:1015B000F4FFFFFF40067805B004E803840320032E
:1015C000BC025802F40190012C01FA00C8009600F8
:1015D000640032001900FFFF00006400C8009001A1
:1015E000BC021A04DC059E07F609800CA00F241328
:1015F000A2174C1D5424442FFF3FFFFF0000FF03A0
:10160000FF07FF0BFF0FFF13FF17FF1BFF1FFF233A
:10161000FF27FF2BFF2FFF33FF37FF3BFF3FFFFF6E
:1016200001020101000101010201010201010101A8
:101630000101020101020101020101010000010298
:101640000101020101010100010201010201010089
:101650000202010201010201000202020102010173
:101660000200010202020102010100000002020266
:101670000102010101000002020201020100020256
:10168000020202020102000202010202020201023F
:101690000002020201020202010100020202020231
:1016A0000202010000020200020202020002010224
:1016B000020202020202000200020202020202020E
:1016C000FBFFFFFFF7FFFFFFF4FFFFFFFBFFFFFF45
:1016D000F7FFFFFFF4FFFFFFFDFFFFFFF7FFFFFF37
:1016E000F4FFFFFFFDFFFFFFF8FFFFFFF4FFFFFF29
:1016F000FAFFFFFFF7FFFFFFF4FFFFFFFBFFFFFF16
:10170000F7FFFFFFF4FFFFFFFBFFFFFFF7FFFFFF08
:10171000F4FFFFFFFBFFFFFFF7FFFFFFF4FFFFFFFB
:10172000FDFFFFFFF8FFFFFFF4FFFFFFFDFFFFFFDF
:10173000F8FFFFFFF4FFFFFFFDFFFFFFF8FFFFFFD4
:10174000F4FFFFFFFAFFFFFFF8FFFFFFF4FFFFFFCB
:101750000000D007800CD80E0010C012EC130C173C
:10176000FA19141E6022AC265C2B0C30BC34023AF1
:10177000FF3FFFFF00000000070000000C0000001A
:101780001000000013000000180000001C00000002
:1017900000000000070000000C0000001300000023
:1017A000180000001F0000002400000000000000DE
:1017B0000C000000180000002400000030000000B1
:1017C0003C0000004800000000000000FBFFFFFF9D
:1017D000F4FFFFFFEFFFFFFFE8FFFFFFE3FFFFFF67
:1017E000DCFFFFFF00000000F4FFFFFFE8FFFFFF4A
:1017F000DCFFFFFFD0FFFFFFC4FFFFFFB8FFFFFFCD
:10180000FBFFFFFFF8FFFFFFF4FFFFFFFAFFFFFF03
:10181000F7FFFFFFF4FFFFFFFDFFFFFFF9FFFFFFF3
:10182000F4FFFFFFFAFFFFFFF7FFFFFFF4FFFFFFEB
:10183000FCFFFFFFF7FFFFFFF4FFFFFFFBFFFFFFD2
:10184000F8FFFFFFF4FFFFFFFDFFFFFFFAFFFFFFC1
:10185000F4FFFFFFFBFFFFFFF8FFFFFFF4FFFFFFB9
:10186000FDFFFFFFF8FFFFFFF4FFFFFFFCFFFFFF9F
:10187000F7FFFFFFF4FFFFFFFBFFFFFFF8FFFFFF96
:10188000F4FFFFFFFCFFFFFFF7FFFFFFF4FFFFFF89
:10189000FBFFFFFFF8FFFFFFF6FFFFFFFAFFFFFF71
:1018A000F8FFFFFFF6FFFFFFFDFFFFFFFBFFFFFF5E
:1018B000F9FFFFFFFDFFFFFFF9FFFFFFF7FFFFFF4E
:1018C000FEFFFFFFFCFFFFFFF7FFFFFFFBFFFFFF38
:1018D000F8FFFFFFF6FFFFFFFCFFFFFFFAFFFFFF30
:1018E000F6FFFFFFFDFFFFFFFBFFFFFFF9FFFFFF1D
:1018F000FCFFFFFFFAFFFFFFF6FFFFFFFEFFFFFF0A
:10190000FCFFFFFFF7FFFFFFFBFFFFFFF8FFFFFFFD
:10191000F6FFFFFFFEFFFFFFFCFFFFFFF7FFFFFFEC
:101920000000580246056608540BA00FD417282360
:10193000F82A442F643284354038663A8C3C803E25
:10194000FF3FFFFF2C011301FA00E100C800AF00C8
:1019500096007D0064004B0032001900000000007A
:10196000CDCC4C3DCDCCCC3D9A99193ECDCC4C3E06
:101970000000803E9A99993E3333B33ECDCCCC3EA5
:101980006666E63EFBFFFFFFF7FFFFFFF6FFFFFF88
:10199000FBFFFFFFF7FFFFFFF6FFFFFFFBFFFFFF70
:1019A000F7FFFFFFF6FFFFFFFDFFFFFFFCFFFFFF5D
:1019B000F8FFFFFFFDFFFFFFFCFFFFFFF8FFFFFF4A
:1019C000FDFFFFFFFCFFFFFFF8FFFFFFFBFFFFFF37
:1019D000F7FFFFFFF6FFFFFFFBFFFFFFF7FFFFFF34
:1019E000F6FFFFFFFBFFFFFFFAFFFFFFF8FFFFFF20
:1019F000FCFFFFFFF9FFFFFFF8FFFFFFFDFFFFFF09
:101A0000FCFFFFFFF8FFFFFFFCFFFFFFFAFFFFFFF8
:101A1000F7FFFFFFFBFFFFFFF7FFFFFFF4FFFFFFF5
:101A2000FBFFFFFFF7FFFFFFF4FFFFFFFBFFFFFFE1
:101A3000F7FFFFFFF4FFFFFFFDFFFFFFF8FFFFFFD2
:101A4000F4FFFFFFFDFFFFFFF8FFFFFFF4FFFFFFC5
:101A5000FDFFFFFFF8FFFFFFF4FFFFFFFBFFFFFFAE
:101A6000F7FFFFFFF4FFFFFFFBFFFFFFF7FFFFFFA5
:101A7000F4FFFFFFFBFFFFFFF8FFFFFFF4FFFFFF97
:101A8000FCFFFFFFF9FFFFFFF4FFFFFFFDFFFFFF7C
:101A9000F8FFFFFFF4FFFFFFFCFFFFFFF7FFFFFF73
:101AA000F4FFFFFF00007805220B0410B414321974
:101AB000B01DFC214826FE29822D383126344637B8
:101AC000663A223DFF3FFFFF0000D007100E88134B
:101AD0003219AA1E282374275C2B442F64328435C4
:101AE0004038663A8C3C803EFF3FFFFF0000540BBD
:101AF000EC13FA1908201C253629EC2C0C302C3359
:101B0000E8357238663AF63B863D163FFF3FFFFFE9
:101B10000000CC10581BFC21AC26C62A7C2E383184
:101B2000F4334C36A438983A5A3C543D803E7A3FC0
:101B3000FF3FFFFFA41B01007E9CFF1F0000FF0F63
:101B4000329EFF1F0000FF0FF1560000701B0100C6
:101B50002C9EFF1F32005E0100000000000000000C
:101B60009156000054485200534E53004D415800C6
:101B7000544F5543482053454E5345004558545201
:101B80004120434F4E54524F4C4C455200000000F0
:101B900050495443482042454E4400004249544570
:101BA0000000000042524541544800FF7C1B0100E8
:101BB000969DFF1FF401A00F8C9DFF1FF401A00F45
:101BC0009D5600009C1B01003A9CFF1FBC025C124A
:101BD000109EFF1FBC025C12D5560000901B010036
:101BE000E09DFF1FF401A00F009CFF1FF401A00F58
:101BF000B9560000342501003C25010028250100CC
:101C00002C2501003025010094230100EC24010063
